:020000040800F2
:10000000F8270120430500088D040008E5070208D1
:100010009104000893040008950400080000000003
:10002000000000000000000000000000970400082D
:1000300099040008000000009B0400089D040008CB
:100040009F040008A1040008A3040008A5040008F8
:10005000A7040008A9040008AB040008AD040008C8
:10006000AF040008B1040008B3040008B504000898
:10007000B7040008B9040008BB040008BD04000868
:10008000BF040008C1040008C3040008C504000838
:10009000C7040008C9040008CB040008CD04000808
:1000A000CF040008D1040008D3040008D5040008D8
:1000B000D7040008D9040008DB040008DD040008A8
:1000C000DF040008E1040008E3040008E504000878
:1000D000E7040008E9040008EB040008ED04000848
:1000E000EF040008F1040008F3040008F504000818
:1000F000F7040008F9040008FB040008FD040008E8
:10010000FF040008010500080305000805050008B4
:1001100007050008090500080B0500080D05000883
:100120000F05000811050008130500081505000853
:1001300017050008190500081B0500081D05000823
:100140001F050008210500082305000825050008F3
:1001500027050008290500082B0500082D050008C3
:100160002F05000831050008330500083505000893
:1001700037050008390500083B0500083D05000863
:080180003F05000841050008DD
:10020000DECEA5ED02003078463430370000000025
:100210000000000000004441385F313431310000FB
:100220000000000000004170706C69636174696FC8
:100230006E00000000000000000000000000000050
:100240000000000000000503B300DAF7DECEA5EDE4
:100250000200307846343037000000000000000013
:10026000000053504C6174436F6E74726F6C6C6518
:1002700072004170706C69636174696F6E00000098
:10028000000000000000000000000000000000006E
:0802900000000000FE00DAF797
:100298000100020818000000610202080D000000B9
:1002A8008506020803000000C10C020806000000D1
:1002B8003110020809000000B5150208020000000C
:1002C800C1160208100000007D180208FF00000097
:1002D800BD1F02080C000000C9230208000000002E
:1002E8000526020805000000414C02081200000023
:1002F800694F02080A000000B15302080A00000012
:10030800655C020814000000F160020808000000A3
:100318000968020807000000B16E0208100000001A
:1003280099720208130000003984020813000000C3
:1003380045B10208160000000D0A03081700000066
:10034800114403081600000039450308170000008F
:080358000D5803081500000018
:100360002F49072291438D462E492F480A1A06D05D
:100370000722914381F30988022282F314882B48D3
:100380002B492C4A00F039F82B482C492C4A00F014
:1003900034F82C482C492D4A00F02FF82C482D49D0
:1003A0002D4A00F02AF82D482D492E4A00F025F854
:1003B0002D482E492E4A00F020F82E482E490022C2
:1003C00000F026F82D482E49091A082903DB0022DF
:1003D0000260043001601F481F49884205D002684E
:1003E000043003B4904703BCF7E700208646EC4690
:1003F00000200021234A9047FEE7884207D0521A86
:1004000005D0037801300B700131013AF9D1704702
:10041000884202D002700130FAE770471A487047EC
:10042000F8270120F82F0120F8270120C0BA03087F
:1004300088010020140200200000020800000208C9
:10044000E08B0308C0BA030888010020880100205F
:100450009C0500089C0500089C0500089C050008F8
:100460009C0500089C050008E08B0308E08B03084E
:10047000C0BA030814020020AC240120F824012093
:10048000F82401203D340208FFFFFFFFFEE7FEE7EE
:10049000FEE7FEE7FEE7FEE7FEE7FEE7FEE7FEE734
:1004A000FEE7FEE7FEE7FEE7FEE7FEE7FEE7FEE724
:1004B000FEE7FEE7FEE7FEE7FEE7FEE7FEE7FEE714
:1004C000FEE7FEE7FEE7FEE7FEE7FEE7FEE7FEE704
:1004D000FEE7FEE7FEE7FEE7FEE7FEE7FEE7FEE7F4
:1004E000FEE7FEE7FEE7FEE7FEE7FEE7FEE7FEE7E4
:1004F000FEE7FEE7FEE7FEE7FEE7FEE7FEE7FEE7D4
:10050000FEE7FEE7FEE7FEE7FEE7FEE7FEE7FEE7C3
:10051000FEE7FEE7FEE7FEE7FEE7FEE7FEE7FEE7B3
:10052000FEE7FEE7FEE7FEE7FEE7FEE7FEE7FEE7A3
:10053000FEE7FEE7FEE7FEE7FEE7FEE7FEE7FEE793
:10054000FEE71348854600F022F84EF68850CEF2BA
:100550000000016851F47001016000BF00BF00BFDE
:10056000F1EE100A50F04070E1EE100A4FF000007A
:1005700080F314884EF63C71CEF20001086850F00A
:1005800040700860034804490160FFF7E9BE704706
:0C0590000000022008ED00E00000000860
:020000040801F1
:1000000000000000000000000000000000000000F0
:1000100000000000000000000000000000000000E0
:100020000000000000000000000000000000015877
:10003000830035F4301E00000A830140014413F5AB
:100040003183014CF5330000F4030057000000F445
:1000500003011D000000094A004A0F5100980000EA
:100060000000AF00AF018F15008F16009617961B8A
:10007000430542048F21008F14FF680020F406F42A
:100080000220140092F407000064007F8301468080
:10009000007D420542044A0F710044236700206638
:1000A000042370004A0F524422680422AE009624B2
:1000B000AE019628AE02962CAE039630AE0496346E
:1000C000AE059638AE06963CAE07964045210C012B
:1000D0008200D40C4421F535F406F4024514600086
:1000E0002000EEF5358100EE0C018200EE0C45217A
:1000F000128100FEF40700006400DA8000576900F6
:100100002045154516554A0F52510045164A0F52C3
:100110005F009417AF00941BAF018000961E000093
:10012000648301400145131281011D44131E000028
:10013000648301400145131282012BF53180011DBA
:1001400070044A0F52096E012080014C60012001A9
:1001500055F5390009F53901092123140BFFFFFF7B
:10016000FFFFFFFFFFFFFFFFFFFFFFFFFFFFFFFF9F
:10017000FFFFFFFFFFFFFFFFFFFFFFFFFFFFFFFF8F
:10018000FFFFFFFFFFFFFFFFFFFFFFFFFFFFFFFF7F
:10019000FFFFFFFFFFFFFFFFFFFFFFFFFFFFFFFF6F
:020000040802F0
:1000000030B583B04FF0000400944FF0F80501952F
:10001000204621464FF007024FF0010302F06EFD2B
:1000200040F21420C2F2010040F21421C2F2000199
:100030004FF480324FF0020315F048FD4FF00600F8
:10004000294614F0A3FC4FF00300214640F2A10220
:10005000C0F6020203F056FD4FF0010040F2B1017C
:10006000C0F6020140F29102C0F6020203F04AFD1E
:100070004FF004004FF00501024610F0F1FB48F686
:10008000FC30C0F6030007F093FB03B030BD00BFA7
:1000900008B519B94FF0030015F082FB08BD00BF89
:1000A00008B5012903D14FF0010015F079FB08BD17
:1000B00008B54FF0060001F06DF808BD4FF00003E1
:1000C00003704FF004000870704700BF10B14FF08C
:1000D0000202027011B14FF004000870704700BFB7
:1000E00040F23421C2F201014FF00000086040F2FA
:1000F0004423C2F201034FF000021A8048605A8084
:1001000088609A80C860DA80704700BFA0F1020062
:10011000C0B2032814D869B140F23423C2F20103FB
:1001200003EB800003680B604FF0000111704FF08B
:10013000010070474FF0160313704FF00100704735
:100140004FF00000704700BF684620F007018D4661
:1001500001B441F21043C4F200034FF000021A60F0
:1001600040F23020C2F20100018801F101018BB29E
:100170000380FF2B38D94FF00002028040F2442365
:10018000C2F20103198831B140F61840C4F20200EE
:100190004FF01002028040F24423C2F2010359885A
:1001A00031B140F61840C4F202004FF0080202805C
:1001B00040F24423C2F20103998831B140F618405D
:1001C000C4F202004FF00402028040F24423C2F263
:1001D0000103D98800293FD040F61840C4F202003C
:1001E0004FF00202028037E040F24422C2F20102E4
:1001F0001088984206D140F61A42C4F202024FF02B
:100200001001118040F24420C2F2010042889A425B
:1002100006D140F61A40C4F202004FF008010180F6
:1002200040F24422C2F201029088984206D140F680
:100230001A42C4F202024FF00401118040F244203D
:10024000C2F20100C2889A4206D140F61A43C4F2B3
:1002500002034FF00201198001BC8546704700BFC0
:1002600038B540F29010C2F200004FF0010109F0E1
:10027000BDFE40F29810C2F200004FF0010109F0FB
:10028000E1FE40F28810C2F200004FF0010109F0D7
:1002900031FF42F20804CEF20404236843F0200048
:1002A000206040F24910C0F602004FF00F014FF0FD
:1002B000370200F04BFA43F64001C4F202010A682B
:1002C00042F020050D6041F20045C4F2000548F6F9
:1002D0004443C0F603031868286049F6E811C0F6E5
:1002E0000301C86915F018FC17A3D3E9002315F022
:1002F00057FE4FF000024FF00003C3F6F07315F005
:1003000009FD15F075FC41F22C42C4F20002108088
:100310004FF0000041F22843C4F20003188048F671
:100320004041C0F603010A6841F20C43C4F20003E5
:100330001A60298841F001022A80236860F345137E
:10034000236038BDAFF300808DEDB5A0F7C6D03E79
:1003500008B507EE901AA0F10200C0B2032822D817
:1003600040F23423C2F2010303EB8001C1ED007AB5
:100370009FED117A27EE870AFCEEC00A10EE903A44
:1003800099B240F24422C2F2010222F8103040F247
:100390002C23C2F201031A5C42B951B900F0FAFEF3
:1003A0004FF0010008BD4FF0000008BD4FF0010004
:1003B00008BD4FF0010008BD0000804338B5044679
:1003C0000D4603282BD84FF00003137099B100F0AD
:1003D000E1FE40F23422C2F2010202EB84034FF04C
:1003E0000000186040F24421C2F201014FF0000207
:1003F00021F814200BE040F24420C2F2010030F852
:10040000141021B920464FF0000100F0C3FE40F265
:100410002C23C2F201031D554FF0010038BD4FF0EF
:10042000000038BD38B50C461546032815D889B1EB
:1004300040F24421C2F2010131F810201AB14FF00C
:100440000100207002E000F083FE20704FF00003F6
:100450002B7002E04FF0160313704FF0000038BD10
:1004600038B50C46154603281AD899B140F24421F4
:10047000C2F2010131F810201AB14FF001002070D2
:1004800002E004F0CFFC20704FF000032B704FF01F
:10049000010038BD4FF0160313704FF0010038BD56
:1004A0004FF0000038BD00BF38B50C461546032894
:1004B0001ED8B9B140F24421C2F2010131F8102036
:1004C00002F1FF3399B2FE2903D84FF001002070EA
:1004D00002E004F0D7FC20704FF000022A704FF0C9
:1004E000010038BD4FF0160313704FF0010038BD06
:1004F0004FF0000038BD00BF38B50C461546032844
:100500001AD899B140F24421C2F2010131F8102009
:100510001AB14FF00100207002E004F09DFC207041
:100520004FF000032B704FF0010038BD4FF0160361
:1005300013704FF0010038BD4FF0000038BD00BF10
:1005400038B504460D46032828D899B110F036FA7C
:1005500040F23421C2F2010101EB84034FF00002AA
:100560001A6040F24420C2F201004FF0000120F86E
:1005700014100BE040F24423C2F2010333F81000E0
:1005800020B920464FF0000110F018FA40F22C2359
:10059000C2F201031D554FF0010038BD4FF00000BD
:1005A00038BD00BF48F65843C0F603031A684EF63C
:1005B0000C50CEF200000260FEE700BF08B5FFF766
:1005C000F1FF00BF51E8002FBFF35F8F41E8000348
:1005D000012B3FF4F7AF1046704700BF13461A4691
:1005E0002DE9F00F0B460C460D460E460F46884689
:1005F00089468A468B46092AC0F00780A0E8F80F92
:10060000A2F10902092ABFF4F9AF4FF0080303FB76
:1006100002F2144B1A44974600F020B800BF00BF06
:10062000046000F01BB800BF80E8300000F016B88E
:1006300080E8700000F012B880E8F00000F00EB81A
:1006400080E8F00100F00AB880E8F00300F006B896
:1006500080E8F00700F002B880E8F00FBDE8F00F86
:100660007047134618060208EFF311804FF080011F
:1006700081F3118870474FF0000000BF80F31188AC
:10068000704700BF30B440F20003C0F6000340F2F0
:100690008812C0F60002D01A4FEAA001B1F5C47F5B
:1006A00004D81346264A9A4201D324E0FEE7254D9A
:1006B000254C601B20F003054FF0000340F20002C0
:1006C000C2F2000240F20001C0F6000105F1040090
:1006D000C5F380045D589D5003F10403834226D185
:1006E00009E05C589C5003F104035C58D45003F1BA
:1006F00004038342F5D14EF60853CEF2000340F2D4
:100700000002C2F200021A604FF0B501CBF26B1189
:1007100042F2F840C2F2010001604EF61453CEF2EC
:1007200000031A6842F01001196030BC7047002CB9
:10073000D7D05C589C5003F104038342D1D1DAE74F
:1007400000000008040000088B01000810B40346F4
:1007500000283ED002F1100440F20000C2F2000076
:1007600040F82430002A0ADA12F10C0F35DB02F1CE
:100770000C024EF61850CEF2000011542DE04EF24D
:100780000014CEF200040F299CBF0901C9B24EF239
:100790000043CEF20003D1541146002AB8BF02F143
:1007A0001F014FEA611004EB80014FF01F03C8F2F4
:1007B00000031340002B05DA03F1FF3262F01F0340
:1007C00003F1010358B24FF0010202FA00F30B608B
:1007D00003E0002AC8DB024CD5E710BC704700BF1D
:1007E00080E100E01EF0040F0CBFEFF30880EFF390
:1007F000098020E9F00F00F001B800BF10B50268D1
:1008000042F2AC43C2F201031A6041685960826847
:100810009A60C168D96002691A6141695961826947
:100820009A61C169D961026A1A62416A5962826A2F
:100830009A62C16AD962026B1A63416B5963826B17
:100840009A63C16BD96300F1400018644EF62850DA
:10085000CEF2000002685A6418F082F9002800F015
:10086000FB8148F65C40C0F6030018F07FF94EF6B5
:100870002C54CEF200042368002B05DA48F66C40B5
:10088000C0F6030018F072F94EF62C51CEF20001BA
:10089000086810F0020F05D048F67C40C0F603004F
:1008A00018F064F94EF62852CEF200025478002C6B
:1008B00072D048F69440C0F6030018F057F94EF68F
:1008C0002853CEF20003597811F0010F05D048F6F5
:1008D000A440C0F6030018F049F94EF62850CEF2B5
:1008E0000000427802F00204E3B22BB148F6C440A3
:1008F000C0F6030018F03AF94EF62851CEF2000186
:10090000487800F00402D4B22CB148F6E840C0F6B2
:10091000030018F02BF94EF62853CEF20003597855
:1009200001F00800C2B22AB148F60C50C0F603002C
:1009300018F01CF94EF62854CEF20004637803F048
:100940001001C8B228B148F62C50C0F6030018F0C8
:100950000DF94EF62852CEF20002547804F020032E
:10096000D9B229B148F64C50C0F6030018F0FEF891
:100970004EF62850CEF20000427802F08004E3B236
:1009800053B14EF63851CEF20001096848F66C506A
:10099000C0F6030018F0EAF84EF62850CEF2000038
:1009A000428894B2002C5ED048F68C50C0F603000A
:1009B00018F0DCF84EF62853CEF20003598811F0F7
:1009C000010F05D048F69C50C0F6030018F0CEF891
:1009D0004EF62850CEF20000428802F00204A3B284
:1009E0002BB148F6C850C0F6030018F0BFF84EF619
:1009F0002851CEF20001488800F0040294B22CB1D4
:100A000048F6EC50C0F6030018F0B0F84EF6285344
:100A1000CEF20003598801F0080082B22AB148F6EC
:100A20002C60C0F6030018F0A1F84EF62854CEF260
:100A30000004638803F4807188B228B148F65C60D2
:100A4000C0F6030018F092F84EF62852CEF20002DB
:100A5000548804F4007399B229B148F67860C0F65E
:100A6000030018F083F84EF62850CEF2000002780A
:100A7000002A63D048F69060C0F6030018F076F8BC
:100A80004EF62854CEF20004237813F0010F05D05F
:100A900048F6A060C0F6030018F068F84EF628513A
:100AA000CEF20001087800F00202D4B22CB148F670
:100AB000C060C0F6030018F059F84EF62853CEF285
:100AC0000003197801F00800C2B22AB148F6D860D4
:100AD000C0F6030018F04AF84EF62854CEF200048F
:100AE000237803F01001C8B228B148F6FC60C0F6C4
:100AF000030018F03BF84EF62852CEF200021478AC
:100B000004F02003D9B229B148F62070C0F60300E2
:100B100018F02CF84EF62850CEF20000027802F0C1
:100B20008004E3B253B14EF63451CEF200010968AD
:100B300048F64070C0F6030018F018F842F2AC44D2
:100B4000C2F20104216A48F66C70C0F6030018F086
:100B50000DF8616A48F68070C0F6030018F006F8D8
:100B6000A16A48F69470C0F6030017F0FFFFE16A2F
:100B700048F6A870C0F6030017F0F8FF216848F6A1
:100B8000BC70C0F6030017F0F1FF616848F6D07042
:100B9000C0F6030017F0EAFFA16848F6E470C0F65B
:100BA000030017F0E3FFE16848F6F870C0F60300B1
:100BB00017F0DCFF216949F20C00C0F6030017F0C2
:100BC000D5FF616949F22000C0F6030017F0CEFF9F
:100BD000A16949F23400C0F6030017F0C7FFE169CC
:100BE00049F24800C0F6030017F0C0FF216B49F23C
:100BF0005C00C0F6030017F0B9FF216C49F27000E9
:100C0000C0F6030017F0B2FF616B49F28400C0F632
:100C1000030017F0ABFFA16B49F2A800C0F6030078
:100C200017F0A4FF42F2F440C2F20100026849F258
:100C3000CC00C0F603001146126817F097FF41F68A
:100C4000B003C2F201031A6849F2E400C0F60300DF
:100C50001146126817F08AFFFFF7B0FC10BD00BF05
:100C600000B505F0EBFF002808BF5DF804FBEFF3CB
:100C70000981EFF3118221E9F40F5DF804EB1EF016
:100C8000100F08BF21ED108A41F804ED0B4C2268CB
:100C9000002A18BF516006F043F82268516851F8E5
:100CA00004EB1EF0100F08BFB1EC108AB1E8F40F8E
:100CB00082F3118881F3098870470000F424012031
:100CC00008B540F66140C0F602004FF0FF016FF03A
:100CD0000102FFF73BFD08BDF8B507460C461E466E
:100CE0000799089D14F0030F00D0FEE722B1A4EB92
:100CF0008500A0F1480401E004F14800012D01D86D
:100D0000A16205E02A4601F08BFCA7EB8507A762EC
:100D10004FF0000363604FF01130E0624FF022317A
:100D200021634FF0333262634FF04433A3604FF0DE
:100D30005530E0604FF0663121614FF077326261EB
:100D40004FF08833A3614FF09930E0614FF0AA3142
:100D500021624FF0BB3262624FF0CC33A363E66393
:100D6000069820644FF0807161646FF00202226087
:100D700005F11200F8BD00BF62B64EF60453CEF284
:100D800000031A6842F08050186000BF4FEA00105C
:100D900049F2FC03C0F603031A5849F6E011C0F605
:100DA000030151F82200704738B504460D46FFF79D
:100DB000EDFF49F2FC03C0F6030303EB0414616882
:100DC000012902D0022903D101E0856038BD4561C7
:100DD00038BD00BF10B540F20403C4F202031A6824
:100DE0001A6040F20440C4F202000168016040F65B
:100DF0000403C4F202031C6849F2F011C0F60301B7
:100E00008A6824EA020449F23C12C0F603029068A0
:100E100004431C6040F60443C4F202031868C96826
:100E200020EA0100D26840EA02041C6041F2040397
:100E3000C4F202031868186041F20441C4F20201CE
:100E40000A680A6041F60404C4F2020423682360BD
:100E500041F60440C4F202000168016042F2040459
:100E6000C4F202042268226040F20C01C4F20201C2
:100E70000C6849F2C822C0F60302136824EA03048E
:100E800049F2CC13C0F60303186804430C6040F227
:100E90000C41C4F202010C68506824EA000458684E
:100EA00004430C6040F60C01C4F202010C68906827
:100EB00024EA0004986804430C6040F60C41C4F234
:100EC00002010C68D06824EA0004D86804430C606E
:100ED00041F20C01C4F202010868126920EA020022
:100EE0001B6940EA03040C6041F20C41C4F20201A8
:100EF0000868086041F60C03C4F202031A681A601D
:100F000041F60C44C4F202042168216042F20C0054
:100F1000C4F20200036803604FF0000440F21402C0
:100F2000C4F20202146040F21441C4F202010C60E7
:100F300049F21423C0F603039A6840F61400C4F281
:100F400002000260D96840F61443C4F2020319603B
:100F500041F21402C4F20202146041F21440C4F2DD
:100F60000200046041F61401C4F202010C6041F673
:100F70001443C4F202031C6042F21402C4F20202DF
:100F8000146040F20004C4F202042068206040F2C1
:100F90000041C4F202010C6849F2A022C0F603022B
:100FA000536824EA030449F27823C0F6030358681F
:100FB00004430C6040F60001C4F202010C68906822
:100FC00024EA0004986804430C6040F60041C4F22F
:100FD00002010C68D06824EA0004D8682043086045
:100FE00041F20001C4F202010868126920EA02001D
:100FF0001B691843086041F20041C4F202010A680B
:101000000A6041F60003C4F202031868186041F652
:101010000041C4F202010A680A6042F20003C4F20D
:101020000203186818604FF0010003F0D1FE10BDF4
:1010300008B543F63002C4F2020213686FEA532087
:101040006FEA4021116043F62003C4F201031A68DD
:1010500042F001001860FFF7BDFE08BD2DE9F00168
:101060009DF814709DF81860079D49F26014C0F651
:10107000030454F820004FEA4104FF2F12D0D0F8A7
:101080000C8049F2C41CC0F6030C1CF8077007FA68
:1010900004FC4FF0030707FA04F728EA07074CEAB5
:1010A0000707C760FF2B10D0D0F804C049F2C8175B
:1010B000C0F60307FF5C07FA01F74FF0010303FADC
:1010C00001F32CEA03033B434360FF2E0FD08768F4
:1010D00049F29C23C0F603039E5D06FA04F64FF026
:1010E000030303FA04F327EA030333438360B5F1F0
:1010F000FF3F16D04FEAD10303F1080350F82360F5
:1011000001F007014FEA810105F00F0505FA01F52D
:101110004FF00F0707FA01F126EA0101294340F8D1
:101120002310FF2A10D0016849F2C423C0F603033C
:101130009B5C03FA04F34FF0030202FA04F421EA81
:10114000040143EA01040460BDE8F001704700BFF8
:1011500049F2A413C0F6030353F820100A6849F2B9
:101160005823C0F6030353F820100A4049F23823ED
:10117000C0F6030353F82000824214BF0020012070
:10118000704700BF49F26013C0F6030353F8200014
:101190000069704749F25823C0F6030353F8203022
:1011A0007BB139B149F28411C0F6030151F8202016
:1011B0001360704749F21C12C0F6030252F8200077
:1011C0000360704700EB800049F2EC23C0F6030394
:1011D00053F8202002F1FF300D2800F28680DFE86E
:1011E00000F0071019222B343D464F58616A737C7A
:1011F00043F64400C4F20200036861F30003036095
:10120000704743F64003C4F202031A6861F3000218
:101210001A60704743F64003C4F20203186861F392
:1012200041001860704743F64000C4F202000268B3
:1012300061F382020260704743F64000C4F202008C
:10124000036861F3C3030360704743F64003C4F2CD
:1012500002031A6861F304121A60704743F64003F0
:10126000C4F20203186861F345101860704743F632
:101270004400C4F20200026861F341020260704758
:1012800043F64400C4F20200036861F310430360B4
:10129000704743F64403C4F202031A6861F35142F3
:1012A0001A60704743F64403C4F20203186861F3FE
:1012B00092401860704743F64000C4F20200026892
:1012C00061F386120260704743F64000C4F20200E8
:1012D000036861F3C7130360704743F64003C4F229
:1012E00002031A6861F308221A60704700EB80005D
:1012F00049F2EC23C0F6030353F8202049F62421D9
:10130000C0F6030151F82200704700BF2DE9F84FE5
:1013100004468A46914698469DF928709DF92C60AE
:101320009DF93050FFF7E2FF04EB840249F2EC2311
:10133000C0F6030303EB82035A68022A94BF836951
:10134000C369016A02F1FF3CBCF1030F2ED8DFE84C
:101350000CF0021802186FF30103BAF1000FC8BFB6
:101360006AF38203B9F1000FC8BF69F3C303B8F190
:10137000000FC8BF68F30613002F17DD67F3C7130C
:1013800014E06FF30923BAF1000FC8BF6AF38A2390
:10139000B9F1000FC8BF69F3CB23B8F1000FC8BF84
:1013A00068F30E33002FC8BF67F3CF3302F1FF3766
:1013B000032F44D8DFE807F002142638312C04D17B
:1013C000002E06DD66F3820103E0002EC8BF66F33F
:1013D0000001002DC8BF65F341016FF3C30130E088
:1013E000332C04D1002E06DD66F3861103E0002EB7
:1013F000C8BF66F30411002DC8BF65F345116FF334
:10140000C7111EE0352C04D1002E06DD66F38A21BB
:1014100003E0002EC8BF66F30821002DC8BF65F3A6
:1014200049216FF3CB210EE0002EC8BF66F30C31CB
:10143000002DC8BF65F34D316FF3CF3103E0022AB1
:1014400001D8836100E0C361016204EB840449F2C6
:10145000EC20C0F6030050F82430012B02D0082BFA
:1014600016D10BE049F24C73C0F603031A6840F240
:101470004401C4F201010A60BDE8F88F49F24C72E0
:10148000C0F60302116840F24440C4F2010001605A
:10149000BDE8F88F38B504460D46FFF727FF04EB8B
:1014A000840149F2EC23C0F6030303EB8104626874
:1014B00002F1FF3103290AD8DFE801F0020406082F
:1014C000456338BD856338BDC56338BD056438BD27
:1014D00040F24C23C2F201031B689BB1A8B91A6801
:1014E0006FF300021A604FF00000586240F2502182
:1014F000C2F2010108801A6842F0010018604FF042
:10150000010070474FF0000070474FF00000704737
:1015100010B483B040F24C23C2F201031B6803B342
:1015200010BB40F25022C2F20102586A148840EA0D
:101530000440019000BF00BF00BF00BF00BF586A59
:10154000148840EA04400090019C00988442ECD149
:10155000DDED017AB8EEE70A81ED000A4FF00100F7
:1015600004E04FF0000001E04FF0000003B010BCB9
:10157000704700BF40F24C23C2F201031B689BB1CD
:10158000A8B91A686FF300021A6059624FEA114154
:1015900040F25020C2F2010001801A6842F00101BD
:1015A00019604FF0010070474FF0000070474FF096
:1015B0000000704743F67403C4F20203186847F250
:1015C0000402C4F20002136840F25222C2F2010285
:1015D0004FF00001117013F0010F04D010464FF0CE
:1015E000040202703EE04FEA106212F0600F07D072
:1015F00040F25221C2F201014FF020030B7031E0A2
:1016000002F00401C9B239B140F25220C2F2010025
:101610004FF04002027025E0C3F3400343EAD0607C
:1016200010F0010F07D040F25221C2F201014FF039
:1016300080030B7016E002F01001CBB23BB140F218
:101640005220C2F201004FF0010202700AE002F0E3
:101650000202D0B230B140F25221C2F201014FF089
:1016600002030B7043F67401C4F202010B6843F0ED
:101670008070086047F20001C4F200010A6842F07D
:1016800008030B6042F2F440C2F20100016840F22C
:101690005422C2F201021160704700BF40F252238F
:1016A000C2F201031878704708B547F61021C1F659
:1016B000FF714FF00C0215F071FC4FF00C0008BDEB
:1016C00010B542F20803CEF204031A6842F010008B
:1016D000186041F27970C0F602004FF00F014FF030
:1016E0003602FFF733F843F64001C4F202010C68FA
:1016F00044F010030B6041F20004C4F2000449F20C
:101700005072C0F603021068206049F6E811C0F676
:101710000301886914F000FA15A3D3E9002314F03B
:101720003FFC4FF000024FF00003C3F6F07314F0DB
:10173000F1FA14F05DFA41F22C03C4F200031880B0
:1017400041F22800C4F200004FF00002028049F28A
:101750005471C0F60301086841F20C03C4F200039F
:101760001860228842F00101218010BDAFF3008093
:101770002D431CEBE2362A3F684620F007018D46D8
:1017800001B541F21003C4F200034FF000021A60E9
:1017900005F064FDBDE801408546704770B504461C
:1017A000B0F5CC7F2FD940F23233984216D940F2AF
:1017B0006560844215D940F6CB418C4214D941F67C
:1017C0009712944213D943F22F36B44212D946F2FB
:1017D0005F639C4298BF06250ED90FE04FF00105CC
:1017E0000AE04FF0020507E04FF0030504E04FF078
:1017F000040501E04FF00505072D06D1FEF7DEFEDA
:101800004FF0070501E04FF00005FEF72DFF0646FB
:1018100004EB84044FEAC40049F25871C0F6030196
:1018200051F83520B0FBF2F39CB2012C05D9B4F588
:10183000805F04D3FEF7C2FE01E04FF0020443F2E2
:101840000000C4F2000045F25551016049F258729F
:10185000C0F6030202EBC5052B7943F20401C4F282
:1018600000010B6043F20802C4F2000214604AF661
:10187000AA2303603046FEF701FF70BD08B543F2AE
:101880000003C4F200034CF6CC421A604FF0C800CB
:10189000FFF784FF08BD00BF43F20003C4F200035A
:1018A0004AF6AA221A60704710B5044643F21003A4
:1018B000C4F20003186810F0010F74D04FF032002A
:1018C00006F076FF43F21001C4F200010A6812F03C
:1018D000010F68D04FF0320006F06AFF43F21003A8
:1018E000C4F20003186810F0010F5CD04FF0320012
:1018F00006F05EFF43F21001C4F200010A6812F024
:10190000010F50D04FF0320006F052FF43F21003A7
:10191000C4F20003186810F0010F44D04FF03200F9
:1019200006F046FF43F21001C4F200010A6812F00B
:10193000010F38D04FF0320006F03AFF43F21003A7
:10194000C4F20003186810F0010F2CD04FF03200E1
:1019500006F02EFF43F21001C4F200010A6812F0F3
:10196000010F20D04FF0320006F022FF43F21003A7
:10197000C4F20003186810F0010F14D04FF03200C9
:1019800006F016FF43F21001C4F200010A6812F0DB
:10199000010F08D04FF0320006F00AFF43F21003A7
:1019A000C4F200031B682046FFF7F8FE10BD00BF1D
:1019B00002469CF8043043B1DCF8000040B141F22B
:1019C000D421C2F2010141F82200DCF8000050B934
:1019D00041F2D423C2F2010353F8220049F64042F7
:1019E000002808BF104670474FF0010303FA00F0CB
:1019F00010F00A0F0CBF00200120704770B50D4693
:101A000049F64403C0F6030353F82040002C45D0A8
:101A100000EB800040F25826C2F2010606EBC00639
:101A200030464FF0000104F09FFB122D07D142F227
:101A30000431C4F201010A6842F480030B60606B58
:101A400065F304006063E36C4FF0050006F0B0FE40
:101A5000A16841F08042A260236813F0020FFBD01E
:101A6000E46C122D16D142F20430C4F20100016878
:101A70006FF39651016042F20002CEF20402136845
:101A80004FEA03504FEA105140F2194291420CBF05
:101A9000A4006400304604F075FC01E04FF0FF3410
:101AA000204670BD38B52DED028B044608EE101AA5
:101AB00049F2BC75C0F6030505EB8005F7EE007A28
:101AC000B4EEE78AF1EE10FA09DC084614F07AFC6D
:101AD00000289FED260A18BFB0EE408A01E0B7EE5D
:101AE000008A2B78012B1CD16878FFF7FFFBD0ED23
:101AF0000B1A6D78B8EE612A62EE082A12EE900A8F
:101B000014F0B0F84FF000024FF00003C3F6E0739A
:101B100014F002F914F06CF801462846FFF7BAFCFD
:101B200018E0022B16D16D78DFED110A28EE201A8D
:101B300011EE100A14F096F84FF000024FF0000377
:101B4000C3F6E07314F0E8F814F052F801462846A2
:101B5000FFF72AF940F2D020C2F2010000EB840422
:101B600084ED008ABDEC028B38BD00BF0000000090
:101B700000F07F4510B54FF000044FF00000214603
:101B8000FFF790FF4FF001002146FFF78BFF4FF06A
:101B900002002146FFF786FF4FF003002146FFF7C2
:101BA00081FF4FF004002146FFF77CFF4FF0050056
:101BB0002146FFF777FF4FF006002146FFF772FF3F
:101BC00040F20C03C4F202031A6849F2EC71C0F649
:101BD0000301086822EA000249F65401C0F6030135
:101BE000086802431A6040F20C43C4F202031A6808
:101BF0001A6040F60C01C4F202010868086040F661
:101C00000C43C4F202031A681A6041F20C01C4F2D8
:101C100002010868086041F20C43C4F202031A682A
:101C20001A6041F60C01C4F202010868086041F62E
:101C30000C43C4F202031A681A6042F20C01C4F2A7
:101C400002010868086040F20003C4F202031A6847
:101C500049F61401C0F60301086822EA000249F2BD
:101C60009871C0F60301086802431A6040F200430D
:101C7000C4F202031A681A6040F60001C4F20201BD
:101C80000868086040F60043C4F202031A681A604C
:101C900041F20001C4F202010868086041F2004309
:101CA000C4F202031A681A6041F60001C4F202018C
:101CB0000868086041F60043C4F202031A681A601B
:101CC00042F20001C4F202010868086010BD00BFC2
:101CD00008B508280ED849F63803C0F60303195C86
:101CE000FF290AD049F29072C0F60302105CFFF798
:101CF00085FE08BD4FF0FF3008BD4FF0FF3008BD36
:101D000010B50446FFF7E4FF07EE900AB8EE677AD5
:101D100049F63803C0F60303185D11280BD147F6C6
:101D20002A21C1F6FF710A8801EE102AF8EEC11AC5
:101D3000C1EE870A03E09FED030AC7EE000A10EE2A
:101D4000900A10BD00F07F4540F2D023C2F201039B
:101D500003EB80000068704738B50D46044600B3B9
:101D60000E2801D9FEF72AFC49F6E813C0F6030352
:101D700053F8240055B1B0FBF5F14FEA114202F1DE
:101D80000103B0FBF3F0B0FBF5F502E04FF0000506
:101D90002A4649F62421C0F6030151F824309A62FC
:101DA000DD6238BD10B582B000918DF8042007289F
:101DB00040F0E2804FF00000FFF716FE48B1EC461D
:101DC0004FF00000FFF7F4FD01464FF00000FFF771
:101DD000C3FF4FF00100FFF707FE48B1EC464FF09C
:101DE0000100FFF7E5FD01464FF00100FFF7B4FFEA
:101DF0004FF00200FFF7F8FD48B1EC464FF002004B
:101E0000FFF7D6FD01464FF00200FFF7A5FF4FF0A8
:101E10000300FFF7E9FD48B1EC464FF00300FFF780
:101E2000C7FD01464FF00300FFF796FF4FF0040097
:101E3000FFF7DAFD48B1EC464FF00400FFF7B8FDBC
:101E400001464FF00400FFF787FF4FF00500FFF752
:101E5000CBFD48B1EC464FF00500FFF7A9FD014668
:101E60004FF00500FFF778FF4FF00600FFF7BCFDCD
:101E700048B1EC464FF00600FFF79AFD01464FF0DF
:101E80000600FFF769FF4FF00700FFF7ADFD48B10F
:101E9000EC464FF00700FFF78BFD01464FF00700BF
:101EA000FFF75AFF4FF00800FFF79EFD48B1EC46E0
:101EB0004FF00800FFF77CFD01464FF00800FFF7E8
:101EC0004BFF4FF00900FFF78FFD48B1EC464FF094
:101ED0000900FFF76DFD01464FF00900FFF73CFFD9
:101EE0004FF00A00FFF780FD48B1EC464FF00A00C2
:101EF000FFF75EFD01464FF00A00FFF72DFF4FF0A0
:101F00000B00FFF771FD48B1EC464FF00B00FFF7F7
:101F10004FFD01464FF00B00FFF71EFF4FF00C0086
:101F2000FFF762FD48B1EC464FF00C00FFF740FDB3
:101F300001464FF00C00FFF70FFF4FF00D00FFF7C9
:101F400053FD48B1EC464FF00D00FFF731FD01465F
:101F50004FF00D00FFF700FF4FF00E00FFF744FDBC
:101F600048B3EC464FF00E00FFF722FD01464FF05C
:101F70000E00FFF7F1FE1EE049F2BC73C0F603034A
:101F800013F82010012916D149F2BC72C0F60302E1
:101F900002EB8000447804EB840349F2EC21C0F6A4
:101FA000030151F82340EC462046FFF701FD0146AE
:101FB0002046FFF7D1FE02B010BD00BF70B584B05F
:101FC00040F25825C2F2010549F65004C0F6030458
:101FD0002846214604F0B0F805F12800214604F017
:101FE000ABF805F15000214604F0A6F843F644038F
:101FF000C4F202031A6842F480701860196841F450
:1020000000761E6049F2E475C0F603052C6842F2C2
:102010000433C4F201031C6049F2E072C0F603020B
:10202000106842F20401C4F20101086042F2041691
:10203000C4F20106306049F64005C0F603052C687D
:1020400042F20C03C4F201031C6042F20C12C4F20F
:102050000102146049F2DC70C0F60300016842F22C
:102060001006C4F20106316042F21015C4F20105F7
:10207000296049F2D874C0F60304236842F22C02A6
:10208000C4F20102136042F22C10C4F2010003609A
:1020900049F61001C0F603010E6842F20805C4F2C9
:1020A00001052E6042F20814C4F2010426604FF0CC
:1020B0001C004FF00101FFF785F84FF01D004FF0B5
:1020C0000101FFF77FF84FF036004FF00101FFF7F5
:1020D00079F84FF0000400944FF001060196029445
:1020E0004FF01C00214632464FF00603FFF70EF971
:1020F00049F2EC25C0F6030595F83C02D5F84012EC
:1021000000940194D5F8383202934FF0030223462D
:10211000FEF7A4FF0094019602944FF01D002146A3
:1021200032464FF00603FFF7F1F895F85002D5F864
:10213000541200940194D5F84C2202924FF00302FD
:102140002346FEF78BFF0094019602944FF0360071
:10215000214632464FF00603FFF7D8F895F84404BD
:10216000D5F8481400940194D5F8405402954FF0E6
:1021700003022346FEF772FF4FF007002146224676
:10218000FFF710FE4FF0000520462946FFF78AFCB6
:1021900030462946FFF786FC4FF002002946FFF73C
:1021A00081FC4FF003002946FFF77CFC4FF0040050
:1021B0002946FFF777FC4FF005002946FFF772FC30
:1021C0004FF006002946FFF76DFC3046FFF70CFC88
:1021D00050B149F62420C0F60300416849F2E87383
:1021E000C0F603031A680A604FF00200FFF7FCFB19
:1021F00050B149F62420C0F60300816849F2E87323
:10220000C0F603031A680A604FF00300FFF7ECFB07
:1022100050B149F62420C0F60300C16849F2E873C2
:10222000C0F603031A680A604FF00400FFF7DCFBF6
:1022300050B149F62420C0F60300016949F2E87361
:10224000C0F603031A680A604FF00500FFF7CCFBE5
:1022500050B149F62420C0F60300416949F2E87301
:10226000C0F603031A680A604FF00600FFF7BCFBD4
:1022700050B149F62420C0F60300816949F2E873A1
:10228000C0F603031A680A604FF00700FFF7ACFBC3
:1022900050B149F62420C0F60300C16949F2E87341
:1022A000C0F603031A680A604FF00800FFF79CFBB2
:1022B00050B149F62420C0F60300016A49F2E873E0
:1022C000C0F603031A680A604FF00900FFF78CFBA1
:1022D00050B149F62420C0F60300416A49F2E87380
:1022E000C0F603031A680A604FF00A00FFF77CFB90
:1022F00050B149F62420C0F60300816A49F2E87320
:10230000C0F603031A680A604FF00B00FFF76CFB7E
:1023100050B149F62420C0F60300C16A49F2E873BF
:10232000C0F603031A680A604FF00C00FFF75CFB6D
:1023300050B149F62420C0F60300016B49F2E8735E
:10234000C0F603031A680A604FF00D00FFF74CFB5C
:1023500050B149F62420C0F60300416B49F2E873FE
:10236000C0F603031A680A604FF00E00FFF73CFB4B
:1023700050B149F62420C0F60300816B49F2E8739E
:10238000C0F603031A680A60FFF7F4FB04B070BDDF
:1023900010B504464FF000004FF01101FFF72EFB7F
:1023A00047F62A23C1F6FF73198807EE901AB8EE94
:1023B000670A06EE900AB8EE667AC0EE070AC4ED28
:1023C000000A4FF0010010BD30B472B649F6800328
:1023D000C0F603031A684EF63470CEF200000260B5
:1023E00049F68C01C0F603010A684EF68853CEF216
:1023F00000031A6049F69000C0F60300016842F23B
:102400000802CEF20402116049F69403C0F60303F9
:10241000186842F20C01CEF20401086043F6000392
:10242000C4F202031A6842F48030186019460B683F
:1024300013F4003FFBD043F64000C4F202000268F0
:1024400042F08051016047F20003C4F200031868B3
:1024500040F480421A6049F67801C0F6030108682A
:1024600043F60803C4F20203186049F68402C0F67A
:102470000302116843F60040C4F20200016049F60D
:102480008803C0F603031A6843F60401C4F202018C
:102490000A6043F60000C4F20200036843F0807251
:1024A00002600146086810F0007FFBD043F6080385
:1024B000C4F202031A684FF0020161F301021A60CC
:1024C0001846036803F00C02082AFAD143F64401C7
:1024D000C4F20201086840F480430B6043F6300008
:1024E000C4F20200026842F48011016047F2000366
:1024F000C4F200031A6842F48071196047F20403C1
:10250000C4F200031A6842F400711960036843F4CE
:102510008022026043F61440C4F20200016848F6CB
:102520001843C0F603031B6849F67C02C0F6030299
:1025300010686FEA000259400A4206D048F6184077
:10254000C0F603004178CC2904D12A4B2A4999428C
:1025500021D344E043F60841C4F2020142F63B2095
:10256000C0F61900086046F67F60C4F65D4008605A
:10257000134043F61442C4F202021360136843F09E
:102580000201116043F60C40C4F20200026812F42A
:10259000803FFBD1D9E7194C194D281B20F00305CA
:1025A0004FF0000340F20002C1F200024BF64C3142
:1025B000C0F6030105F10404C5F380005D589D5089
:1025C00003F10403A3420CD109E05858985003F1D9
:1025D00004035858985003F10403A342F5D130BCCA
:1025E00070470028F1D05858985003F10403A342D3
:1025F000EBD1F4E7D8F703084CBB030850BB030842
:10260000DBF7030843F63003C4F202031A6842F40E
:1026100000101860196841F480021A60704700BF0A
:102620002DE9F0011546002A66D041F6C003C2F23A
:10263000010353E8002F02F1010243E80024012CBA
:10264000F7D049F69C02C0F60302146846F2084629
:10265000C4F20206346049F69807C0F603073A68E8
:1026600046F22843C4F202031A604FF6FF7846F29E
:10267000304CC4F2020C46F23447C4F2020746F270
:102680002C46C4F202061C46454534BF2B46434641
:10269000CCF8001038603360226842F001022260FA
:1026A000ED1A4FEA8303C918C018226812F0010F0F
:1026B000FBD1002DE8D141F6C003C2F2010353E87B
:1026C000002FA2F1010243E80024012CF7D053E8C7
:1026D000002FB2F1004F0DD14FF0000243E800246B
:1026E000012CF4D04EF60450CEF20000016841F007
:1026F00080510160BFF32F8FBDE8F001704700BF2C
:1027000070B41646002A37D046F21045C4F20205CE
:102710002C6814F0010FFBD149F6A402C0F60302A5
:10272000146846F20842C4F20202146046F21842EB
:10273000C4F20202116046F21C41C4F202010860B8
:1027400046F21440C4F20200066049F6A002C0F648
:102750000302116846F21040C4F2020001600268F0
:1027600042F0010101603BB146F21040C4F20200A8
:10277000036813F0010FFBD170BC704743F61043A0
:10278000C4F20203186800280DDA43F60441C4F2CB
:10279000020140F22312C4F267520A6048F6AB13FA
:1027A000CCF6EF530B6043F61040C4F20200016810
:1027B00001F00042002A14BF02200020704700BF31
:1027C00043F61043C4F202031868002807DB43F6FF
:1027D0001041C4F202010A6842F000430B607047E6
:1027E00000F17840B0F5801F2CBF00200120704719
:1027F0002DE9F04F83B006460D46FFF7F1FF0028A4
:1028000056D02846FFF7ECFF002854D0AE4255D8EA
:10281000FDF72AFF0190FFF7B1FF0446002841D1E0
:1028200006F178434FEA933049F6AC02C0F6030252
:1028300012F8008041F28830FFF736F84FF00209B5
:1028400043F6104BC4F2020B43F60C47C4F20207E6
:1028500049F6F40AC0F6030AFFF71EF8494668F382
:10286000C60169F3092141F48033CBF800303868A0
:1028700010F4803FFBD15AF82820B61808F101085F
:102880005FFA88F8B542E7D24FF06400FFF70CF822
:1028900049F6A801C0F60301086843F61043C4F2E4
:1028A00002031860FFF78CFF0198FDF7E7FE07E0D1
:1028B0004FF0020404E04FF0020401E04FF0020484
:1028C000204603B0BDE8F08F2DE9F04106460C46E6
:1028D00015460846FFF784FF002861D005F1FF3058
:1028E0002018FFF77DFF00285DD041F6C003C2F23B
:1028F000010353E8002F02F1010243E800210129FE
:10290000F7D0FFF73BFF074630BB49F6EC01C0F6B6
:1029100003010A6843F61040C4F2020002608DB160
:1029200006F1FF3843F60C46C4F20206336813F48E
:10293000803FFBD118F8011F04F8011BFEF7ACFF24
:10294000013DF3D149F6F004C0F60304226843F6D2
:102950001040C4F202000260FFF732FF41F6C003EC
:10296000C2F2010353E8002FA2F1010243E8002460
:10297000012CF7D053E8002FB2F1004F0DD14FF0EA
:10298000000243E80024012CF4D04EF60450CEF2AD
:102990000000016841F080510160BFF32F8F04E017
:1029A0004FF0020701E04FF002073846BDE8F08122
:1029B00041F21833C2F20103186849F63012C0F62A
:1029C0000302116801604FF00003036049F63412FE
:1029D000C0F603021168416049F6DC13C0F6030338
:1029E0001A68C2614FF00D01016249F63813C0F652
:1029F00003031A680260704741F21033C2F2010308
:102A00001868704770B48568C668446806FB05405E
:102A10004118196041F21030C2F201000068814291
:102A20000CD2521890420CD341F21430C2F2010081
:102A30000268891819604FF0010004E04FF00000AF
:102A400001E04FF0000070BC704700BF2DE9F0417D
:102A50000546FEF721FF4FF01E044FF0000841F23B
:102A60001836C2F201064FF00107052D26D8DFE81F
:102A700005F0030A0F14191E3268936983F00200EF
:102A8000C0F340011BE03068416901F0010116E02C
:102A900032685369C3F3400111E030684169C1F302
:102AA000C0110CE032685369C3F3801107E033684A
:102AB000986980F0010101F0010100E0414689B907
:102AC00033685A6912F4807F10D1586910F4806F0E
:102AD00010D1384605F06CFE013CC6D14FF0000025
:102AE000BDE8F0814FF00100BDE8F0814FF000003B
:102AF000BDE8F0814FF00000BDE8F0812DE9F04124
:102B000084B014461D46072900F2AD80072A00F262
:102B1000AD8001EB810249F63C13C0F6030303EBE1
:102B20008202137C002B40F0A48004EB840249F65F
:102B30003C13C0F6030303EB8202137C012B40F02D
:102B40009B8049F63C13C0F6030301EB810653F862
:102B5000262004EB840653F826309A4240F08F80FA
:102B600041F21C37C2F201073870022A15D0032A3D
:102B700025D0012A34D143F64000C4F20200066891
:102B800046F40012026041F21833C2F2010345F22A
:102B90000047C4F200071F6022E043F64000C4F281
:102BA0000200066846F48002026041F21833C2F265
:102BB000010345F60007C4F200071F6010E043F66A
:102BC0004000C4F20200066846F40002026041F2CE
:102BD0001833C2F2010345F60047C4F200071F6034
:102BE00049F63C18C0F6030801EB810108EB8102AD
:102BF000107991684FF0000700974FF00106019699
:102C0000D36802934FF003023B46FEF727FA04EB2A
:102C1000840408EB84042079A16800970196E26897
:102C200002924FF003023346FEF718FAFFF7C0FE98
:102C300045B341F21430C2F201000A99016041F239
:102C40001032C2F201020B9B136041F22030C2F23B
:102C5000010049F62411C0F603012A463B4607F05D
:102C600075FA304610E04FF000000DE04FF0000024
:102C70000AE04FF0000007E04FF0000004E04FF0E2
:102C8000000001E04FF0010004B0BDE8F08100BF9A
:102C900038B5044641F21833C2F201031D68A86931
:102CA00010F0020F63D0FFF783FEA96911F0020F45
:102CB0005DD03BE041F21835C2F201052B684FF0C0
:102CC000A0021A614FF00200FFF7C0FE2868816978
:102CD00011F0010F08D0456915F4806F00F03882BB
:102CE000036843F4007202604FF0050003F032FE07
:102CF0004FF0000516E041F21830C2F20100016801
:102D00004FEA14230B614FF00300FFF79FFE38B129
:102D100041F21832C2F201021068E4B2046101E02B
:102D20004FF00005281C18BF012038BD4FF00000EF
:102D300038BD4FF0000038BD4FF0000038BD4FF0F7
:102D4000000038BD4FF0000038BD4FF0000038BD26
:102D50004FF0000038BD4FF0000038BD4FF00000CC
:102D600038BD4FF0000038BD4FF0000038BD41F2D3
:102D70001832C2F2010213684FF00000586119685E
:102D800060F3492119601A6842F4807018604FF0AE
:102D90000100FFF75BFE0028CBD041F21835C2F2EC
:102DA00001052B684FF0A00119614FF00200FFF7F9
:102DB0004DFE2868826912F0010F08D0436913F4B0
:102DC000806F00F0C881016841F4007202604FF02A
:102DD000050003F0BFFD41F21830C2F201000368A4
:102DE0004FF0000159611A6861F349221A601868AE
:102DF00040F4807119604FF00100FFF727FE0028B2
:102E00009AD041F21835C2F201052B684FF0A002AA
:102E10001A614FF00200FFF719FE2868816911F06E
:102E2000010F08D0436913F4806F00F097810268A6
:102E300042F4007101604FF0050003F08BFD41F298
:102E40001830C2F2010003684FF0000159611A689E
:102E500061F349221A60186840F4807119604FF0DC
:102E60000100FFF7F3FD00283FF469AF41F2183588
:102E7000C2F201052B684FF0A0021A614FF0020068
:102E8000FFF7E4FD2868816911F0010F08D043695C
:102E900013F4806F00F06581026842F400710160F4
:102EA0004FF0050003F056FD41F21830C2F2010068
:102EB00003684FF0000159611A6861F349221A60F2
:102EC000186840F4807119604FF00100FFF7BEFDF3
:102ED00000283FF437AF41F21835C2F201052B68E4
:102EE0004FF0A0021A614FF00200FFF7AFFD286813
:102EF000816911F0010F08D0436913F4806F00F06D
:102F00003381026842F4007101604FF0050003F064
:102F100021FD41F21830C2F2010003684FF00001B8
:102F200059611A6861F349221A60186840F4807187
:102F300019604FF00100FFF789FD00283FF405AF4D
:102F400041F21835C2F201052B684FF0A0021A6158
:102F50004FF00200FFF77AFD2868816911F0010F38
:102F600008D0436913F4806F00F00181026842F4D5
:102F7000007101604FF0050003F0ECFC41F21830E5
:102F8000C2F2010003684FF0000159611A6861F351
:102F900049221A60186840F4807119604FF00100EE
:102FA000FFF754FD00283FF4D3AE41F21835C2F2CA
:102FB00001052B684FF0A0021A614FF00200FFF7E5
:102FC00045FD2868816911F0010F08D0436913F4A9
:102FD000806F00F0CF80026842F4007101604FF012
:102FE000050003F0B7FC41F21830C2F2010003689B
:102FF0004FF0000159611A6861F349221A6018689C
:1030000040F4807119604FF00100FFF71FFD0028A8
:103010003FF4A1AE41F21835C2F201052B684FF022
:10302000A0021A614FF00200FFF710FD28688169C5
:1030300011F0010F08D0436913F4806F00F09D80F8
:10304000026842F4007101604FF0050003F082FC59
:1030500041F21830C2F2010003684FF000015961DB
:103060001A6861F349221A60186840F48071196087
:103070004FF00100FFF7EAFC00283FF46FAE41F289
:103080001835C2F201052B684FF0A0021A614FF00B
:103090000200FFF7DBFC2868816911F0010F07D0FF
:1030A000436913F4806F6BD0026842F400710160D1
:1030B0004FF0050003F04EFC41F21830C2F201005F
:1030C00003684FF0000159611A6861F349221A60E0
:1030D000186840F4807119604FF00100FFF7B6FCEA
:1030E00000283FF43EAE41F21835C2F201052B68CC
:1030F0004FF0A0021A614FF00200FFF7A7FC28680A
:10310000816911F0010F07D0436913F4806F3AD041
:10311000026842F4007101604FF0050003F01AFCF0
:1031200041F21830C2F2010003684FF0000159610A
:103130001A6861F349221A60186840F480711960B6
:103140004FF00100FFF782FC00287FF4B3AD0BE6DF
:103150004FF0010519E04FF00A0516E04FF00905A0
:1031600013E04FF0080510E04FF007050DE04FF0B9
:1031700006050AE04FF0050507E04FF0040504E0FE
:103180004FF0030501E04FF0020541F21C30C2F29E
:103190000100017801F1FF33DAB2012A3FF6B8AD40
:1031A000A9E500BFF8B50D461446002A6FD080B2DD
:1031B000FFF76EFD002865D04FF00300FFF746FCD7
:1031C00000285FD041F21833C2F201031868026888
:1031D00042F4807101604FF00100FFF737FC0028D6
:1031E00050D041F21833C2F20103186814F1FF31D4
:1031F00018BF0121026861F38A2202604FF0A10327
:1032000003614FF00200FFF721FC00283AD041F2A1
:103210001830C2F2010001688A6912F0010F31D042
:103220004B6913F4806F2DD14FF0040641F218372B
:10323000C2F201073046FFF709FC18B304F1FF346E
:10324000012C27D1FDF710FA39680A696FEA0203E9
:1032500005F8013B0A686FF38A220A60FDF70EFA4F
:10326000E8E72B681B6902E04FF004060E4D30467C
:10327000FFF7ECFB0028F4D10B4B1868016841F410
:1032800000720260D4F1010038BF0020F8BD4FF099
:103290000100F8BD386801696FEA010205F8012BE9
:1032A000002CC7D1E0E700BF1813012030B583B070
:1032B00015461C461A4601ABFFF7A4FB48B101981E
:1032C00029462246FFF76EFF00280CBF1820002079
:1032D00001E04FF01F0003B030BD00BF2DE9F84FF3
:1032E00093460D4600295DD004464FF0030841F295
:1032F0001839C2F2010901E0002E40D01FFA8BF00C
:10330000FFF7C6FC00283DD00BF0070715F0010FB2
:103310004CD14046FFF79AFB002836D0072F1AD829
:10332000DDB13CB1D9F8000014F8011B6FEA0103CC
:10333000036104E0D9F800604FF0FF02326107F149
:103340000107BA4605F1FF3635464046FFF77EFBDA
:10335000002845D119E02E4600E02E46D9F800009D
:10336000026842F4007101600BF1080B2BF0070BAF
:103370004FF00500FFF76AFB0028BDD107E04FF0D2
:10338000010004E04FF0000001E04FF0000041F2C6
:103390001833C2F2010319680A6842F400730B6023
:1033A000BDE8F88F4FF00100BDE8F88F4046FFF709
:1033B0004DFB0028E9D0072FCDD82CB9D9F8003023
:1033C0004FF0FF021A6106E0D9F8000014F8011B63
:1033D0006FEA0103036107F1010705F1FF3598E783
:1033E000072FB8D82CB9D9F800504FF0FF022A6146
:1033F00006E0D9F8000014F8011B6FEA010303612D
:1034000007F1010706F1FF3583E700BF30B583B050
:1034100015461C461A4601ABFFF7F4FA48B1284698
:103420002146019AFFF75AFF00280CBF1820002000
:1034300001E04FF01F0003B030BD00BF08B542F2FD
:10344000F840C2F2010042F2F872C2F20102131A0D
:103450004FF0FF314FEAA302FDF7C0F842F2F870D7
:10346000C2F2010042F6F871C2F201010A1A4FEAF3
:10347000A2024FF0FF31A2F12002FDF7AFF802F0F7
:1034800055FA41F23030C2F2010044F20001C4F2B8
:1034900002014FF480524FF0030312F017FBFDF7C7
:1034A0006BFC4FF0000008BDBFF36F8F704700BF8B
:1034B00049F66023C0F60303185C00EB400149F6AF
:1034C0004432C0F6030252F821305B68704700BFF7
:1034D00038B549F66023C0F603031B5C03EBC30455
:1034E00041F24832C2F2010202EB840282F821105A
:1034F00014693CB141F24835C2F201051346D26964
:103500009B69A04738BD00BFF8B506460F4649F68F
:103510006023C0F603031D5C05EBC50041F248348F
:10352000C2F2010404EB8004D4F810C0BCF1000F17
:1035300007D0E2698A4204D030464FF00001A36907
:10354000E047E76163695BB105EBC50041F24832D2
:10355000C2F2010202EB8002304639469269984776
:1035600094F8201079B127696FB105EBC50541F2D8
:103570004833C2F2010303EB8505304694F821106D
:10358000E269AB69B847F8BD49F66023C0F60303AA
:10359000185C00EB400149F64432C0F6030252F8D1
:1035A0002130D86840F08001D9607047F8B50446F2
:1035B00000EB400249F64433C0F6030353F822609F
:1035C00035686FEA0500306005F0010215F0020F62
:1035D0001CBF42F00202D2B215F0040F18BF42F035
:1035E000080215F0080F18BF42F0040215F4807F9E
:1035F00005D0316911F4804F18BF42F0100215F068
:10360000200F00D1E2B104EBC40741F24833C2F20B
:10361000010303EB870087688FB1716804EBC40076
:1036200041F24833C2F2010303EB800349F608304C
:10363000C0F60300005DC9B29B69B84700E073683B
:10364000F26812F0800F1CD015F0800F19D0F168CD
:103650006FF3C711F16004EBC40041F24833C2F2CA
:10366000010353F8203063B141F24832C2F2010243
:1036700002EB800249F60830C0F60300005D916954
:10368000984715F0400F17D004EBC40141F24833BE
:10369000C2F2010303EB810253686BB1084641F2A9
:1036A0004831C2F2010101EB800249F60830C0F650
:1036B0000300005D91699847F8BD00BF684620F09F
:1036C00007018D4601B54FF00600FFF76FFFBDE81B
:1036D00001408546704700BF684620F007018D46CF
:1036E00001B54FF00500FFF761FFBDE801408546D9
:1036F000704700BF684620F007018D4601B54FF0C6
:103700000400FFF753FFBDE801408546704700BF46
:10371000684620F007018D4601B54FF00300FFF722
:1037200045FFBDE801408546704700BF684620F070
:1037300007018D4601B54FF00200FFF737FFBDE8E6
:1037400001408546704700BF684620F007018D465E
:1037500001B54FF00100FFF729FFBDE801408546A4
:10376000704700BF10B582B08DF8071049F660238E
:10377000C0F60303185C00EB400249F64431C0F682
:10378000030151F82240236813F0800FFBD002A9F7
:1037900011F8012D626000EBC00041F24834C2F222
:1037A000010404EB8004608C4FF0010205F018F86E
:1037B000608404F1200402B010BD00BF70B582B077
:1037C0008DF8071049F66023C0F60303185C00EB80
:1037D000400149F64432C0F6030252F82140256800
:1037E00015F0800F1DBF9DF807506560012600266B
:1037F00000EBC00341F24830C2F2010000EB830548
:10380000688C0DF107014FF0010204F0E9FF6884B4
:1038100005F12005E16841F08002E260304602B027
:1038200070BD00BF2DE9F84F81468B4690461E467D
:103830009DF828A049F66023C0F603031D5C05EB44
:10384000450249F64430C0F6030050F822409DF886
:103850002C70012F14BF00270127082E06D0072E39
:1038600002D1B8F1000F01D1FCF7A8FE0AF1FF3137
:10387000CBB2012B01D9FCF7A1FE49F62832C0F6E4
:10388000030252F82500B0FBFBF1A1604FF00002EB
:1038900067F38612BAF1010F04D0002F0CBF022388
:1038A000002301E04FF0000363F30D3267F38E3223
:1038B00022614FF06C00B8F1020F14BF0023012306
:1038C00063F3492018F1000818BF4FF0010868F3AE
:1038D0008A20082E18BF4FF0000868F30C3040F41F
:1038E0000051E1604846FFF7E3FDBDE8F88F00BFF7
:1038F000F0B585B00D461E4649F66023C0F60303B9
:10390000195C01EB410449F64437C0F6030757F848
:10391000247049F62433C0F60303185C00EB400121
:1039200049F69834C0F6030404EBC1040AB1FCF76D
:1039300045FE75B9207B21699DF82C2000924FF03F
:1039400001030193626902924FF003023346FDF7CF
:1039500085FB207861689DF8283000934FF00102C4
:103960000192A36802934FF003023346FDF776FB02
:1039700049F6F420C0F603000168012D14BF0025AC
:10398000012565F3C301796105B0F0BD2DE9F84368
:10399000054649F66023C0F60303185C00EBC0023D
:1039A00041F24834C2F2010404EB820449F6443186
:1039B000C0F6030100EB40064FEA860301EB030863
:1039C00051F80390FCF750FE064694F82000B8B179
:1039D0004FF00007C9F80C703846394698F90420B2
:1039E000FCF7B4FE28463946FFF772FDE3681BB1C9
:1039F0002846E169A26998474FF0000284F8202028
:103A00003046FCF73BFEBDE8F88300BF2DE9F04FE0
:103A100085B005468B469246994649F66023C0F626
:103A200003031E5C41F24838C2F2010806EBC607E8
:103A30004FEA870708EB070406EB460049F64431D6
:103A4000C0F6030101EB8006FCF70EFE039043F67F
:103A50004003C4F20203186849F60031C0F60301BE
:103A60000A6820EA020E49F6F822C0F6030210683E
:103A70004EEA0000186043F64403C4F202031868DB
:103A8000496820EA010052681043186049F6103175
:103A9000C0F6030105EB8503C818C95C427883783A
:103AA00090F803C0CDF800C0007901902846FFF7D8
:103AB0001FFF9DF8382000929DF83C100191284688
:103AC000594652464B46FFF7ADFE109B48F807306B
:103AD0001298A060119A62601399E160149BA3612F
:103AE000B0684FF00F0196F90420FCF72FFE4FF05D
:103AF000010084F820000398FCF7C0FD05B0BDE884
:103B0000F08F00BF49F66023C0F60303185C00EB9A
:103B1000C00341F24830C2F2010000EB8303196197
:103B20005A61704749F62433C0F60303185C00EB72
:103B3000400149F66422C0F6030202EB011070470F
:103B4000FA2884BF0530C0B2032812D849F6602392
:103B5000C0F60303185C00EBC00141F24832C2F228
:103B6000010202EB81034FF6FF7058844FF0010011
:103B700070474FF000007047FA2884BF0530C0B28C
:103B800003280ED849F66023C0F60303185C00EB47
:103B9000C00141F24832C2F2010202EB8103588CAB
:103BA00070474FF000007047082806D9102807D941
:103BB00020288CBF4020202070474FF0080070471D
:103BC0004FF01000704700BF022809D0032804D02E
:103BD000012814BF0020012070474FF003007047F8
:103BE0004FF00200704700BF40F60013C5F200031B
:103BF000186840F60802C5F200021168C1F34103DB
:103C0000022B12BF6FF30200032363F3020040F4A0
:103C100000406FF3995040F60012C5F200021060A8
:103C200040F60401C5F200010B6843F4807008609F
:103C3000704700BF49F6E833C0F603031A6840F640
:103C40001030C5F200000260704700BF10B441F6AA
:103C50005C63C2F201031A5CE0B14FF0000341F66D
:103C6000F831C2F201014FF04C0404FB0212D1689A
:103C700021F0030202F1040262F312034FF001018A
:103C800061F3DC4349F6EC32C0F6030202EB40106C
:103C900081690B6010BC704770B440F22003C5F21C
:103CA00000031868C0F34342022A01D0062A29D132
:103CB00000F00F0149F68445C0F6030555F8216070
:103CC000C0F30A1505F1030398081BD041F2000167
:103CD000C5F2000100F1FF3404F001040A68334624
:103CE00072604FF0010282420ED10AE00C6803F1CB
:103CF000040343F8044F0C685C6002F10202824244
:103D0000F4D1356070BC7047002CEFD00C6803F123
:103D100004035C6002F101028242E7D1F1E700BFD7
:103D200070B449F66C43C0F6030353F82060326860
:103D3000002A3CD049F6EC31C0F6030101EB4011FA
:103D400002F103024FEA9202CB691B689A420CD936
:103D500040F63402C5F2000211684FF0010303FA85
:103D600000F008431060184623E006F10403C2B1D6
:103D700002F1FF3000F00105086953F8044B0460BC
:103D8000501E18D10DE00C691A4652F8045B2560EC
:103D900000F1FF300C695B68236002F10403013815
:103DA000F1D14FF0000131604FF0010001E04FF020
:103DB000000070BC7047002DE5D00A6953F8044B31
:103DC00014600138DFD1ECE708B54FF0010303FAC6
:103DD00000F041F24642C2F201021388184210D0AC
:103DE00023EA000341F24640C2F201000380CA6B9D
:103DF00052B1086A4FF0000103F03EFF4FF000009F
:103E000008BD4FF0000008BD4FF0010008BD00BF25
:103E100070B540F21403C5F200031C6849F6E030A7
:103E2000C0F6030001680C4200F0BB8141F6EC32A1
:103E3000C2F201021378012B40F2B38140F2180064
:103E4000C5F20000016849F69C42C0F603021368FF
:103E5000194200F0A68140F61800C5F20000016882
:103E600011F0010F56D040F60815C5F200052A687A
:103E700040F60830C5F2000003682A60036041F68E
:103E80005C61C2F20101087841F6F831C2F2010129
:103E90004FF04C0505FB001503F00100E96A0143F2
:103EA000E962C3F3C000296B0143296303F00803EF
:103EB000D8B258BBD2B212F0010F0ED01DE0EA6AA0
:103EC00022B105F1100000F063FF2BE02B6B002BFB
:103ED000F7D1686B0028F4D124E012F0900FEED0F7
:103EE00040F63403C5F20003186820F001011960A0
:103EF0004FF00000FFF714FFE1E76E6B4FF000009A
:103F00002946FFF761FF30436863D8E74FF00001AF
:103F1000E963CFE740F61802C5F20002136813F414
:103F2000803FA0D140F61801C5F200010A6802F0F6
:103F3000020398B2002856D040F62815C5F20005B5
:103F40002A6840F62830C5F2000003682A60036042
:103F500041F65C61C2F20101487841F6F831C2F2E3
:103F600001014FF04C0505FB001503F00100E96A63
:103F70000143E962C3F3C000296B0143296303F0E5
:103F80000803D8B258BBD2B212F0010F0ED01DE018
:103F9000EA6A22B105F1100000F0FAFE2FE02B6B67
:103FA000002BF7D1686B0028F4D128E012F0900FB5
:103FB000EED040F63403C5F20003186820F0020189
:103FC00019604FF00100FFF7ABFEE1E76E6B4FF0B9
:103FD00001002946FFF7F8FE30436863D8E74FF049
:103FE0000001E963CFE740F61801C5F200010A6855
:103FF0004FEA124303F0020081B200299CD140F63F
:104000001801C5F200010A6802F0040398B2002802
:1040100056D040F64815C5F200052A6840F64830EB
:10402000C5F2000003682A60036041F65C61C2F2D9
:104030000101887841F6F831C2F201014FF04C05D8
:1040400005FB001503F00100E96A0143E962C3F3CF
:10405000C000296B0143296303F00803D8B258BBA1
:10406000D2B212F0010F0ED01DE0EA6A22B105F1C2
:10407000100000F08DFE2FE02B6B002BF7D1686B4A
:104080000028F4D128E012F0900FEED040F634036F
:10409000C5F20003186820F0040119604FF0020017
:1040A000FFF73EFEE1E76E6B4FF002002946FFF797
:1040B0008BFE30436863D8E74FF00001E963CFE738
:1040C00040F61801C5F200010A684FEA124303F0F6
:1040D000040081B200299CD140F61801C5F200010C
:1040E0000A6802F0080398B258B940F61801C5F200
:1040F00000010A684FEA124303F0080081B2002968
:104100004FD040F66815C5F200052A6840F66830C1
:10411000C5F2000003682A60036041F65C61C2F2E8
:104120000101C87841F6F831C2F201014FF04C05A7
:1041300005FB001503F00100E96A0143E962C3F3DE
:10414000C000296B0143296303F00803D8B210B102
:104150004FF00001E963D2B212F0010F08D06E6B8C
:104160004FF003002946FFF72FFE304368630EE04F
:1041700012F0900F0BD040F63403C5F2000318681C
:1041800020F0080119604FF00300FFF7C9FDEA6A4B
:104190001AB92B6B0BB9686B18B105F1100000F060
:1041A000F7FD14F0100F01D0FFF776FD14F4805FD7
:1041B0000DD041F6EF31C2F201014FF001020A7059
:1041C00041F6BC33C2F20103186802F02DFA14F470
:1041D000005F01D0FFF708FD14F4006F14D041F622
:1041E000EE30C2F201004FF00101017041F6596357
:1041F000C2F201034FF000021A7041F6BC30C2F265
:104200000100006802F010FA002C14DA41F6EE31D9
:10421000C2F201014FF000030B7041F65960C2F287
:1042200001004FF00102027041F6BC31C2F20101FF
:10423000086802F0F9F940F21403C5F200031C60AB
:1042400070BD00BF684620F007018D4689B500AFFC
:10425000FFF7DEFDBD46BDE889408546704700BFDB
:104260002DE9F04141F6F836C2F201064FF04C0359
:1042700003FB0066304650F8205F49F6EC38C0F684
:1042800003084FEA451708EB07044FF000014FF011
:104290001C0212F0A7FE35624FF00100B06258F820
:1042A00007204FF00003136061690B60A0684FF0B6
:1042B000FF02026061680B60A0690360E1680A6048
:1042C00049F68442C0F6030252F82500036049F61D
:1042D0006C41C0F6030151F825201360BDE8F08160
:1042E00000B583B04FF00003019340F21001C5F216
:1042F00000010A68B0F1FF3F08BF102060F3891287
:1043000042F0200040F21003C5F200031860194685
:1043100040F63F52C0F20302019800F10100019003
:104320000B6813F0200F02D001989042F4D94FF09F
:10433000030004F03DFA03B000BD00BF2DE9F843CF
:104340004FF04C0303FB00F041F6F831C2F20101DB
:104350004418256A4FF0010606FA05F649F6EC32D4
:10436000C0F6030202EB45174058002867D0A36847
:10437000FBB1D7F80080D8F8001011F4004F18D125
:10438000D8F80020914663F30A09007AFFF71CFC75
:1043900060F3934949F4004965F3995949F0805015
:1043A000C0F3404363F39A60C8F800002846FFF763
:1043B00097FFE168F1B17A68106810F4004F19D1E5
:1043C0002846FFF743FCD7F80480D8F80070E3686C
:1043D00063F30A072168087AFFF7F6FB60F3934757
:1043E00047F4004242F01047C7F3404060F39A6739
:1043F000C8F8007049F68443C0F6030353F825104B
:104400004FF000020A60A06858B140F61C03C5F2E4
:104410000003196846EA010290B2196860F30F01BF
:104420001960E3685BB140F61C00C5F20000026849
:1044300046EA1246B6B2016866F31F410160BDE864
:10444000F88300BF70B582B04FF00002019240F2D5
:104450001003C5F20003196841F0010018600192D1
:104460001A6812F0010F19D0019940F63F53C0F2BB
:104470000303994212D840F21000C5F2000040F642
:104480003F52C0F20302019901F101010191036859
:1044900013F0010F02D001999142F4D94FF00300BB
:1044A00004F086F94FF00000019040F21002C5F2CE
:1044B00000021368002B1DDB019940F63F50C0F24B
:1044C0000300814216D84FF0030640F21005C5F2F2
:1044D000000540F63F54C0F20304304604F068F98A
:1044E000019A02F1010201922B68002B02DB019973
:1044F000A142F2D902B070BD00B583B04FF0000305
:10450000019340F21000C5F20000026842F0100171
:10451000016040F63F52C0F20302019B03F1010328
:104520000193016811F0100F02D0019B9342F4D95E
:104530004FF0030004F03CF903B000BD50B149F660
:104540008041C0F603010A6840F21803C5F2000377
:104550001A60704749F69443C0F603031A6840F2A4
:104560001800C5F200000260704700BF38B54FF078
:10457000000440F60063C5F200031C6040F6000230
:10458000C5F20002106840F0030164F3820164F395
:104590000A11116040F22405C5F200052B684FF0A6
:1045A000400262F30F032B60204662F31F40214656
:1045B00062F31F4162F30F0140F22805C5F20005C6
:1045C00029604FF0800363F30F0040F20412C5F23C
:1045D000000210604FF0C00161F30F0040F20815B7
:1045E000C5F2000528604FF4807363F30F0040F2BA
:1045F0000C12C5F2000210604FF0FF30FFF770FEA2
:10460000FFF77AFF40F61000C5F20000046040F6A4
:104610001401C5F200010C604FF0FF3540F618039D
:10462000C5F200031D6040F61C02C5F200021460D2
:104630002046FFF715FE4FF00100FFF711FE4FF087
:104640000200FFF70DFE4FF00300FFF709FE4FF0E9
:104650000400FFF705FE4FF00500FFF701FE4FF0E5
:104660000600FFF7FDFD4FF00700FFF7F9FD40F2F0
:104670001800C5F20000046040F21401C5F2000108
:104680000D604FF00100FFF759FF38BD41F246437E
:10469000C2F2010319884FF0010202FA00F008404B
:1046A00000280CBF02200320704700BF40F6001313
:1046B000C5F200031B68C3F3076202F08000C1B2B9
:1046C00009B143F0804343F4001040F60012C5F2F4
:1046D00000021060704700BF2DE9F84305461646FA
:1046E00049F6EC38C0F6030808EB401849F66C436D
:1046F000C0F6030353F820704FF0010909FA00F9DE
:104700000C46A9B9386840B941F24643C2F20103E8
:10471000188819EA000F5AD10AE041F24641C2F264
:1047200001010A8819EA020F02D02846FFF7D8FDD6
:1047300006F1030107F1040388081CD000F1FF32E1
:1047400002F0010CA4F1040151F8042F43F8042BEA
:1047500001383ED10FE001F1040249681C4644F8DB
:10476000041B00F1FF3002F1040152685A6004F1A9
:1047700004030138EFD13E6041F24643C2F2010327
:10478000198849EA0109A3F8009065B940F61010AC
:10479000C5F2000002684FF0010161F3D44266F3F4
:1047A0000602026009E0D8F8140002684FF0010325
:1047B00063F3DC4266F312020260D8F80030186836
:1047C00040F004421A6016B12846FFF7A9FABDE886
:1047D000F883BCF1000FBED051F8042F43F8042B2E
:1047E0000138B8D1C7E700BF70B5044649F6844325
:1047F000C0F6030353F82060334653F8045BAA4223
:1048000038BF1546084619462A4612F0C7FB4FF036
:10481000000030602046FFF719FA49F6EC31C0F687
:10482000030101EB441463681A6842F00440186005
:10483000284670BDF8B5054641F6F833C2F20103CB
:104840001868002871D041F6F831C2F20101CA6C33
:10485000002A71D041F6F834C2F20104D4F898600D
:10486000002E6DD041F6F837C2F20107D7F8E430D8
:10487000002B69D041F6F830C2F20100D0F83011B7
:10488000002965D041F6F832C2F20102D2F87C412B
:10489000002C61D041F6F836C2F20106D6F8C87194
:1048A000002F5DD041F6F833C2F20103D3F81402B1
:1048B000002859D041F6F831C2F20101D1F8602246
:1048C000002A55D0464E4FF00807FBF777FE2C7AAA
:1048D000002C53D041F24442C2F20102108801463A
:1048E00010F0020F55D04FF0010404F1010441FA19
:1048F00004F212F0010FF8D14FF0010101FA04F1B6
:10490000084341F24443C2F20103188044B9688964
:10491000FFF74AF9B060A889FFF746F9F06042E076
:104920006A89B260A989F1603DE041F6F836C2F2C9
:1049300001064FF000071EE02A4E4FF001071AE073
:10494000294E4FF0020716E0284E4FF0030712E001
:10495000274E4FF004070EE0264E4FF005070AE001
:10496000254E4FF0060706E0244E4FF0070702E001
:104970001B4E4FF00807072FA9D9A6E741F2444381
:10498000C2F20103188840F0010119804FF00004C1
:10499000BDE740F0020441F24443C2F201031C802F
:1049A0004FF00104BCE741F65C60C2F2010007551C
:1049B000374647F8205B38464FF000014FF01C02A5
:1049C00012F010FB34626B68B36306F110004FF015
:1049D00006012A683B4600F0BBF92046F8BD00BF3F
:1049E000581E0120441C0120901C0120DC1C0120C9
:1049F000281D0120741D0120C01D01200C1E012056
:104A0000022907D140F60003C5F200031A6860F3DB
:104A10000A121A60704700BF10B54FF0000440F64C
:104A20003403C5F200031C6040F60400C5F2000028
:104A3000026842F0010101602046FFF711FC4FF0CF
:104A40000100FFF70DFC4FF00200FFF709FC4FF0EB
:104A50000300FFF705FC4FF00400FFF701FC4FF0E7
:104A60000500FFF7FDFB4FF00600FFF7F9FB4FF0E5
:104A70000700FFF7F5FB4FF0FF30FFF731FC41F285
:104A80004643C2F201031C8040F61800C5F2000044
:104A90004FF0FF32026049F69841C0F60301086802
:104AA00040F61C03C5F20003186049F6E432C0F674
:104AB0000302116840F61400C5F20000016049F6D7
:104AC0007C43C0F603031A6840F61001C5F20001EA
:104AD0000A6020464FF00201FFF792FFFFF7AAF8A5
:104AE0002046FFF72BFC4FF00100FFF727FC4FF0AB
:104AF0000200FFF723FC4FF00300FFF71FFC4FF00D
:104B00000400FFF71BFC4FF00500FFF717FC4FF008
:104B10000600FFF713FC4FF00700FFF70FFC10BD76
:104B200008B5FFF779FF08BD704700BFF0B585B045
:104B3000054641F28830FCF7B7FE002D62D043F6FF
:104B40003401C4F202010C6844F080060E604FF09C
:104B5000000400944FF0030601964FF00A070297F5
:104B600020464FF00B0132462346FCF777FA0094BB
:104B70000196029720464FF00C0132462346FCF77F
:104B80006DFA40F20C06C5F20006336843F04002AD
:104B90003260FFF757FC40F23800C5F200004FF4D6
:104BA0000411016044F6206003F002FEFCF774FE7D
:104BB000336843F0400064F3082064F349204FF069
:104BC000050262F38D2064F35D7040F08041316036
:104BD00044F6206003F0ECFDFCF75EFEFFF7C6FC38
:104BE00040F20803C5F2000340F28110186044F25D
:104BF0004520C0F602004FF00F014FF04302FBF7D3
:104C0000A5FD13E04FF000004FF00F014FF04302FD
:104C1000FBF79CFD4FF0000340F23802C5F20002A2
:104C2000136040F21800C5F2000003602846FFF749
:104C30007BFF4FF06400FCF737FE05B0F0BD00BF0E
:104C40002DE9F04182B049F6A047C0F6030744F6CB
:104C50002156C0F6020640F2A015C2F200054FF040
:104C60000408CDF8008038464FF0800132462B46CC
:104C700001F026FE41F24844C2F201042060CDF862
:104C8000008038464FF08101324605EB080301F001
:104C900017FE6060CDF8008038464FF08201324642
:104CA00005F1080301F00CFEA060CDF80080384645
:104CB0004FF08301324605F10C0301F001FEE06084
:104CC000CDF8008038464FF08401324605F11003DC
:104CD00001F0F6FD2061CDF8008038464FF08501E7
:104CE000324605F1140301F0EBFD6061CDF8008060
:104CF00038464FF08601324605F1180301F0E0FD19
:104D0000A061CDF8008038464FF08701324605F1AA
:104D10001C0301F0D5FDE06102B0BDE8F08100BFE9
:104D200008B505464FF000060BE0FBF79DFC2C682C
:104D3000616829606660FBF7A1FC22680AB1A0687F
:104D400090472B68B3F1FF3FEFD101F03BFCF8E750
:104D50000260B3F1FF3F18BF8360FF290ED142F21A
:104D6000F443C2F201031A6822B192F829304FEAE3
:104D7000530101E04FF007010173704701F07F011B
:104D80000173704710B14FF000020260704700BF1E
:104D900038B50446FBF768FC0546A4B1636893B9CF
:104DA000227B40F2A010C2F2000050F82210616095
:104DB00040F82240227B41F24843C2F2010353F8FB
:104DC000220001F031FC2846FBF758FC38BD00BF3B
:104DD00010B5044641F25860C2F201004FF00001E4
:104DE0004FF0240212F0FEF8D4B141F2B040C2F20A
:104DF00001004FF000014FF0480212F0F3F841F2C9
:104E00002C50C2F201004FF000014FF0240212F0CA
:104E1000E9F841F22453C2F201034FF002021A7082
:104E200010BD00BF38B549F6C443C0F6030353F8BC
:104E3000205041F2F841C2F2010151F8204049F6F8
:104E4000F442C0F60302105CFCF79CF92840A04233
:104E500014BF0020012038BD49F6F443C0F6030317
:104E60001A5C41F22C51C2F2010151F8222049F69C
:104E7000C443C0F6030353F8200002420CBF0020D5
:104E80000120704770B441F6C003C2F2010353E839
:104E9000002F02F1010243E800210129F7D049F671
:104EA000F442C0F60302155C41F25861C2F20101FE
:104EB00051F8254049F6C446C0F6030656F82020AE
:104EC00024EA020041F8250053E8005FA5F101053E
:104ED00043E80056012EF7D053E8005FB5F1004FCC
:104EE0000DD14FF0000543E80056012EF4D04EF6E8
:104EF0000450CEF20000016841F080510160BFF320
:104F00002F8F14420CBF0020012070BC704700BFDF
:104F100049F60053C0F60303185C704710B5044609
:104F2000FCF730F940F2C013C2F2000353F824102A
:104F3000484010BD10B504464FF00100FFF748FF90
:104F400049F60C53C0F6030353F8342041F22851BC
:104F5000C2F201010A6003EBC404606841F25453D9
:104F6000C2F20103186010BD00B585B04FF000001B
:104F7000FFF7E0FF4FF00003009341F25852C2F2F6
:104F8000010201924FF04000029049F6E840C0F65D
:104F900003004FF0020145F23D02C0F6020201F0AB
:104FA0007BFB41F21C53C2F20103186005B000BD47
:104FB0002DE9F001804600283CD04FF000034FEA75
:104FC0008302086850F823404D6855F8236086EA4C
:104FD0000407886850F8235084EA050C4CEA070758
:104FE0006FEA070CC86850F8235026EA050707EA5D
:104FF0000C0705EA0C0C66EA0C06354040F8235015
:10500000CD6855F82300384345F823000D6955F85D
:105010002300384345F823004D690DB145F823704E
:1050200048688558886885504868845003F10103B2
:105030004345C4D1BDE8F001704700BF2DE9F843F6
:1050400041F22858C2F2010841F25056C2F201065C
:1050500041F26844C2F201044FF0000541F2545796
:10506000C2F20107D8F8000000EB800001F072FCEA
:105070003368002B40F04381204629464FF024023C
:1050800011F0B0FF3BE14FF0090049F6AC41C0F62A
:105090000301FFF78DFF41F22453C2F20103197897
:1050A00059B101F1FF3041F22452C2F201021070F5
:1050B00041F25863C2F201031D6041F22051C2F275
:1050C0000101086848B941F22052C2F2010215609C
:1050D000136813B1284605F00FFF41F22451C2F2C4
:1050E0000101087858B100F1FF3341F22452C2F2B5
:1050F0000102137041F25861C2F201014D6041F2A8
:105100002050C2F2010003684BB941F22052C2F2B2
:1051100001021560116811B1284605F0EDFE41F25B
:105120002450C2F2010003785BB103F1FF3141F278
:105130002452C2F20102117041F25860C2F2010021
:10514000856041F22053C2F20103196849B941F266
:105150002052C2F201021560106810B1284605F015
:10516000CBFE41F22453C2F20103197859B101F187
:10517000FF3041F22452C2F20102107041F2586332
:10518000C2F20103DD6041F22051C2F20101086860
:1051900048B941F22052C2F201021560136813B1FE
:1051A000284605F0A9FE41F22451C2F20101087817
:1051B00058B100F1FF3341F22452C2F201021370E0
:1051C00041F25861C2F201010D6141F22050C2F278
:1051D000010003684BB941F22052C2F2010215608E
:1051E000116811B1284605F087FE41F22450C2F241
:1051F000010003785BB103F1FF3141F22452C2F2A6
:105200000102117041F25860C2F20100456141F2A1
:105210002053C2F20103196849B941F22052C2F287
:1052200001021560106810B1284605F065FE41F2D4
:105230002453C2F20103197859B101F1FF3041F250
:105240002452C2F20102107041F25863C2F201030B
:105250009D6141F22051C2F20101086848B941F252
:105260002052C2F201021560136813B1284605F0FE
:1052700043FE41F22451C2F20101087858B100F115
:10528000FF3341F22452C2F20102137041F258611D
:10529000C2F20101CD6141F22050C2F20100036867
:1052A0004BB941F22052C2F201021560116811B1EE
:1052B000284605F021FE41F22450C2F20100037895
:1052C0005BB103F1FF3141F22452C2F201021170CD
:1052D00041F25860C2F20100056241F22053C2F26D
:1052E0000103196849B941F22052C2F20102156066
:1052F000106810B1284605F0FFFD3560B2E6D4F81D
:1053000000902846FFF70AFE40EA09012160D4F820
:1053100004904FF00100FFF701FE40EA09026260CD
:10532000D4F808904FF00200FFF7F8FD40EA0900BA
:10533000A060D4F80C904FF00300FFF7EFFD40EAB7
:105340000903E360D4F810904FF00400FFF7E6FD86
:1053500040EA09012161D4F814904FF00500FFF7ED
:10536000DDFD40EA09026261D4F818904FF00600B2
:10537000FFF7D4FD40EA0900A061D4F81C904FF07B
:105380000700FFF7CBFD40EA0903E361D4F8209062
:105390004FF00800FFF7C2FD40EA090121623068C2
:1053A00000F1010030603A689042FFF45BAE6AE6BB
:1053B00000B585B04FF00003009341F2B462C2F231
:1053C000010201924FF04000029049F62C60C0F6B5
:1053D00003004FF0060145F2F132C0F6020201F07F
:1053E0005BF941F27C63C2F20103186005B000BDB5
:1053F0002DE9F04F85B041F624031E46C2F20106A6
:1054000041F2DC700746C2F2010741F29061C2F23C
:105410000101019101F0D6F83268002AFAD061E169
:10542000E359002B53D02846FFF778FD01996258C5
:10543000605090434BD0E35910EA030247D00399E0
:1054400091F800E049F63469C0F603094FEA4518BF
:1054500041F28061C2F201014FF6FF7C49F62C5AFD
:10546000C0F6030A41F2B87BC2F2010B0095704608
:10547000C2F10003134022EA030218B954F80B509A
:105480002B4221D15FEA136E04D01AF80E3003F1DB
:1054900018030EE01D0C04D01AF8053003F11003B8
:1054A00007E05FEA132E1ABF1AF80E3008331AF815
:1054B0000330434419F8035031F815E0E6451CBFAA
:1054C0000EF1010E21F815E0002AD1D1009D05F161
:1054D000010504F10404092DA2D1029C621E02926E
:1054E00040F0F7800399087800F10100C3B20B7017
:1054F0000B2B03D14FF000040C7002E0002B40F0A6
:10550000E58041F60002C2F20102116891B16FEA32
:1055100001003B6803403B6041F2B875C2F20105EF
:105520002C682040286041F60001C2F201014FF0D2
:1055300000020A6041F60000C2F20100436893B124
:105540006FEA03057C682C407C6041F2B872C2F2BD
:10555000010251680D40556041F60000C2F20100A1
:105560004FF00003436041F60005C2F20105AC684C
:1055700094B16FEA0400BA680240BA6041F2B873AD
:10558000C2F2010399680840986041F60005C2F232
:1055900001054FF00004AC6041F60000C2F20100CA
:1055A000C26892B16FEA0203F9681940F96041F2EA
:1055B000B875C2F20105EC682340EB6041F60000CB
:1055C000C2F201004FF00002C26041F60003C2F2D5
:1055D0000103196991B16FEA01053C692C403C61F6
:1055E00041F2B870C2F2010002691540056141F64E
:1055F0000003C2F201034FF00001196141F60005FA
:10560000C2F201056C6994B16FEA04007A69024044
:105610007A6141F2B873C2F20103596908405861D6
:1056200041F60005C2F201054FF000046C6141F63D
:105630000000C2F20100826992B16FEA0203B96907
:105640001940B96141F2B875C2F20105AC69234055
:10565000AB6141F60000C2F201004FF0000282612E
:1056600041F60003C2F20103D96991B16FEA010565
:10567000FC692C40FC6141F2B870C2F20100C269C1
:105680001540C56141F60003C2F201034FF000016D
:10569000D96141F60005C2F201052C6A94B16FEAA6
:1056A00004003A6A02403A6241F2B873C2F201035E
:1056B000196A0840186241F60005C2F201054FF070
:1056C00000042C624FF4FA70029002E04FF4FA7575
:1056D00002954FF0010001F03DF93268002A3FF4D5
:1056E00099AE07E04FF4FA75029541F2B474C2F234
:1056F000010403944FF00004254691E610B54FF0E5
:10570000000441F62403C2F201031C6041F2B870A8
:10571000C2F2010021464FF00902FAF75FFF41F2A1
:10572000DC70C2F2010021464FF00902FAF756FF81
:1057300041F60000C2F2010021464FF00902FAF7DB
:105740004DFF41F29060C2F2010021464FF0090284
:10575000FAF744FF41F28060C2F2010021464FF0A7
:10576000100211F03FFC41F2B470C2F2010004706B
:1057700010BD00BF70B549F6F443C0F603031B5CCF
:1057800049F6C442C0F6030252F8202041F6240034
:10579000C2F20100046841F2DC75C2F2010555F85D
:1057A0002300104206D104F1010641F62405C2F29D
:1057B00001052E6049B141F2B871C2F2010151F800
:1057C0002350154341F8235009E041F2B871C2F269
:1057D000010151F8235025EA020541F823501043F6
:1057E00041F2DC71C2F2010141F8230041F60001EF
:1057F000C2F2010151F8230020EA020241F82320FD
:1058000034B941F27C63C2F20103186800F00CFF66
:1058100070BD00BF30B449F6F443C0F603031B5C0F
:1058200049F6C442C0F6030252F8202041F2DC706F
:10583000C2F2010050F82300104229D041F624049E
:10584000C2F20104256805F10105256071B141F638
:105850000001C2F2010151F82340144341F82340F2
:1058600041F2B471C2F20101097889B96FEA02020A
:1058700041F2B871C2F2010151F82340144041F8DD
:105880002340024041F2DC70C2F2010040F82320C4
:1058900030BC704730B4034641F6C002C2F2010288
:1058A00052E8000F00F1010042E80004012CF7D09B
:1058B00041F28060C2F2010030F8132039B141F2A8
:1058C0008061C2F201014FF0000421F8134041F65B
:1058D000C003C2F2010353E8004FA4F1010443E8FE
:1058E0000045012DF7D053E8004FB4F1004F0DD122
:1058F0004FF0000443E80045012DF4D04EF604506B
:10590000CEF20000016841F080510160BFF32F8F9B
:10591000104630BC704700BF41F2B473C2F20103BD
:105920001878D0F1010038BF002070472DE9F84FFA
:10593000DFF834814B4FC8EB07004FEAD00707F17F
:1059400001074FF0000540F2982AC0F6000A40F225
:105950006039C0F6000931E044464FF000066FEAB6
:10596000060B0BEB070101F0010B58F8043CAB42AE
:1059700029D135E054F8043CAB4205D154F8080C69
:105980008047FBF789FF0BE0FF2B09D9FF2D07D1DB
:1059900054F8040C4FF0070154F8082C00F09CFF59
:1059A00006F1010604F1080454F8041CA94240D190
:1059B0004CE005F10105B5F5807F02D0CA45CBD397
:1059C000F7E7BDE8F88FFF2B0FD9FF2D0DD158F861
:1059D000040C4FF0070158F8082C00F07DFF04E09C
:1059E00058F8082C9047FBF757FF06F1010604F121
:1059F0000804BE42DDD0BBF1000FBBD054F8040C4C
:105A0000A8420AD0FF280DD9FF2D0BD14FF0070176
:105A100054F8082C00F060FF04E054F8081C884794
:105A2000FBF73AFF06F1010604F10804BE42A1D1DA
:105A3000BFE7FF290FD9FF2D0DD154F8040C4FF00B
:105A4000070154F8082C00F047FF04E054F8082C34
:105A50009047FBF721FF06F1010604F10804BE425E
:105A600088D1A6E767030008A0020008027841F683
:105A70008D03C2F201031B789A4206D34FF0000255
:105A80000270087800F1010008700A7841F68E0370
:105A9000C2F201031878824224BF002008707047C8
:105AA00010B5A0F10803052B3DD8DFE803F01F3C3B
:105AB0002C3C038341F62C00C2F201004FF0200180
:105AC0004FF0540211F08EFA41F68000C2F201004C
:105AD0004FF0FF314FF00C0211F084FA41F69400C0
:105AE000C2F20100026802F1010202604FF00001FF
:105AF00041F62803C2F20103197041F62900C2F2EF
:105B00000100017056E041F62801C2F201014FF098
:105B100000030B7041F62900C2F20100027802F185
:105B2000010202703CE041F62802C2F20102127842
:105B300041F62901C2F201010B7841F68D01C2F252
:105B40000101097801FB032341F62C01C2F2010196
:105B5000C95C81421DD041F62C04C2F20104E0541C
:105B60004FEA531041F68001C2F2010103F01F0316
:105B70004FF0010404FA03F351F820401C4341F8AC
:105B8000204041F69400C2F20100016801F10101D8
:105B9000016002F1010241F62803C2F201031A700A
:105BA00041F62800C2F2010041F62901C2F20101CA
:105BB000FFF75CFF4FF0000010BD00BF70B4039D05
:105BC000049C064628B141F69000C2F2010000781C
:105BD000307029B141F69800C2F2010000780870D7
:105BE0002AB141F68C01C2F20101087810702BB184
:105BF00041F69902C2F20102117819702DB141F6F5
:105C00002803C2F20103187828702CB141F629024A
:105C1000C2F201021178217070BC704706281DD8AD
:105C2000002808BF052041F69003C2F20103187056
:105C300049F65473C0F6030313F8101041F68D02B1
:105C4000C2F20102117003EB4000417841F68E036D
:105C5000C2F2010319704FF0010070474FF00000CD
:105C6000704700BF08B541F69803C2F201034FF038
:105C700001021A704FF00500FFF7D0FF4FF00C0043
:105C80004FF00001FFF70CFF08BD00BF08B541F65B
:105C90002802C2F20102107041F62903C2F2010388
:105CA000197010461946FFF7E1FE08BD034628B1FA
:105CB00041F68D00C2F201000078187029B141F65A
:105CC0008E03C2F20103187808702AB141F69401DC
:105CD000C2F201010B68136041F62C00C2F2010010
:105CE000704700BF2DE9F00141F62C07C2F2010711
:105CF0003F1853284BD8002A49D03B4607F10107EB
:105D000002F1FF3257FA82F74FF0000641F68004A5
:105D1000C2F201044FF001056FEA030C0CEB07021D
:105D200002EA050C13F8018B01F1FF3111F8012F84
:105D300090452FD13DE013F801CB01F101004978E6
:105D40008C450ED003F8011C4FEA521102F01F06D9
:105D500005FA06FC54F821604CEA060644F8216076
:105D60002E4602F10102D2B2542A07D013F801CB19
:105D700000F101014078844542D150E03EB141F646
:105D80009403C2F20103196801F101011960BDE831
:105D9000F001704703F8012C4FEA501600F01F087D
:105DA00005FA08F854F8262048EA020244F82620AA
:105DB0002E4600F10100C2B2542ADFD0BB42DDD032
:105DC000BCF1000FB7D013F801CB11F8010F8445D7
:105DD0000ED003F8010C4FEA521002F01F0605FA2C
:105DE00006FC54F820604CEA060644F820602E4673
:105DF00002F10102D2B2542AC0D0BB429BD1BDE70E
:105E000003F8010C4FEA521002F01F0605FA06FCD7
:105E100054F820604CEA060644F820602E4602F151
:105E20000102D2B2542AA9D0BB4284D1A6E700BF56
:105E3000003018BF012041F69803C2F20103187028
:105E4000003118BF012141F68C00C2F2010001703F
:105E5000003218BF012241F69903C2F201031A7001
:105E6000704700BF41F68F03C2F201034FF00002FA
:105E70001A7070474FF05400704700BF41F68F030F
:105E8000C2F201034FF001021A707047034628B1B5
:105E90000868834214BF0020012070474FF00000C3
:105EA000704700BF10B441F6C003C2F2010353E8CB
:105EB000002F02F1010243E800210129F7D0046814
:105EC000C4B16268824202D19268626002E04368B3
:105ED000816899602368834202D15B68236002E095
:105EE000826841685160A26802F1FF31A1604FF001
:105EF0000004046041F6C003C2F2010353E8002F1E
:105F0000A2F1010243E80024012CF7D053E8002F4E
:105F1000B2F1004F0DD14FF0000243E80024012CF4
:105F2000F4D04EF60450CEF20000016841F08051EA
:105F30000160BFF32F8F10BC704700BF38B5044617
:105F40000D464FF000014FF0100211F04BF8E560E4
:105F500038BD00BFF8B504460F46C6688D192946FE
:105F6000FFF794FF00283CD141F6C003C2F20103C1
:105F700053E8002F02F1010243E800210129F7D084
:105F80004FF0000068606168A96001B14D6022684F
:105F900002B925606560BC51A36803F10103A360E9
:105FA00041F6C003C2F2010353E8002FA2F101023F
:105FB00043E80024012CF7D053E8002FB2F1004F42
:105FC0000DD14FF0000243E80024012CF4D04EF62E
:105FD0000450CEF20000016841F080510160BFF32F
:105FE0002F8FF8BD2DE9F04104468846C6688D190B
:105FF0009719C2B941F6C003C2F2010353E8002F5A
:1060000002F1010243E800210129F7D002686A6029
:1060100005604FF00000A860616809B9656020E084
:106020006B689D601DE03946FFF730FF00283FD0C8
:106030002846FFF737FF41F6C003C2F2010353E8D9
:10604000002F02F1010243E800210129F7D0B868CE
:10605000A8606F60BD602168B9420EBF2560A96865
:106060004D6048F80640A26802F10102A26041F6C4
:10607000C003C2F2010353E8002FA2F1010243E87A
:106080000024012CF7D053E8002FB2F1004F0DD1BE
:106090004FF0000243E80024012CF4D04EF60450E7
:1060A000CEF20000016841F080510160BFF32F8FF4
:1060B000BDE8F081C368C918486808B1C01A7047C4
:1060C0004FF00000704700BF036813B1C068181A92
:1060D00070474FF00000704708B5C368C918FFF754
:1060E000D5FE08BD08B5C0680818FFF7DBFE08BD7F
:1060F00008B541F69C00C2F201004FF01C01FFF709
:106100001DFF08BD70B5054600F108063046FFF7D3
:10611000DBFF0446686050B130462146FFF7E2FFDE
:106120004FF00100A861204600F07EFA70BD4FF0EC
:106130000003AB6170BD00BF38B504460D464FF09B
:1061400000014FF0280210F04DFF204640F8085B98
:106150004FF01C01FFF7F2FE41F69C00C2F2010075
:106160002146FFF7F7FE38BD2DE9F0410746884686
:1061700042F2F443C2F201031868002800F0FE80E6
:1061800041F6C004C2F2010454E8002F02F10102FA
:1061900044E800210129F7D0796831B142F2F44294
:1061A000C2F20102136899422ED142F2F440C2F2C7
:1061B000010004687C60B96901F10101B96141F62F
:1061C000C003C2F2010353E8002FA2F1010243E829
:1061D0000024012CF7D053E8002FB2F1004F0DD16D
:1061E0004FF0000243E80024012CF4D04EF6045096
:1061F000CEF20000016841F080510160BFF32F8FA3
:106200004FF00100BDE8F081B8F1FF3F24D141F625
:10621000C003C2F2010353E8002FA2F1010243E8D8
:106220000024012CF7D053E8002FB2F1004F0DD11C
:106230004FF0000243E80024012CF4D04EF6045045
:10624000CEF20000016841F080510160BFF32F8F52
:106250004FF00000BDE8F08107F108052846FFF780
:1062600033FF0246F0B142F2F446C2F20106306852
:1062700092F8294090F829108C4208D912E033682E
:1062800092F8290093F82940A04204D90AE042F28A
:10629000F446C2F2010628461146FFF70BFF0246FC
:1062A0000028ECD1284642F2F441C2F2010109680B
:1062B000FFF798FE41F6C006C2F2010656E8002F2D
:1062C000A2F1010246E80024012CF7D056E8002F85
:1062D000B2F1004F0DD14FF0000246E80024012C2E
:1062E000F4D04EF60450CEF20000016841F0805127
:1062F0000160BFF32F8FB8F1000F04D008EB8800C6
:1063000000F028FB01E000F05DF941F6C004C2F2A4
:10631000010454E8003F03F1010344E80032012A7C
:10632000F7D042F2F446C2F2010628463168FFF780
:10633000D9FE54E8003FA3F1010344E80032012AEA
:10634000F7D054E8003FB3F1004F0DD14FF00003F8
:1063500044E80032012AF4D04EF60450CEF2000098
:10636000016841F080510160BFF32F8F7868326877
:10637000904214BF00200120BDE8F0814FF00100E1
:10638000BDE8F08110B5044642F2F443C2F20103C5
:106390001868002860D06268904201D0FAF70EF9C0
:1063A00041F6C003C2F2010353E8002F02F10102DB
:1063B00043E800210129F7D0A16901F1FF30A06174
:1063C00018B341F6C003C2F2010353E8002FA2F153
:1063D000010243E80024012CF7D053E8002FB2F16A
:1063E000004F0DD14FF0000243E80024012CF4D0FF
:1063F0004EF60450CEF20000016841F08051016079
:10640000BFF32F8F4FF0000010BD2046FFF77AFE3C
:1064100041F6C003C2F2010353E8002FA2F10102CA
:1064200043E80024012CF7D053E8002FB2F1004FCD
:106430000DD14FF0000243E80024012CF4D04EF6B9
:106440000450CEF20000016841F080510160BFF3BA
:106450002F8F4FF0010010BD4FF0010010BD00BFA5
:10646000F8B5054641F6C003C2F2010353E8002F18
:1064700002F1010243E800210129F7D041F69C0016
:10648000C2F20100FFF720FE0446E0B141F69C078E
:10649000C2F201076068A84203D12046FFF732FE2E
:1064A0000AE004F1080630462946FFF715FE18B148
:1064B00030462946FFF716FE38462146FFF7FAFD1B
:1064C00004460028E6D141F6C003C2F2010353E8B6
:1064D000002FA2F1010243E80024012CF7D053E879
:1064E000002FB2F1004F0DD14FF0000243E800241D
:1064F000012CF4D04EF60450CEF20000016841F0B9
:1065000080510160BFF32F8FF8BD00BF08B549F679
:106510006073C0F60303195C012906D011B102298A
:106520000BD105E0FDF7FEFA08BD02F001F908BD48
:10653000FAF744F84FF0000008BD4FF0000008BD26
:106540004EF60453CEF200031A6842F080501860F1
:10655000704700BF4FF0010280F8282041F6BC03CD
:10656000C2F2010390F8291002FA01F218880243DE
:106570001A80704710B441F6B803C2F201031A68DA
:10658000C2B1904213D104E088420FD102F114024B
:1065900003E041F6B802C2F2010243691BB19C69F3
:1065A0008169611899614369136003E00A46516982
:1065B0000029E9D14FF0000282614FF0FF314161C3
:1065C00010BC704710B5FAF74FF8044642F2F44396
:1065D000C2F20103186890F82820032A1BD0FAF7AA
:1065E00043F842F2F443C2F2010319684FF000028B
:1065F00081F8282091F82920096941F6AC13C2F2EC
:10660000010343F82210FAF739F82046FAF736F872
:10661000FFF796FF10BD4FF0020180F828102046CA
:10662000FAF72CF810BD00BF38B5044690B30368E4
:1066300083B3FAF719F8054694F8280010BB2046F2
:10664000FFF788FF42F2F441C2F201010B6843B147
:1066500094F8292093F8290020F00101531A002B07
:1066600015DA41F6C002C2F20102106838B140F0FA
:10667000004141F6C003C2F20103196007E0FFF7D1
:106680005FFF04E0022804BF032084F828002846A6
:10669000F9F7F4FF38BD00BF2DE9F04F85B006468D
:1066A0000F46934698460F9DDDF84090F9F7DCFFC2
:1066B000824641F60413C2F2010319685048814230
:1066C0000FD240F20002C2F2020252F82C4C54B136
:1066D0004C4B1C468B4207D953F82C090028F8D1A3
:1066E00002E0474C00E0464CA14206D1A1F12C014A
:1066F00041F60412C2F20102116020464FF000017F
:106700004FF02C0210F06EFC4FF0FF3161611EB9AA
:1067100049F66476C0F603062660B8F1000F08D08B
:106720000E9B042B08D9184600F103004FEA90068F
:1067300004E04FF0000601E04FF000060DBB42F60A
:10674000F879C2F2010941F6AC05C2F201052968E7
:1067500046F6B530C0F602000090CDF804800296EF
:1067600048464FF000025B46FAF7B6FA2A68A26084
:10677000E0604FEA800153182B60C1EB09006060B4
:1067800020E028464FF0FF314A46F9F727FF4AF24A
:10679000ED52CDF6CE622A60E56005EB89056560B5
:1067A00046F6B531C0F602010091CDF8048002969C
:1067B000284629464FF001025B46FAF78DFAA5EB11
:1067C000800363606FEA0702C2F3C01101EB470761
:1067D00007F0FF0784F8297041F6C403C2F20103F1
:1067E00053F82700206143F827405046F9F746FF49
:1067F0002046FFF719FF204605B0BDE8F08F00BF27
:10680000D4FF0120A8FF012030B585B04FF0000172
:1068100042F2F443C2F201031960284C40F2000531
:10682000C2F202052A1B20464FEAA202F9F7D6FE61
:1068300041F6AC00C2F201000460A5F12C0541F65E
:106840000411C2F201010D6042F2F873C2F20103B9
:106850004FF0B504CBF26B141C6003F14C004FF009
:10686000FF3243F8042F43F8042F43F8042F8342E8
:10687000F9D14FF00004009441F60811C2F2010171
:1068800001914FF02803029349F67070C0F603009F
:106890004FF0070146F63512C0F602022346FFF715
:1068A000FBFE41F6A812C2F20102106041F6C400DC
:1068B000C2F20100C46305B030BD00BFFC2F01204F
:1068C00010B584B0069C00944FF00004019402942B
:1068D000FFF7E2FE04B010BD00B585B04FF0000335
:1068E000009301930293FFF7D7FE05B000BD00BFF0
:1068F00038B542F2F443C2F201031868C0B1F9F7A7
:10690000B3FE054642F2F444C2F201042068FFF7E8
:1069100021FE216891F82920086941F6AC13C2F2E2
:10692000010343F822002846F9F7A8FEFFF708FE06
:1069300038BD00BF38B542F2F445C2F2010541F658
:10694000C404C2F201042B6822681A61FFF7D0FF69
:10695000F9E700BF38B542F2F443C2F20103196807
:10696000002900F0918020B9FFF7C2FF4FF001022B
:106970009AE0B0F1FF3F04D1FFF724FE4FF0000290
:1069800092E041F6C004C2F2010454E8002F02F183
:10699000010244E800210129F7D041F6B802C2F211
:1069A00001021568002D7AD0AB6998426FD3C01AE6
:1069B00005F114016D691DB1AB698342F7D96AE035
:1069C00042F2F445C2F201052B68986108685861EB
:1069D0001846F9F7F7FD41F6C004C2F2010454E885
:1069E000003FA3F1010344E80032012AF7D054E844
:1069F000003FB3F1004F0DD14FF0000344E80032E7
:106A0000012AF4D04EF60450CEF20000016841F0A5
:106A100080510160BFF32F8FFFF7D4FD54E8003F92
:106A200003F1010344E80032012AF7D028684169E4
:106A3000B1F1FF3F04D0FFF79DFD4FF0000201E0F0
:106A40004FF0010241F6C003C2F2010353E8004FC8
:106A5000A4F1010443E80045012DF7D053E8004FAD
:106A6000B4F1004F0DD14FF0000443E80045012D73
:106A7000F4D04EF60450CEF20000016841F080518F
:106A80000160BFF32F8F0FE04FF001020CE041F6E1
:106A9000B801C2F20101AC69221AAA6190E741F67D
:106AA000B801C2F201018BE7104638BDF8B50446C3
:106AB00000287AD0F9F7D8FD064641F60413C2F251
:106AC000010319683948814211D240F20002C2F232
:106AD000020252F81C5CA54263D0354B1D468B4226
:106AE00005D9A3F12C03D86BA042F7D15AE094F852
:106AF000293041F6C402C2F2010252F82300A0423A
:106B000006D1016941F6C402C2F2010242F8231023
:106B10002046FFF72FFD2046FFF7A2FC94F829003E
:106B2000236941F6AC11C2F2010141F8203042F272
:106B3000F442C2F201021068A04229D0A06838B322
:106B4000E76800EB870541F6AC07C2F201073B6836
:106B50005A1B29464FEAA2024FF00003FBF7D0FD73
:106B6000E1683868A0EB81033B6041F60412C2F291
:106B7000010211680D4B99420AD29A68954203D8D6
:106B8000E068A2EB80029A60A3F12C038B42F4D858
:106B90004FF00001216084F828103046F9F76EFDAF
:106BA000F8BD024D21692961A1E7F8BDD4FF01209C
:106BB000A8FF012000BFF04772B642F2F444C2F2CF
:106BC00001042068FFF772FF4FF000032360FAF71B
:106BD000D3F800BF41F6B803C2F20103196849B106
:106BE000886950B100F1FF328A61D2F1010038BFEB
:106BF000002070474FF0000070474FF000007047D2
:106C000070B541F6B803C2F201031C68A4B1A069D3
:106C100090B941F6B805C2F201054FF0FF36606940
:106C20002946F9F7CFFC66612046FFF7FDFC2C688A
:106C300014B1A1690029F2D070BD00BFF0B472B6E2
:106C400041F6BC03C2F201031C882CB941F6A8131B
:106C5000C2F2010318685FE049F6787CC0F6030CC5
:106C600041F6AC15C2F2010541F6C406C2F20106B6
:106C7000C4F1000323401A0A1ABF1CF8021008319D
:106C80001CF8031011F0010F0AD141F0010055F872
:106C9000200038B190F82820012A38D81F4602E099
:106CA0001F4600E01F4655F82120B2B192F8283067
:106CB0007BB141F6BC00C2F20100048010462BE01B
:106CC00090F8283033B141F6BC02C2F201021480C0
:106CD00022E0104600690028F2D156F821008242D5
:106CE00007D1BC43C4D141F6BC01C2F201010C8002
:106CF000ACE745F8210011F0010FD4D114EA4703A5
:106D0000D1D04FEA4707BFB241F00101CBE741F6CE
:106D1000BC01C2F201010C8062B6F0BC704700BF3A
:106D200070B542F2F443C2F201031B6883420FD1F3
:106D300093F82820012A9CBF022283F8282093F888
:106D4000291041F6AC10C2F2010040F8213070BDAC
:106D500041F6B002C2F20102136042F2F441C2F203
:106D60000101086090F8292041F6AC13C2F201033A
:106D700043F8220090F8281001299CBF022180F8D6
:106D800028108268AAB9C1684AF2ED53CDF6CE63E5
:106D90000868984201D0F9F711FC42F2F442C2F2BD
:106DA000010211684868CB6898427ED2F9F706FC68
:106DB00070BD41F6B403C2F201031B68984274D05F
:106DC00093B3586842F6F874C2F20104251A4FEAE8
:106DD000A501D96042F2F872C2F2010290420AD3D0
:106DE0004FF0B503CBF26B1342F2F870C2F2010020
:106DF00004689C4201D0F9F7E1FB41F6B405C2F208
:106E000001052A6841F6AC04C2F201042068516809
:106E1000D2684FF00003FBF773FC296823688B608E
:106E2000C86803EB8002226042F2F441C2F2010121
:106E30000B6841F6B400C2F201000360DA68002A70
:106E400033D0586899684FF00103FBF759FC42F2C0
:106E5000F446C2F201063568A868EC6800EB8404C9
:106E600041F6AC06C2F201063268131B21464FEA16
:106E7000A3024FF00003FBF743FCE9683068A0EB86
:106E80008102326041F60413C2F201031968074B14
:106E900099420AD29A68944203D8E868A2EB800229
:106EA0009A60A3F12C038B42F4D870BDD4FF01206B
:106EB00000B585B041F64830C2F201004FF0000144
:106EC000FFF73CF841F6F010C2F201004FF000016C
:106ED000FFF734F84FF00003009341F60822C2F2A6
:106EE000010201924FF0500002904AF27800C0F681
:106EF0000300194647F20522C0F60202FFF7CCFB59
:106F000041F6EC13C2F20103186005B000BD00BFEA
:106F100008B5FFF7D9F8034648B1C06850B100F191
:106F2000FF31D960D1F1010038BF002008BD4FF01A
:106F3000000008BD4FF0000008BD00BF70B5054659
:106F40000E46144641F6C003C2F2010353E8002F77
:106F500002F1010243E800210129F7D0FFF7B4F85C
:106F60000246002839D0C06884422DD3241A28460E
:106F70001146FFF79FF8024600282ED0C068A042B5
:106F8000F4D921E041F6C003C2F2010353E8002F17
:106F9000A2F1010243E80024012CF7D053E8002FAE
:106FA000B2F1004F0DD14FF0000243E80024012C54
:106FB000F4D04EF60450CEF20000016841F080514A
:106FC0000160BFF32F8F70BDF460D1680B1BD360DD
:106FD00028463146FFF706F8D4E7F46028463146E4
:106FE000FEF7B8FFCEE700BFF8B50646FFF76CF82E
:106FF0000446F8B1C368EBB930462146FFF75AF8AA
:107000000546F9F731FB074630462146FFF76AF897
:107010003846F9F733FB22691AB130462146FFF7AB
:107020008DFF04F11400FDF7B3FE1DB12C46E86896
:107030000028E1D0F8BD00BF08B541F60423C2F234
:1070400001031A6802F101021A6041F6F010C2F25F
:107050000100FFF75DFF28B141F6F010C2F2010018
:10706000FFF7C2FF08BD00BF08B5014641F6483032
:10707000C2F20100FFF730F820B141F64830C2F209
:10708000010008BD41F6F010C2F2010008BD00BFCA
:1070900070B5044641F6C003C2F2010353E8002F65
:1070A00002F1010243E800210129F7D0FFF7DCFFDC
:1070B00005462146FFF710F8002845D041F6C000EC
:1070C000C2F2010050E8002F02F1010240E8002165
:1070D0000129F7D028462146FEF7ECFF18B1C16818
:1070E000E2688B18C360F9F7BFFA064628462146C6
:1070F000FEF7F8FF3046F9F7C1FA4FF0FF35E560CB
:1071000041F6C003C2F2010353E8002FA2F10102CD
:1071100043E80025012DF7D053E8002FB2F1004FCE
:107120000DD14FF0000243E80025012DF4D04EF6BA
:107130000450CEF20000016841F080510160BFF3BD
:107140002F8F4FF0010501E04FF0000504F114000E
:10715000FDF718FE41F6C003C2F2010353E8002F09
:10716000A2F1010243E80024012CF7D053E8002FDC
:10717000B2F1004F0DD14FF0000243E80024012C82
:10718000F4D04EF60450CEF20000016841F0805178
:107190000160BFF32F8F284670BD00BF2DE9F0417D
:1071A00005460F4614469846FFF772FF064694B10F
:1071B0009DF82030002B14BF20460020286105F1E7
:1071C00014004146069A079BFDF7C2FD3846294642
:1071D0002246FFF7B3FE3046BDE8F08170B584B0BB
:1071E0000E4615460093089C01949DF824300293A6
:1071F00041F64831C2F2010132462B46FFF7CEFF7D
:1072000004B070BD00B583B04FF0000300934FF0A1
:107210000100019041F65830C2F2010041F288317C
:107220004FF0FF0247F23903C0F60203FFF7D6FF23
:1072300041F64834C2F20104FFF7E2FC2046FFF7B2
:10724000D3FEFFF7BFF9F7E741F60023C2F20103CF
:1072500018681A689042FBD1704700BF10B541F61C
:107260000023C2F201031A6802F101021A60FFF75B
:10727000B1FC044641F64830C2F20100FFF748FE77
:10728000204310F0FF0F06D041F6EC10C2F20100CF
:107290000068FFF7C9F910BD08B54AF21C10C0F626
:1072A00003004FF0060147F2D562C0F60202FFF775
:1072B00013FB41F6BC33C2F20103186008BD00BFE6
:1072C00038B504460D4641F6F833C2F20103586A58
:1072D000A0420AD041F6F831C2F201014C620A68BC
:1072E0001AB115B14948FDF753FD41F6F833C2F222
:1072F0000103186F84420AD041F6F831C2F201014D
:107300000C67CA6C1AB115B14148FDF741FD41F651
:10731000F833C2F20103D3F8BC0084420CD041F62A
:10732000F831C2F20101C1F8BC40D1F898201AB17D
:1073300015B13848FDF72CFD41F6F833C2F20103D0
:10734000D3F8080184420CD041F6F831C2F20101B1
:10735000C1F80841D1F8E4201AB115B12E48FDF763
:1073600017FD41F6F833C2F20103D3F85401844209
:107370000CD041F6F831C2F20101C1F85441D1F804
:1073800030211AB115B12548FDF702FD41F6F83359
:10739000C2F20103D3F8A00184420CD041F6F831C7
:1073A000C2F20101C1F8A041D1F87C211AB115B196
:1073B0001B48FDF7EDFC41F6F833C2F20103D3F8A8
:1073C000EC0184420CD041F6F831C2F20101C1F85F
:1073D000EC41D1F8C8211AB115B11248FDF7D8FC1B
:1073E00041F6F833C2F20103D3F83802A0420CD0C0
:1073F00041F6F831C2F20101C1F83842D1F8142245
:107400001AB115B10848FDF7C3FC38BD081C0120AE
:10741000541C0120A01C0120EC1C0120381D01205F
:10742000841D0120D01D01201C1E01202DE9F047E4
:1074300007460D4691460898DDF828800C683E689E
:10744000D8F800108A19944202D80219964203D340
:1074500004192C60BDE8F087341B061BB14234BF11
:107460008A46B246099931B1D9F8000008181919AD
:1074700052460FF093FDD8F80030CAEB0302C8F86B
:1074800000203E6806EB0A013960D9F8000000EBE5
:107490000A03C9F800302E68A41954442C60BDE8D2
:1074A000F08700BF70B584B09CF81960157A947BA2
:1074B0004FF007038CF810304FF005028CF81120C4
:1074C00006F00F0260F3C7128CF812204FF0000094
:1074D00065F301008CF813004FF0000261F30A021B
:1074E000ACF814208CF81640DCF80C100093DCF893
:1074F00004300193CDF808C001F104000CF108023A
:107500000CF11003FFF792FF04B070BD2DE9F04FAE
:107510008FB00746059114464FF0000307931360A0
:1075200012896068131A8B4238BF059305990029A8
:1075300000F0AA8041F6F035C2F201052D6815B3BE
:107540004FEAC5054FF000024FF0FF01134641F628
:107550007060C2F20100A5F10806C6F3C00E16580D
:10756000F6798E4240F0958096E01658F6798E4274
:107570001CBF0133314602F108028658F6798E426B
:1075800040F09F80A0E04FF0000303EB43024FEA7E
:10759000C20000F1100008904FF48071ADF8241083
:1075A0004FF00402ADF826208DF828300DF12900A7
:1075B0004FF000014FF007020FF014FD04F1040B2F
:1075C00004944FF010030093019705A802905846C9
:1075D000214607AA08ABFFF729FF0599002951D0DA
:1075E0004FF001028DF821200DF132004FF0000123
:1075F0004FF006020FF0F6FC41F6F033C2F2010341
:10760000186800283ED04FF0FF014FF0000441F60B
:107610007069C2F201094AF28808C0F6030841F60F
:10762000F03AC2F2010A59F83450ED798D4223D074
:107630008DF820404FEA05160DF1220008EB0601F7
:107640004FF008020FF0AAFC06F108010DF12A0024
:1076500041444FF008020FF0A1FC4FF018020092D5
:10766000019705AB02935846049907AA08ABFFF7A8
:10767000DDFE059830B1294604F10104DAF8002056
:10768000A242D0D8079801E04FF0FF300FB0BDE81C
:10769000F08F03F10103314602F10802AA423FF4E0
:1076A00074AFBEF1000F3FF460AF1658F6798E420A
:1076B0001CBF0133314602F10802AA427FF455AFE4
:1076C00063E703F10103314602F10802AA427FF4A5
:1076D0004CAF5AE72DE9F0414FF00100FDF726FAD3
:1076E0004AF22C10C0F60300FDF7A4F841F6EC3383
:1076F000C2F201034FF001021A7041F6E030C2F20B
:107700000100016841B941F6E034C2F20104FEF71C
:1077100059FF2568002DFAD041F6EF37C2F2010774
:1077200041F6EC34C2F2010441F6EE36C2F2010633
:1077300041F65965C2F2010541F66C68C2F20108D2
:107740003B783BB14FF000023A704FF002002070DE
:10775000FDF7E6F9317859B14FF000033370227824
:1077600062F07F0020704FF001000146FFF7A8FD96
:10777000297851B14FF000002870237803F07F0280
:1077800022704FF00101FFF79BFD98F8000010B93F
:10779000FEF718FFD4E741F6EC31C2F201014FF0D9
:1077A00002030B704FF00000FDF7C0F9BDE8F08157
:1077B00008B541F6E033C2F20103186041F6BC306F
:1077C000C2F201000068FEF72FFF08BD70B5054644
:1077D0000E4641F6F433C2F201031868032801D9BA
:1077E000F8F7ECFE41F6F432C2F20102116841F6FC
:1077F000C034C2F2010444F8316004EBC104656096
:1078000001F10101116070BD70B505460C461646C8
:10781000032801D9F8F7D2FE41F67063C2F20103E2
:1078200053F8350008B1F8F7C9FE41F67061C2F2AD
:10783000010141F8354001EBC5056E6041F6F033BA
:10784000C2F201031A6802F101021A60206930B124
:10785000FCF7F0FF04F1040420690028F8D170BDA2
:1078600008B541F6F833C2F20103196881425AD0D3
:1078700041F6F832C2F20102D36C834234D041F6B1
:10788000F831C2F20101D1F8982082422FD041F69E
:10789000F833C2F20103D3F8E41081422AD041F652
:1078A000F832C2F20102D2F83031834225D041F6DB
:1078B000F831C2F20101D1F87C21824220D041F698
:1078C000F833C2F20103D3F8C81181421BD041F64C
:1078D000F832C2F20102D2F81432834216D0F8F71D
:1078E0006DFE4FF0080013E04FF0010010E04FF084
:1078F00002000DE04FF003000AE04FF0040007E043
:107900004FF0050004E04FF0060001E04FF00700E3
:1079100041F6F831C2F201014FF04C0202FB0010B7
:1079200090F8200008BD4FF00000F1E72DE9F04F7E
:107930008FB0089007910A924FF0000309931360EB
:10794000546813891B1B8B4238BF07930799002982
:1079500000F04A81082C69D841F6F034C2F20104E3
:10796000D4F800E041F6F435C2F201052E680EEBC2
:10797000CE0707EBC60404F109044FF0000141F6FD
:107980007067C2F20107CB598BB1DD68641903F14E
:1079900010051B695BB15E890EB104F107049B8978
:1079A0000BB104F1070455F8043F002BF3D101F1AA
:1079B00008012029E7D141F6E031C2F201010D684A
:1079C0002F7E6E7EEB8A03F10103C3F347054FF070
:1079D00000010C914FF009038DF82C304FF002019B
:1079E0008DF82D10ADF82E408DF830E04FF00101EC
:1079F0008DF831104FF0000167F3451166F38611E1
:107A000061F07F018DF833108DF8345000930190B0
:107A100007A8029002F10400114609AA0BABFFF778
:107A200005FD079A002A00F0DD80E0E04FF0090034
:107A30001060DCE05BF83640002C00F0CE80059D45
:107A4000286800284BD07A68B2420CD04FF000036F
:107A500010F0010F3ED1DFE007EBC3025268B242E3
:107A600040F0E38001E04FF0000357F83300D2B25A
:107A700090F8048090F805C090F806E0C579016898
:107A800019B143F01000C3B201E04FF000034FF012
:107A900008008DF82C004FF00B018DF82D108DF89B
:107AA0002E208DF82F808DF830C08DF831E08DF8C4
:107AB00032508DF833300A990090089A019207AB42
:107AC000029301F1040009AA0BABFFF7AFFC079882
:107AD00028B987E003F101052B468542BCD104F1AA
:107AE000100523697BB129464FF00002588908B17F
:107AF00002F101029B890BB102F1010251F8043F2E
:107B0000002BF3D101E04FF000025FFA86FCD2B205
:107B100094F804E06079A17923681BB146F0200352
:107B2000DBB201E04FF000038DF82CA04FF0040809
:107B30008DF82D808DF82EC04FF0000C8DF82FC0E1
:107B40008DF830208DF831E08DF832008DF833104B
:107B50008DF834300A99CDF800A0089A019207A850
:107B6000029001EB080009AA0BABFFF75FFC079935
:107B7000002937D0A3686BB10A99E268009208988F
:107B8000019007AA029201EB080009AAFFF74EFC38
:107B9000079B3BB3246904B34FF001084FF0000981
:107BA0002046FFF75DFE8DF83500618939B10DF192
:107BB0001C0C40462246FFF775FC079991B1A1893C
:107BC00039B10DF11C0C48462246FFF76BFC0798B3
:107BD00040B155F8044F002CE2D106F10106042E05
:107BE0007FF428AF099814E04FF0FF3011E04FF018
:107BF000000641F6706BC2F2010B41F6F434C2F29A
:107C0000010405944FF0090A41F6C037C2F201079A
:107C100010E70FB0BDE8F08F03F1010307EBC301DC
:107C20004A68B2427FF456AF1FE705F1010307EB44
:107C3000C3014A68B2427FF44DAF16E708B541F67A
:107C40005C63C2F201031A5C41F6F831C2F2010131
:107C50004FF04C0000FB0210436AD3F1010238BF21
:107C6000002242634FF00001C1630164416400F1EE
:107C70001000FDF78DF808BD2DE9F04790B0814662
:107C80008A4641F65C63C2F201031A5C41F6F830A1
:107C9000C2F201004FF04C0404FB020404F1480658
:107CA0004FF001084FF00007354640463146F8F7DF
:107CB00089FC28B14FF002003146F8F783FC36E02A
:107CC000BAF1000F05D148464146FCF7DFFC032816
:107CD00027D0256C75B16846A168E26BA8470546B8
:107CE000B0F1FF3F14D06064484669462A46FCF76D
:107CF000F3FC0EE0616CA5688D4228BF0D46484636
:107D0000E16B2A46FCF7E8FCE36B5A19E26300E0FA
:107D10003D46606CA16888423CBFE7632764451B11
:107D2000656438463146F8F74DFC0228BCD010B0E7
:107D3000BDE8F087F8B505460E46174641F65C6388
:107D4000C2F201031A5C41F6F830C2F201004FF0B2
:107D50004C0404FB02044FF00000FCF7EFFBE76368
:107D600026644FF00001616428464FF00101FFF7DF
:107D700083FF4FF00100FCF7E1FBF8BDF8B50546C5
:107D80000F46164641F65C63C2F201031A5C41F6E7
:107D9000F830C2F201004FF04C0404FB0204A16869
:107DA000B1420DD242F2F873C2F201039F4207D3EF
:107DB00042F6F872C2F20102974201D2F8F7FEFBD6
:107DC0004FF00000FCF7BAFBE7634FF000002064BF
:107DD000666428464FF00101FFF74EFF4FF00100A7
:107DE000FCF7ACFBF8BD00BF08B5FCF7FDFC08BD17
:107DF00070B586B005460C46164602A8F9F754FC45
:107E000001462EB102A82A46234600F09BFD07E05A
:107E10004FF00103009302A82A46234600F044FED7
:107E200006B070BD70B58AB00378212B00F0938046
:107E300004D86BB1012B40F0D88186E0A12B00F073
:107E4000A781C02B00F0B481802B40F0CE8195E05B
:107E50004178052903D0092940F0CA8146E04088CD
:107E600041F6EC32C2F201021378022B02D0032B4E
:107E700033D118E000F1FF318AB27E2A30D8C0B287
:107E800041F65863C2F2010318704FF00201FCF78B
:107E9000B7FD41F6EC30C2F201004FF00301017072
:107EA0004FF00100C3E170B941F65862C2F201021D
:107EB000107041F6EC30C2F201004FF00203037083
:107EC0004FF00100B3E17F280DD841F65861C2F2AE
:107ED000010108704FF00100A9E14FF00200A6E196
:107EE0004FF00200A3E14FF00200A0E1827841F6DA
:107EF000EC33C2F201031978022923D972B941F691
:107F0000EC33C2F201034FF0030119704FF001008E
:107F10000146FFF7D5F94FF0010088E1012A18BFAB
:107F2000022040F0848141F6EC30C2F201004FF0B3
:107F3000040202704FF000000146FFF7C1F94FF054
:107F4000010074E14FF0020071E140780B280CBF92
:107F5000012002206BE18388032B00F24C8141F663
:107F60007064C2F2010404EBC3035B68002B00F0F1
:107F700045819847002808BF022058E142781AB18D
:107F8000062A40F03E8121E0C18802291BD14FF032
:107F90000000ADF8040041F6E032C2F201021268BE
:107FA0000346517E61F30003ADF80430127E62F3A4
:107FB00041030AA921F8243D4FF00202FFF7DEFE3B
:107FC0004FF0030033E14FF0020030E18278C188C6
:107FD0008CB2C378022B2ED0032B3DD0012B40F066
:107FE000D48041F67C35C2F2010528464AF20811D8
:107FF000C0F603014FF012020EF0D0FF41F6E03060
:10800000C2F2010001688A892A81CB896B81088AC2
:10801000A8818A7C2A71CB7C6B71097DA9714FF094
:1080200000002946122C34BF22461222FFF7A6FE7A
:108030004FF00300FBE041F69062C2F201021181B1
:108040004FF00000506047F62D11C0F60201FFF717
:1080500071FE4FF00300EAE0D2B941F67C34C2F27F
:10806000010404F102004AF28401C0F603014FF05A
:1080700002020EF093FF4FF0040222704FF003054E
:1080800065704FF000002146FFF778FE2846CEE0ED
:10809000012A06D141F6E033C2F2010319680968EA
:1080A0002FE0022A06D141F6E032C2F20102106846
:1080B000416826E0032A06D141F6E033C2F201030B
:1080C000196889681DE002F00F0022F00F03102BE1
:1080D00008D15A4B196888420EDA594A52F83000D2
:1080E00001680EE0202B07D1032805D8554951F827
:1080F000300008B1016804E0EE2A04D04FF002001D
:1081000095E009B93EE05049B1F1FF3F40F0888069
:1081100001A84FF020014FF00102FFF769FE0AAD00
:108120002A184FF0000002F8240C01A978E000F1B1
:108130000206428003F10102134611F8015F5DB1AE
:1081400000F10400758002F1010311F8012F002AEB
:108150006FD101E04FF0000341F67C31C2F2010122
:108160004FF003054D7003F101034FEA4303DAB208
:108170000A704FF00000A24228BF2246FFF7FEFD22
:10818000284654E04FF0020051E04FF002004EE06C
:108190008388032B38D841F67064C2F2010404EBE3
:1081A000C3035B689BB39847002808BF02203EE0EA
:1081B0004378212B2ED1C18841F69063C2F201038E
:1081C00019814FF000025A608088042825D110469A
:1081D00047F20D51C0F6020141F69062C2F201026F
:1081E000FFF7A8FD4FF0030021E04FF002001EE072
:1081F0004FF002001BE04FF0020018E04FF00200C9
:1082000015E04FF0020012E04FF002000FE04FF0D7
:1082100002000CE04FF0020009E04FF0020006E01F
:108220000A78002A96D009484FF000037FE70AB089
:1082300070BD1E2B7FF47BAF8EE700BFF41B0120C7
:10824000C01B0120701E012020A103087C1B0120FF
:1082500010B50446436993B14FF00000606141F6E8
:10826000EC31C2F201010A78032A08D141F65863C1
:10827000C2F2010318784FF00301FCF7C1FB20693B
:1082800058B34FF000002061E06041F6ED31C2F2DA
:108290000101087041F6E431C2F201014FF0080219
:1082A000FFF7A2FD082853D141F6E432C2F20102E1
:1082B000137813F0800F06D141F6E430C2F20100CA
:1082C000C188002944D141F6E430C2F201004FF0E8
:1082D00000010A46FFF7A6FD2DE0E168002937D02E
:1082E0004FF00000E06041F6ED32C2F20102137877
:1082F00041F67C31C2F20101C3F14002FFF774FD87
:10830000034628B341F6ED30C2F2010001785A1855
:10831000D2B2027041F6E433C2F20103D88890422F
:1083200016D141F6E430C2F2010041F67C31C2F2CE
:108330000101FFF777FD012804D0022808D1FCF7DE
:10834000B5F910BD4FF0000001460246FFF716FDDB
:1083500010BD00BF08B541F69C63C2F201031B6962
:108360003BB14FF0000141F69C62C2F2010252693A
:10837000984741F69C60C2F201004FF00001017085
:1083800041608160C1600161416108BD41F69C604E
:10839000C2F2010081614AF23C11C0F603018A5C1D
:1083A00042778377037F6FF3070303774FF0000172
:1083B0004162704730B583B041F69C64C2F201045B
:1083C0002070089D6560099DA5600A9DE5600B9D74
:1083D00025610C9D65619DF8184000949DF81C4036
:1083E0000194FFF7D3FF03B030BD00BF41F69C639B
:1083F000C2F201035B6AB3F1FF3F09D141F69C6110
:10840000C2F201014FF000034B624FF001007047D0
:108410003F2B0BD841F69C62C2F20102106AC15494
:1084200003F1010353624FF0010070474FF0000069
:10843000704700BF704700BF70B541F69C64C2F240
:10844000010404F118004AF20021C0F603014FF0C4
:1084500007020EF0A3FD4FF000004AF2F811C0F63B
:108460000301FFF7B3F948F29566C0F602064FF034
:1084700000004AF28011C0F603013246FFF7C4F94A
:108480004AF29815C0F603054FF00100294632461E
:10849000FFF7BAF92869FFF7E3F984F8280041F6F5
:1084A000C860C2F201004FF0070148F2BD42C0F6B9
:1084B00002024FF00003FCF74BFC70BD38B541F6EB
:1084C000FC63C2F201034FF001021A7041F69C6492
:1084D000C2F2010494F828004FF000010A46FFF7A9
:1084E0004DFC606868B141F69C64C2F201044FF033
:1084F000FF3565626368207861699847616A002981
:10850000F7D041F69C60C2F201004FF000024262D7
:10851000836833B141F69C61C2F201010878496970
:10852000984738BD2DE9F047A2B0804643680BB9A3
:10853000806828B14FF00001C8F80810FFF7BEFFAF
:10854000D8F80C20002A3ED04FF00007C8F80C7075
:10855000D8F8000012A94FF04002FFF745FC07468B
:1085600041F69C63C2F20103D86860B35FB341F681
:108570009C64C2F201044FF0000507F1FF3606F0DB
:10858000010A20789DF848102A466369E668B047DA
:108590004FF001094F456CD115E0E668207812AA2A
:1085A00012F809102A466369B04709F10109E66823
:1085B000207812AB13F809102A466369B04709F115
:1085C00001094F45E9D1D8F8140000284ED04FF0EA
:1085D000000441F6FC61C2F201010C70C8F81440BD
:1085E00041F6D860C2F20100FEF752FD41F69C62EE
:1085F000C2F2010254625368002B30D041F69C65F0
:10860000C2F2010502AC2C622C46656A62682078D1
:1086100061699047606A8542F7D105B3D8F80000D8
:1086200002A92A46FFF7AAFB4FF000010091019131
:1086300041F6D860C2F201004FF04B014FF0FF024B
:1086400048F2BD43C0F60203FEF7C8FD0EE041F656
:108650009C62C2F2010210785169984706E041F627
:108660009C63C2F201039B68002BF0D122B0BDE8ED
:10867000F087BAF1000F90D0E668207812A911F8BF
:1086800009102A466369B04709F101094F4584D1B1
:1086900099E700BF10B544780378212B02D0A12BB5
:1086A00019D10CE0202C02D0222C08D119E0072A85
:1086B0001AD10F480EF072FC4FF0010010BD212CB2
:1086C0000CD14FF000000A494FF00702FFF756FBAC
:1086D0004FF0030010BD4FF0000010BD4FF0000040
:1086E00010BD4FF0010010BD4FF0020010BD00BFE3
:1086F000B41E012008B541F6FC63C2F201031878EC
:1087000070B941F69C61C2F201014A6A72B941F640
:108710009C63C2F2010393F82800FFF78FFA08BDAB
:1087200041F6C860C2F20100FCF732FB08BD00BF91
:108730004AF25010C0F60300704700BF70B40378CF
:1087400001298CBF4478002402298CBF857800253C
:10875000DCF8000048B34FEA93064AF21C20C0F64A
:108760000300365C16704FEA031343EA141303F058
:108770003F031B5C5370012907D94FEA840444EA84
:10878000951303F03F04205C01E04FF03D00907032
:10879000022907D905F03F054AF21C23C0F603035E
:1087A000E95C01E04FF03D01D17070BC704700BF43
:1087B00082B04FF015010CE00191019B03F1FF32F3
:1087C000019233B100BF019B03F1FF320192002BF4
:1087D000F8D100F1FF30B0F1FF3FEDD102B07047AA
:1087E00070B4C4B24FEA10204AF2B026C0F60306B5
:1087F0004AF2B035C0F6030511F8013B1AB94BB97E
:1088000044EA00200BE06340F45C4440E85C013A39
:10881000F2D1F5E76340F45C4440E85CECE770BCFF
:10882000704700BF10B444F6FB43C0F2861311F842
:10883000014B02B9ACB380EA04404FEA400010F0AB
:10884000807F18BF58404FEA400010F0807F18BF6B
:1088500058404FEA400010F0807F18BF58404FEA60
:10886000400010F0807F18BF58404FEA400010F0E1
:10887000807F18BF58404FEA400010F0807F18BF3B
:1088800058404FEA400010F0807F18BF58404FEA30
:10889000400010F0807F18BF5840002AC7D0013A2E
:1088A000C5D120F07F4010BC704700BF82B001905E
:1088B0009DF806304FF0000063F307009DF8052097
:1088C00062F30F209DF8042062F317409DF8072003
:1088D00012F0800F14BF63F07F0103F07F0161F39A
:1088E00007004FEA4201CAB262F31F6013F0800F23
:1088F00018BF42F0010262F31F6002B0704700BF70
:1089000084B0C0F307438DF80C30C0F307228DF814
:108910000D20C3B24FEA10604FEA500210F0010F71
:1089200014BF63F07F0103F07F018DF80E1013F088
:10893000800F18BF62F07F028DF80F20039804B0FB
:10894000704700BF2DE9F04F83B005460F4614462F
:108950001E46019201F1FF3313F1050F44D8032E97
:1089600043D9A6F10400C0F380080DF1040C284699
:10897000FFF7E4FE05F10305A7F1030104F1040488
:10898000A6F10406A7F1040717F1050F67D92CE03B
:108990000DF1040C284639462246FFF7CFFE05F1BB
:1089A000030B5D46A7F1030104F1040A5446A6F146
:1089B00004094E46A7F1040717F1050F15D80F4615
:1089C0000DF1040C58465246FFF7B8FE0BF10305B3
:1089D000A7F103010AF10404A9F10406A7F10408B0
:1089E00018F1050F59D900E0FFE799B396B30DF1DF
:1089F000040C28466A46FFF7A1FE022E11D0032E72
:108A000002D0012E26D11AE0019929B19DF800204B
:108A100022704FF0010301E04FF0000304F1010464
:108A200001E04FF00003019830B102A9CA1812F812
:108A3000080C207003F1010304F1010401E04FF080
:108A40000003019921B102AAD31813F8080C207071
:108A500004F101040199601A03B0BDE8F08F0F46DC
:108A6000032EC2D9B8F1000F92D00DF1040C2846A4
:108A70002246FFF763FE05F10305A7F1030104F1A8
:108A80000404A6F10406A7F1040717F1050FACD8FA
:108A90000F46032E3FF67CAFA7E7A7F10307032E8F
:108AA0003FF676AFA1E700BFF0B49DF81040ECB1FF
:108AB0004FEA41079F421CD2DD1B1DD056194FF0D3
:108AC00030046FEA0203F31803F0010302F8014BCC
:108AD000B24240F0928007E0134603F8014B547015
:108AE00003F10102B242F7D13B4607E04FF0000527
:108AF00004E04FF0000501E04FF0000500293CD0F4
:108B000003F1FF34002B3AD000F10103411828464D
:108B1000521B04F1FF3515F0020F10D032E0A4F122
:108B2000020603F101031F46012C29D03446B44646
:108B300013F8016C4FEA1616092E42D944E01E467E
:108B400013F8015C4FEA1515092D8CBF3735303508
:108B5000155414B900F1010012E013F8016C06F08D
:108B60000F05092D8CBF373530351618757000F19B
:108B7000020528468B42D2D102E0284600E0284672
:108B8000F0BC70471E4613F8015C4FEA1515092D1D
:108B900094BF303537351554002CDBD013F8016CF9
:108BA00006F00F05092D94BF30353735161875704E
:108BB00000F102008B42E3D003F10103A4F10204AF
:108BC000BDE706F1300601E006F137065655BCF167
:108BD000000FBFD013F8016C06F00F06092E94BFEA
:108BE000303637361018467005F102008F42C7D074
:108BF00003F10103A4F10204A1E7002B3FF46CAFE1
:108C000002F8014BB2427FF467AF6DE7DCF8143035
:108C100093F8452083F84420DCF8141091F846308E
:108C200081F84530DCF8141091F8472081F846208F
:108C3000DCF8143083F84700704700BFDCF81430CC
:108C400093F8470093F8462083F84720DCF8141087
:108C500091F8453081F84630DCF8141091F8442042
:108C600081F84520704700BF42F2C012C2F20102F3
:108C7000136840F20001C0F60101C85CC9184978C8
:108C800003F10203136041EA00207047DCF804306E
:108C9000DCF8082002EBD300CCF8080003F0070151
:108CA0004FF0010303FA01F2CCF80420704700BF33
:108CB0002DE9F04F83B004468A4693461E46CDF810
:108CC00004C04FF00007B846B9463DE0254630469F
:108CD000D047034600283DD0B9F1000F0CD1202821
:108CE00029D0092829D00A2829D00D2829D0022DD9
:108CF0004FF0010988BF0225A3F13002D1B2092942
:108D000010D9A3F14100C1B2052903D8A3F137035B
:108D1000D9B207E0A3F16102D0B205281AD8A3F1B5
:108D20005703D9B24FEA0717FCB241EA040708F12A
:108D300001082C4606E02C4604E02C4602E02C46B6
:108D400000E02C463046D847FF2CBFD004F1FF3559
:108D5000002CBCD1DDF804C03846FFF757FF019B5B
:108D60005A69D8F1010838BF4FF0000882F85080E6
:108D700003B0BDE8F08F00BF42F28803C2F20103E6
:108D80001B684B634BB19A68824209D0DB684B6326
:108D90001BB19A688242F9D102E04FF01E00704781
:108DA0004FF00000704700BF884204D8884234BFAB
:108DB0000220002070474FF001007047D0F80431C6
:108DC000D0F80021934214BFC05C0020704700BF60
:108DD000D0F80431FF2B14BF01330023C0F8043155
:108DE000704700BF10B4DCF81420D16C0B46044669
:108DF00058B14FEA016343EA116301F47F4043EA4B
:108E0000002301F47F0143EA1123DCF8040030B1B0
:108E100099B24FEA134060F30F0361F31F435CB94B
:108E20004FEA036141EA136103F47F4041EA002104
:108E300003F47F0341EA1323D36410BC704700BFDF
:108E4000DCF80030FA2B05D841F60872C2F20102B4
:108E5000D05C70474FF00000704700BFDCF8003076
:108E600003F10103CCF80030DCF8140090F8512035
:108E700002F1010280F85120704700BF70B404462F
:108E80000846A1B199188C4211D22518AA420ED2D7
:108E900094423ABFC4EB0206F6B20026A94205D2BC
:108EA0000019821AD31AF118C8B200E0304670BC1B
:108EB000704700BFF0B583B042F26403C2F2010311
:108EC0004FF008021A7042F25000C2F2010004682A
:108ED0003CB3154642F26407C2F201074FF00006A8
:108EE00021680B6873B10DF107000DF10601984779
:108EF0009DF807009DF8061032463B78FFF7BEFF4D
:108F00004519EDB26468002CEAD142F26402C2F263
:108F100001021078A84204D242F26401C2F20101B7
:108F20000D7042F26403C2F201034FF006025A7060
:108F300042F24804C2F2010424683CB3154642F2EE
:108F40006407C2F201074FF000062068036873B19E
:108F50000DF107000DF1060198479DF807009DF8F7
:108F6000061032467B78FFF789FF4519EDB2646839
:108F7000002CEAD142F26401C2F201014A78AA420D
:108F800004D242F26400C2F20100457042F264036E
:108F9000C2F201034FF00801997042F25C04C2F280
:108FA000010424683CB30D4642F26407C2F2010793
:108FB0004FF000062268136873B10DF107000DF140
:108FC000060198479DF807009DF806103246BB78C9
:108FD000FFF754FF4519EDB26468002CEAD142F264
:108FE0006400C2F201008178A94204D242F2640214
:108FF000C2F20102957042F26403C2F201034FF023
:109000000600D87042F2C414C2F2010424683CB3D2
:10901000054642F26407C2F201074FF000062168DC
:109020000A6872B10DF107000DF1060190479DF835
:1090300007009DF806103246FB78FFF71FFF451921
:10904000EDB26468002CEAD142F26403C2F201037B
:10905000D878A84204D242F26401C2F20101CD7074
:1090600003B0F0BD42F2B813C2F20103196840F236
:109070000000C0F60200401A704700BF034610B15E
:1090800082688A4218D042F26003C2F20103186873
:1090900060B182688A4203D10BE083688B420AD0B8
:1090A00040680028F9D14FF0000305E04FF00003BD
:1090B00002E0034600E003461846704710B540F250
:1090C000A064C1F200044FF4117303FB0044D4F810
:1090D0000811B1F1FF3F03D0D4F8042191420DD122
:1090E00023689A6A4FF0FF019047002834D0D4F8E3
:1090F000080100F10100C4F8080110BD91422BD80D
:109100006318197942F2BC12C2F2010213787BB9DA
:10911000FD290FD923689A6A4FF0FE019047D8B114
:1091200042F2BC10C2F201004FF00101017010BD0B
:109130006FEA01012268936AC9B2984760B1D4F816
:10914000080100F10100C4F8080142F2BC11C2F2AA
:1091500001014FF000020A7010BD00BF70B5064655
:1091600040F2A065C1F200054FF4117404FB00F455
:109170002B194FF00101C3F80C112A599369984734
:109180002859016A3046884770BD00BF38B540F2A3
:10919000A061C1F200014FF4117202FB00F28C18C1
:1091A000D4F80831D4F80451AB420DD08958E318F3
:1091B0008A6A1979904738B1D4F80801FF2814BF9A
:1091C00001300020C4F8080138BD00BF38B540F2B6
:1091D000A064C1F200044FF4117202FB00F2A31864
:1091E000D3F80451D3F808118D4206D14FF0000195
:1091F000C3F80C11A2589369984738BD10B440F2D7
:10920000A063C1F200034FF4117202FB003000F5BD
:109210008870D0F80031FF2B14BF5A1C0022D0F800
:109220000441A2421CBFC154C0F8002110BC7047C9
:10923000F8B542F2B814C2F2010424688568C76820
:10924000466807FB05604518611911D2CE180B4816
:10925000864210D8012B04D1635D13704FF00000DB
:10926000F8BD10461A460DF099FE4FF00000F8BD0B
:109270004FF01F00F8BD4FF01F00F8BD01000208BD
:1092800010B542F26803C2F201031A7840F2A060FE
:10929000C1F200004FF4117404FB0204F7F7E4F983
:1092A0004FF0FF31C4F810124FF00003C4F8183229
:1092B00004F58874F7F7E2F910BD00BFF8B506466B
:1092C0004FF00203037044F20000C0F60000C28BAE
:1092D0004FF6FF718A4221D03F4C404BA34222D22D
:1092E00003F110033E4DEF1A4FEA17124FF6FF75C8
:1092F00002F1010002F001071C46D98BA9424FD1AF
:1093000015E01C46D98BA94211D002F1010203F1EC
:1093100010031C46D98BA94257D108E044F200043F
:10932000C0F6000403E044F20004C0F600044FF667
:10933000FF7021464FF00D02FFF752FA4FF6FF7310
:10934000984208BF0020E28982421BD0A4F1100598
:1093500044F20000C0F6000085421AD34FF6FF70B9
:1093600029464FF00D02FFF73BFA4FF6FF71884296
:1093700008BF002034F8024C84420AD12C464FF03A
:10938000010201E04FF00002607BFF2806D132703D
:1093900004E04FF0020333704FF000042046F8BDA4
:1093A0004FF0000202F1010203F110038242BED02D
:1093B000002FA6D01C46D98BA942B8D002F10102D9
:1093C00003F1100382429CD1B1E702F1010203F1E3
:1093D0001003824295D1AAE70080000800400008EF
:1093E0000F80000870B5C0B005460E4620F0FF049F
:1093F000684621464FF04002F9F712F900AB53FAE4
:1094000085F031464FF010020DF0C8FD6846214648
:109410004FF48072F9F758FA40B070BD38B5054680
:1094200040F2A064C1F200044FF4117303FB004446
:10943000D4F81C02FDF73AFB42F26800C2F20100C8
:109440000178A94206D142F26803C2F201034FF04B
:10945000FF021A704FF00000C4F81C0238BD00BFB4
:1094600010B54FF00000FBF7B3FC42F25003C2F21C
:1094700001031C6834B12068016901B18847646840
:10948000002CF8D110BD00BF10B50446072827D81E
:10949000032894BF4FF4FA73322303FB01F140F227
:1094A000A063C1F2000303EBC000C0F8141969B156
:1094B000FDF7CAFE002808BF012040F2A063C1F2F8
:1094C000000303EBC404C4F8100910BD40F2A0610E
:1094D000C1F2000101EBC4044FF00002C4F81029EE
:1094E00010BD00BF38B50446072851D840F2A0632C
:1094F000C1F2000303EBC000D0F8145935B340F2B9
:10950000A061C1F2000101EBC402D2F81039EBB145
:10951000FDF79AFE002808BF012040F2A061C1F2C9
:10952000000101EBC402D2F81039C01A85420CD2F6
:1095300040F2A065C1F2000505EBC4014FF0000543
:10954000C1F81459C1F8105900E02D1A05F10405AD
:109550004CF6CD42CCF6CC42A2FB05234FEA930059
:10956000032C0AD800F1630348F21F51C5F2EB1136
:10957000A1FB03324FEA521038BD00F109014CF64D
:10958000CD42CCF6CC42A2FB01304FEAD00038BD30
:109590004FF0000038BD00BF70B506466446DCF8E9
:1095A00014305D6AFDF750FE6169CA6A0AB9C86283
:1095B00008E0801A05EB850506FB05F6B04224BFDE
:1095C0000020C8626369D96AD1F1010038BF002068
:1095D00070BD00BF10B540F2A063C1F200034FF4AC
:1095E000117404FB003303F58873D3F80841002C91
:1095F0005FD15AB14FF0FF31C3F8001142F20803B6
:10960000C2F201034FF00000187010BDD3F8002122
:10961000B2F1FF3F06D1FF294BD14FF00002C3F852
:10962000002110BDFF291ED142F20801C2F2010142
:109630004FF000040C70012A10D94FF00102C3F85A
:10964000082140F2A063C1F200034FF4117101FB45
:109650000030D0F81C02FCF7E7FF10BD4FF000000F
:10966000C3F8000110BDFE2907D142F20803C2F27F
:1096700001034FF00101197010BD42F20800C2F25F
:109680000100007848B16FEA0101C9B242F2080056
:10969000C2F201004FF000040470FF2A05D899546B
:1096A00002F10102C3F8002110BD4FF0FF32C3F8F0
:1096B000002110BD08B540F2A063C1F200034FF4D1
:1096C000117202FB0030D0F80811D0F8043100F11B
:1096D000040099420AD94FF00002C0F8002142F27A
:1096E0009400C2F201004068FCF79EFF08BD00BF75
:1096F000F8B5654642F28C03C2F201031C7804F00F
:109700000802D7B227B1DCF8146096F8516007E080
:1097100014F0110F06BFDCF8144094F852600026D4
:1097200001EB800411F820304FEA9312012A08D08F
:10973000022A10D111F82070C7F3C20303FB06F709
:109740000BE06A6992F8513011F82070C7F3C20239
:1097500002FB03F701E04FF0000711F8200000F0D2
:109760000701042950D8DFE811F0940140003B00C4
:109770002200050042F2C011C2F201010B6840F262
:109780000007C0F60107FA1892F802E0D0784FEA15
:10979000006040EA0E40527840EA0220FF5C03F18C
:1097A00004030B603843FFF7ABF868602CE042F22B
:1097B000C012C2F20102136840F20000C0F60100BC
:1097C000C11891F801C0C05C4FEA004040EA0C208B
:1097D0008978084303F1030313603F186F6013E0B7
:1097E000FFF742FAC2196A600EE042F2C013C2F2F9
:1097F0000103186840F20001C0F601010A5CBF18BD
:109800006F6000F10100186063784FEA931001283F
:1098100007D002280ED16178C1F3C20202FB06F71D
:109820000AE06F6997F851306078C0F3C20101FB1C
:1098300003F701E04FF00007627802F00703042B02
:1098400050D8DFE813F0260140003B00220005005D
:1098500042F2C011C2F201010B6840F20007C0F6EB
:109860000107FA1892F802E0D0784FEA006040EA67
:109870000E40527840EA0220FF5C03F104030B60C3
:109880003843FFF73DF8A8602CE042F2C012C2F264
:109890000102136840F20000C0F60100C11891F8FF
:1098A00001C0C05C4FEA004040EA0C2089780843C0
:1098B00003F1030313603F18AF6013E0FFF7D4F91F
:1098C000C219AA600EE042F2C013C2F20103186886
:1098D00040F20001C0F601010A5CBF18AF6000F160
:1098E00001001860A3784FEA9310012807D00228DE
:1098F0000ED1A178C1F3C20202FB06F70AE06F693C
:1099000097F85130A078C0F3C20101FB03F701E0E2
:109910004FF00007A27802F00703042B4ED8DFE8CF
:1099200003F0B83E3920030042F2C011C2F2010137
:109930000B6840F20007C0F60107FA1892F802E03F
:10994000D0784FEA006040EA0E40527840EA0220A8
:10995000FA5C03F104030B601043FEF7D1FFE860EB
:109960002CE042F2C012C2F20102136840F2000081
:10997000C0F60100C11891F801C0C05C4FEA004078
:1099800040EA0C208978084303F1030313603F1871
:10999000EF6013E0FFF768F9C219EA600EE042F2E7
:1099A000C013C2F20103186840F20001C0F60101C1
:1099B0000A5CBF18EF6000F101001860E3784FEA1D
:1099C0009310012802D002280FD108E06E6996F8A2
:1099D0005130E078C0F3C20101FB03F607E0E17803
:1099E000C1F3C20202FB06F601E04FF00006E27886
:1099F00002F00703042B4CD8DFE803F04B031318E5
:109A0000300042F2C013C2F20103186840F20001B4
:109A1000C0F601010A5CB6182E6100F10100186061
:109A2000F8BDFFF721F982192A61F8BD42F2C01290
:109A3000C2F20102136840F20000C0F60100C11832
:109A40004C78C05C4FEA004040EA04208978084323
:109A500003F10303136036182E61F8BD42F2C01102
:109A6000C2F201010B6840F20004C0F60104E218E2
:109A70009678D0784FEA006040EA0640527840EA93
:109A80000220E25C03F104030B601043FEF738FF91
:109A90002861F8BD08B503281ED8DFE800F00209E8
:109AA00010174BF20860C0F603000FF069F808BD0C
:109AB0004BF20C60C0F603000FF062F808BD4BF2E9
:109AC0002060C0F603000FF05BF808BD4BF2386071
:109AD000C0F603000FF054F808BD00BF2DE9F843AD
:109AE0000546884616461F4642F26803C2F2010345
:109AF00093F8009042F2F440C2F20100016842F291
:109B00004C02C2F201021368994201D0FFF7B8FB80
:109B1000072D6ED81F2E6CD840F2A064C1F200044D
:109B20004FF4117000FB094442F29400C2F20100AC
:109B30004FF00001FCF718FB217965F34711072D61
:109B400014BF00250125AA1962F304012171CBB2CB
:109B50002DB184F8058043444FF0020001E04FF03E
:109B6000010006F1FF3E5FFA8EFE46B302463F1A41
:109B70000EF0010C3D5C04F1040635545B1902F152
:109B800001020EF1FF31C9B2FF2934D114E0BD5CEE
:109B900004F10406B5545B1902F1010201F1FF3131
:109BA00001F0FF01BD5CB5545B1902F1010201F146
:109BB000FF31C9B2FF29EAD100F101007044221837
:109BC000137100F10100C4F804014FF0FF33C4F831
:109BD000083121680B6A42F26800C2F20100007885
:109BE0009847FCF7EFFC42F29400C2F20100FCF748
:109BF000C9FBBDE8F8834FFA8CF5002DC7D0BD5CDA
:109C000004F10406B5545B1902F1010201F1FF31C0
:109C1000C9B2FF29BBD1CFE738B5054642F20C04E3
:109C2000C2F201042046FCF7ADFBF7F735FE2846EB
:109C3000FCF790FE20464FF00001FCF795FA38BD86
:109C400010B586B00DF10700FFF738FB044618B1D8
:109C50009DF8073023B90FE044F20004C0F6000479
:109C6000E2894FF6FF7082422BD048F20001C0F625
:109C700000018C4209D32AE0304821464FF00D0202
:109C80000CF036FD002848D0EAE74FF6FF7248F2A4
:109C90000000C0F600006FEA0403C118C1F3001110
:109CA00004F11004E389934239D10AE004F110036E
:109CB0001C46D989914204D003F11004E3899342F0
:109CC00039D148F20002C0F60002944207D344F2B0
:109CD0000004C0F6000420462146F8F789FD02A8DA
:109CE00016494FF00D020DF059F94FF0FF008DF8B5
:109CF00015004FF6FF7002A94FF00D02FEF770FD40
:109D00004FF6FF71884212BFADF816000021ADF882
:109D10001610204602A9FFF765FB06B010BD84426D
:109D2000D5D20029C2D004F11004E1899142C8D0F3
:109D30008442BBD3CBE78442B8D3C8E70E1F0120CF
:109D40002DE9F04F85B0884691461D46E2464FF01A
:109D5000000426464FF0020B2DE007462846C04778
:109D6000034670B324B9202822D0092802D11FE06D
:109D7000012C05D12B2B0DD02D2B0DD05C4601E0F5
:109D8000022C01D12E2B09D0A3F13002D0B2092828
:109D900017D805E05C4603E05C4601E04FF00304A1
:109DA0000E2E05D804A98A1902F8103C06F1010606
:109DB0002846C8473846FF28CFD000F1FF37002893
:109DC000CCD1012C12D98EB104ACA6194FF00004ED
:109DD00006F8104C684621460CF0E4FCDAF8141042
:109DE000C864DAF8142082F8504005E0DAF814303C
:109DF0004FF0010083F8500005B0BDE8F08F00BFC0
:109E000010B586B040F20000C0F601003449F8F702
:109E1000EFFC00284BD1334B334A9A421DD240F21B
:109E20000001C0F601010B68B3F1FF3F42D102F11E
:109E300004032E4AD01A20F00302991812F0040FDE
:109E40003FD118468B420CD003F104021B68B3F1DA
:109E5000FF3F3ED04FF0000031E040F20000C0F67E
:109E6000010040F20003C0F60203984225D10DF133
:109E70000700FFF723FA0446B0B19DF80710022946
:109E800012D002A821464FF010020DF087F89DF87D
:109E900015006FF307008DF81500204602A9FFF7A3
:109EA000A1FA4FF001000AE04FF0010007E04FF087
:109EB000000004E04FF0000001E04FF0000006B0A9
:109EC00010BD184603F104030268B2F1FF3FB8D099
:109ED000C0E702F104031068B0F1FF3FB1D0B9E769
:109EE000FFFF01080000020800000108030002084B
:109EF0002DE9F007034600284AD040F20022C0F6C0
:109F0000000292F8469092F8478042F26400C2F252
:109F1000010090F801C092F848A0057842F27C0256
:109F2000C2F201021468177A567A50684FF00002A4
:109F30001A7083F8019083F80280DA704FF0FB0802
:109F400083F804804FF0060883F805809D7183F83C
:109F500007C04FF0040C83F808C083F809C083F8E9
:109F60000AA0DD721A734FEA14255D739C73DF73C8
:109F70001E745A744FF01D029A744FF00202DA7484
:109F80004FF0FE021A755A754FEA10229A75D8756D
:109F900029B142F26403C2F2010318680860BDE807
:109FA000F0077047034628B142F27C02C2F2010278
:109FB0001068186042F27C01C2F20101087A704711
:109FC00070B505460E4614464FF000002946FFF7CF
:109FD00055F808B1F6F7F2FA42F26003C2F2010353
:109FE0001A686260A56026601C6070BD08B539B152
:109FF00042F25003C2F201031A68426018601EE088
:10A0000042F25003C2F201031B6883420FD1586829
:10A0100042F25001C2F20101086010E042685A6049
:10A0200041605A688242F9D013461BB907E033B148
:10A030004FF000015A688242F0D01346F5E7FEF770
:10A0400039FF08BD08B539B142F24803C2F2010335
:10A050001A68426018601EE042F24803C2F201032F
:10A060001B6883420FD1586842F24801C2F20101D5
:10A07000086010E042685A6041605A688242F9D034
:10A0800013461BB907E033B14FF000015A68824212
:10A09000F0D01346F5E7FEF70DFF08BD08B539B15E
:10A0A00042F25C03C2F201031A68426018601EE0CB
:10A0B00042F25C03C2F201031B6883420FD158686D
:10A0C00042F25C01C2F20101086010E042685A608D
:10A0D00041605A688242F9D013461BB907E033B198
:10A0E0004FF000015A688242F0D01346F5E7FEF7C0
:10A0F000E1FE08BD08B539B142F2C413C2F2010352
:10A100001A68426018601EE042F2C413C2F20103F2
:10A110001B6883420FD1586842F2C411C2F2010198
:10A12000086010E042685A6041605A688242F9D083
:10A1300013461BB907E033B14FF000015A68824261
:10A14000F0D01346F5E7FEF7B5FE08BD01604360A9
:10A15000826042F28803C2F201031A68C26018608A
:10A16000704700BF70B582B006464FF000038DF80F
:10A1700007300D4601B10B7042F25000C2F20100EF
:10A18000046874B121684B6843B130460DF1070192
:10A190002A46984710B19DF8070011E06468002C2A
:10A1A000F0D1072E03D83046FAF756FE08E02DB15D
:10A1B0004FF005022A704FF0000001E04FF0000060
:10A1C00002B070BD70B582B006464FF000038DF846
:10A1D00007300D4601B10B7042F25000C2F201008F
:10A1E000046874B121688B6843B130460DF10701F2
:10A1F0002A46984710B19DF8070019E06468002CC2
:10A20000F0D1072E0BD83046FAF73CFE8DF8070048
:10A2100010B13046FAF77CFE9DF8070008E02DB13A
:10A220004FF005022A704FF0000001E04FF00000EF
:10A2300002B070BD70B582B006464FF000038DF8D5
:10A2400007300D4601B10B7042F25000C2F201001E
:10A25000046874B12168CB6843B130460DF1070141
:10A260002A46984710B19DF8070011E06468002C59
:10A27000F0D1072E03D83046FAF7D4FD08E02DB10F
:10A280004FF005022A704FF0000001E04FF000008F
:10A2900002B070BD70B582B006464FF000038DF875
:10A2A00007300D4601B10B7042F24800C2F20100C6
:10A2B00004685CB121688B682BB130460DF1070151
:10A2C0002A46984758B96468002CF3D1052E0CDC57
:10A2D000062E0AD83046F6F73BFF8DF807009DF8AA
:10A2E0000700003018BF012008E02DB14FF0060232
:10A2F0002A704FF0000001E04FF0000002B070BD86
:10A30000F0B583B005460E464FF000038DF80730D8
:10A3100042F24800C2F201000468E4B14FF00007C5
:10A320002168CA681AB1284631469047F0B92368B7
:10A330009B6833B128460DF106010DF107029847DD
:10A3400000E038469DF8071099B9646814B10028F8
:10A35000E6D004E018B9052D0DDC062D0ED82846F0
:10A36000314606F02BFB4FF0000009E04FF00000F3
:10A3700006E0084604E04FF0060001E04FF006005A
:10A3800003B0F0BD70B582B005460E464FF0000335
:10A390008DF8073012B11946FFF7B2FF42F24800BC
:10A3A000C2F2010004686CB121684B68284631464E
:10A3B0000DF10702984710B19DF8070012E064689C
:10A3C000002CF1D1052D08DC062D09D82846314690
:10A3D000F6F7E0FE4FF0000004E04FF0060001E069
:10A3E0004FF0060002B070BD08B54FF00000014606
:10A3F0004FF00102FFF7C6FF08BD00BF70B582B085
:10A4000005460E464FF000038DF8073042F25C001F
:10A41000C2F2010004689CB121684B682846694675
:10A420000DF10702984728B10EB1009830609DF8F1
:10A43000070014E064681CB19DF80720002AEBD0E7
:10A44000072D07D84EB12846F7F75AFC30604FF079
:10A45000000004E04FF00F0001E04FF0000002B0F8
:10A4600070BD00BF70B582B005460E464FF00003C8
:10A470008DF8073042F2C410C2F20100046884B1C2
:10A4800021684B68284631460DF10702984710B104
:10A490009DF8070010E064681CB19DF80720002AB1
:10A4A000EED0052D06D828463146F7F7FBFA4FF0D7
:10A4B000000001E04FF00E0002B070BD70B582B038
:10A4C00005460E464FF000038DF8073042F2C410E7
:10A4D000C2F201000468A4B121688B685BB1284610
:10A4E00069460DF10702984728B10EB10098306017
:10A4F0009DF8070014E064681CB19DF80720002A4D
:10A50000EAD0052D07D84EB12846F7F71DFC30607C
:10A510004FF0000004E04FF0060001E04FF00000B3
:10A5200002B070BD000000002DE9F04F2DED048B4E
:10A530008BB007461546914259D289464FF0000B21
:10A540004FF000089FED908B9FED919B6FEA010605
:10A55000B01800F00106CDF804B0022F4CD150E045
:10A56000CDF804B0022F05D15FFA89F001A9FFF7F9
:10A57000A5FF04E05FFA89F001A9FFF73FFF04EBB4
:10A5800044060AA88119A1F1200601F8209C01F8CF
:10A590001F8C01980BF066FB53EC182B0BF000FDA1
:10A5A00053EC192B0BF0B8FB0BF022FB83B2FF2B03
:10A5B00028BFFF23B37004F101040A2C04D005F175
:10A5C000FF324A450AD14CB104EB44044FF0070076
:10A5D0003946E2B202ABFFF781FA444609F10109BC
:10A5E0004E46CDF804B0022F40F089808DE00BB0CC
:10A5F000BDEC048BBDE8F08FC8B201A9FFF7FEFEE9
:10A6000003E0C8B201A9FFF759FF0AAC04F8209D86
:10A6100084F8018001980BF025FB53EC182B0BF00C
:10A62000BFFC53EC192B0BF077FB0BF0E1FA81B276
:10A63000FF2934BF0B46FF23A3704FF0000404F141
:10A64000010405F1FF324A450DD10AE004EB440450
:10A650004FF007003946E2B202ABFFF73FFA44463B
:10A6600001E0002CF2D109F101094D45BFD9002EBE
:10A670003FF476AFCDF804B0022F05D05FFA89F031
:10A6800001A9FFF7BBFE04E05FFA89F001A9FFF71B
:10A6900015FF04EB44060AA8861906F8209D86F8E3
:10A6A000018001980BF0DEFA53EC182B0BF078FCCC
:10A6B00053EC192B0BF030FB0BF09AFA81B2FF2907
:10A6C00034BF0B46FF23B37004F101040A2C0AD1F6
:10A6D00004EB44044FF007003946E2B202ABFFF747
:10A6E000FDF9444605E005F1FF324A4501D1002C51
:10A6F000EED109F101094D453FF632AF77E75FFA38
:10A7000089F001A9FFF77AFE04E05FFA89F001A958
:10A71000FFF7D4FE04EB44000AA90B18A3F1200AAA
:10A7200003F8206C03F81F8C01980BF09BFA53EC94
:10A73000182B0BF035FC53EC192B0BF0EDFA0BF04A
:10A7400057FA82B2FF2A28BFFF228AF8022004F1BA
:10A7500001040A2C0AD104EB44044FF007003946E7
:10A76000E2B202ABFFF7BAF9444605E005F1FF306B
:10A77000B04201D1002CEED109F101094D453FF65F
:10A78000EFAE34E7AFF300800000000000E06F4060
:10A79000000000000000E03F2DE9F04F95B040F6CA
:10A7A000C410FCF7D7F84FF002004FF0000142F25E
:10A7B0006403C2F20103DA78FFF7B6FE4FF0000B34
:10A7C000DA46D9464FF001074CF6CD44CCF6CC44DE
:10A7D00001944FF07D00FCF7BDF88DF82F90C8462E
:10A7E0004E464C4613E045F0800504F10804E4B2FF
:10A7F0000CABF05CA84202D00CA97554B84606F127
:10A8000001069DF82F50002D50D1202E4ED020460D
:10A810000DF12F01FFF7A6FC051C18BF012504F15F
:10A820000100C0B20DF12F01FFF79CFC10B145F003
:10A830000205EDB204F10201C8B20DF12F01FFF7DC
:10A8400091FC08B145F0040504F10302D0B20DF10A
:10A850002F01FFF787FC08B145F0080504F1040358
:10A86000D8B20DF12F01FFF77DFC08B145F01005BE
:10A8700004F10500C0B20DF12F01FFF773FC08B120
:10A8800045F0200504F10601C8B20DF12F01FFF7D4
:10A8900069FC08B145F0400504F10702D0B20DF1A2
:10A8A0002F01FFF75FFC00289DD19EE7B8F1000F54
:10A8B00002D1BAF1000F0AD14FF002004946F2B2BC
:10A8C0000CABFFF70BF94FF03200FCF743F842F204
:10A8D0006402C2F2010292788AB1019EA6FB0A4389
:10A8E0004FEA131404EB8400BAEB800F07D138460B
:10A8F0004946FFF719FE4FF03200FCF72BF8BBF189
:10A90000000F40F09B8003A849464FF020020CF056
:10A9100069FB42F26401C2F201018D78ADB34E468B
:10A920006FEA0902531903F0010009F0070407FA5E
:10A9300004F29DF80C1042EA01038DF80C3006F188
:10A940000106AE42C0F299801FE014AA02EBD603C2
:10A9500006F0070407FA04F013F8441C40EA010269
:10A9600003F8442C06F1010614AC04EBD60006F003
:10A97000070107FA01F210F8443C42EA030400F828
:10A98000444C06F10106AE42DFDB4FF007004FF00A
:10A9900011014FF01E0203ABFFF7A0F84FF0320099
:10A9A000FBF7D8FF03A849464FF020020CF01AFB32
:10A9B00042F26405C2F20105EE78A6B348466FEA9A
:10A9C00009018A1902F0010309F0070407FA04F5E6
:10A9D0009DF80C1045EA01028DF80C2000F10100F1
:10A9E000864236DC1FE014AD05EBD00200F0070410
:10A9F00007FA04F312F8441C43EA010502F8445C28
:10AA000000F1010014AA02EBD00500F0070407FAD8
:10AA100004F315F8441C43EA010205F8442C00F144
:10AA200001008642DFDC4FF007004FF012014FF0CB
:10AA30001E0203ABFFF752F84FF0060BBAF1000FFE
:10AA400004D10BF1FF3B4FF0280AC2E60AF1FF3AAE
:10AA5000BFE6002BC7D014AB03EBD00500F0070412
:10AA600007FA04F215F8441C42EA010305F8443CD5
:10AA700000F101008642B6DCD5E700283FF465AF5F
:10AA800014A800EBD60206F0070407FA04F312F844
:10AA9000441C43EA010002F8440C06F10106AE42F0
:10AAA000FFF653AF71E700BF2DE9F04F2DED028B9C
:10AAB00087B008EE100A0C4617469946129E139965
:10AAC000B5EEC08AF1EE10FA54BF00250125A84664
:10AAD00004F1FF33D8B2082807D8092A05D8A246BE
:10AAE00001F1FF32944205D808E001F1FF339C42A6
:10AAF00040F2CD8001F1FF34E4B2C8E018EE100A54
:10AB00000BF084FC48B930464FF03F0122460CF070
:10AB100069FA4FF000013155C4E018EE100A0BF04D
:10AB2000E1FC06EE900AF2EE047AF4EEE76AF1EE4A
:10AB300010FA0DDB4FF00100B0EE677A00F1010072
:10AB400067EE877AF4EEE76AF1EE10FAF6DA03E0E0
:10AB50004FF00100F2EE047A21464319A34200F3BC
:10AB60009680C0EB040EC5EB0E0202F1FF3E4AF6E2
:10AB7000005AC0F6030ADFED9C4AF6EE003AB2EE48
:10AB8000044AC0EB040CC5EB0C0303F0010BBEF14F
:10AB9000000F00F38F808AE0BEF1000F04DDBE4598
:10ABA000B4BF72463A4601E04FF000025AF8223034
:10ABB00003EE103AB8EE430A20EE027AB4EEE47ADD
:10ABC000F1EE10FA48BF37EE237ABDEEC73A13EE26
:10ABD00010CABCFBF3FB06EE10BAB8EEC65AB4EED0
:10ABE000E75AF1EE10FA0DDB00F1010C87EE006A76
:10ABF00067EE847A0EF1FF3E6046BEF1000200F37C
:10AC0000C380BEE013EE105AB5FBF3F403FB1454FB
:10AC10002CB916EE107A002F08BF4FF00008B9F1DA
:10AC2000000F07D0C8EB0103181A002A18BF01381B
:10AC3000831A01E04FF0000301F10101B8F1000FA8
:10AC400004D04BF25C67C0F6030703E048F6A04768
:10AC5000C0F6030722B14BF26060C0F6030003E0C8
:10AC600048F6A040C0F603004BF27465C0F6030539
:10AC7000009501978DED026A039004920594304689
:10AC80004BF26462C0F603020BF076FD0AE0304638
:10AC9000002D0CBF2B212D2122460CF0A3F94FF0E3
:10ACA0000000305507B0BDEC028BBDE8F08F4FF0CF
:10ACB000000203E0BE45B4BF72463A465AF822305D
:10ACC00000EE103AB8EE405A65EE260AF4EEE40AB9
:10ACD000F1EE10FA48BF70EEA30ABDEEE03A13EEB3
:10ACE00010CABCFBF3FC06EE10CAF8EEC65AF4EE2E
:10ACF000E75AF1EE10FA85DB00F1010080EE852ABB
:10AD000067EE847A0EF1FF3E42199142BFDBBBF140
:10AD1000000F3FF441AFBEF1000F02DC4FF0000224
:10AD200003E0BE45B4BF72463A465AF8223001EEFF
:10AD3000103AF8EE411A21EE822AB4EEE42AF1EE3E
:10AD400010FA48BF32EE232ABDEEC23A13EE10BA13
:10AD5000BBFBF3FB06EE10BAF8EEC62AF4EEE72AC8
:10AD6000F1EE10FAFFF64EAF00F1010082EE212A5B
:10AD700067EE847A0EF1FF3E43199942BFF60CAF9D
:10AD800085E74FF0000202E0BA42A8BF3A465AF8FF
:10AD9000223006EE903AF8EE660A20EE861AB4EEFD
:10ADA000E41AF1EE10FA48BF31EE231ABDEEC13AB3
:10ADB00013EE10BABBFBF3FB06EE10BAF8EEC65A60
:10ADC000F4EEE75AF1EE10FAFFF61CAF0CF10100B9
:10ADD00081EE202A67EE847A0EF1FF3E42199142FD
:10ADE000BFF6DAAE53E700BF0000004BF8B50546EA
:10ADF0000F46F5F739FC064640F2A062C1F20002A8
:10AE00004FF4117303FB05F01418115811B18A683F
:10AE10002846904784F820724FF00005C4F810527D
:10AE2000C4F81452C4F80451C4F808513046F5F778
:10AE300025FC04F5097029464FF00802F5F7CEFB12
:10AE4000F8BD00BF70B588B0054640F2A064C1F2FD
:10AE500000044FF4117303FB004494F8200200280F
:10AE600047D042F26801C2F201010878FF2803D0FE
:10AE70004FF00401FFF7BAFF28464FF00001FFF73B
:10AE8000B5FF42F26806C2F2010635704BF28060EF
:10AE9000C0F603004FF0070140F28102C0F6030242
:10AEA000FBF71AFDC4F81C02246830784FF0010249
:10AEB00000924FF00002019249F2BD03C0F6020376
:10AEC000029349F2B561C0F60201039149F2D553EC
:10AED000C0F60203049349F21D41C0F60201059138
:10AEE000069264684FF416514FF00803A047FEF72E
:10AEF000C7F908B070BD00BF704700BF10B50C4661
:10AF0000B0F1FF3F28D14FF000000246F6F74AFFAC
:10AF10004FF0010021464FF00002F6F743FF4FF0DB
:10AF2000020021464FF00002F6F73CFF4FF003000D
:10AF300021464FF00002F6F735FF4FF0040021469E
:10AF40004FF00002F6F72EFF4FF0050021464FF0BC
:10AF50000002F6F727FF10BD002806DB052804DCF9
:10AF6000C0B24FF00002F6F71DFF10BD38B505F076
:10AF700019FD42F26903C2F201034FF001021A7097
:10AF80004FF000042546E0B229462A46FFF7FAF9B9
:10AF900048B904F10104E0B229462A46FFF7F2F964
:10AFA000002800F08B804FF0FF304FF00001FFF7DA
:10AFB000A5FF4FF000004FF00001FFF753FA08BB68
:10AFC0004FF001004FF00001FFF74CFAD0B94FF0FD
:10AFD00002004FF00001FFF745FA98B94FF0030067
:10AFE0004FF00001FFF73EFA60B94FF004004FF058
:10AFF0000001FFF737FA28B94FF005004FF00001C4
:10B00000FFF730FA42F2C411C2F201010C6834B108
:10B010002368DA6802B190476468002CF8D142F2E4
:10B020006000C2F2010004683CB121680B680BB1FA
:10B03000A06898476468002CF7D1FAF75FFBFEF729
:10B040000FFA40F2A062C1F2000292F82002042836
:10B0500006D028B14FF000004FF00401FFF7C6FE04
:10B0600040F2A061C1F2000191F86434042B06D0D3
:10B070002BB14FF001004FF00401FFF7B7FE40F293
:10B08000A062C1F2000292F8A806042806D028B1F6
:10B090004FF002004FF00401FFF7A8FE40F2A0615C
:10B0A000C1F2000191F8EC38042B06D02BB14FF01F
:10B0B00003004FF00401FFF799FE38BD04F10104CD
:10B0C000B4F5807F7FF45FAF6DE700BF38B505460C
:10B0D00042F24C04C2F201042068FBF7E7FC4FF097
:10B0E000000323608DB14BF29060C0F603004FF077
:10B0F00007014BF20122C0F60202FBF7EDFB42F220
:10B100005402C2F20102106038BD42F25404C2F28D
:10B1100001042068FBF7CAFC4FF000002060FAF73A
:10B12000A1FEFFF723FF09F037FF42F26801C2F2E8
:10B1300001010878FF2803D04FF00401FFF756FE05
:10B1400038BD00BF70B542F29400C2F201004BF26C
:10B15000A061C0F60301FAF7EFFF42F26803C2F202
:10B1600001034FF0FF021A7040F2A064C1F2000424
:10B170004FF0040684F820624FF00005C4F81C521A
:10B180002846FBF7C3F9206084F86464C4F860546F
:10B190004FF00100FBF7BAF9C4F8440284F8A8663E
:10B1A000C4F8A4564FF00200FBF7B0F9C4F88804C5
:10B1B00084F8EC68C4F8E8584FF00300FBF7A6F9F0
:10B1C000C4F8CC0642F20C00C2F201004BF2AC61B2
:10B1D000C0F60301FAF7B0FF42F26C00C2F20100C0
:10B1E0004BF2B831C0F603012A462B46FEF7AEFFFC
:10B1F000FDF760FE4FF00100FFF768FF70BD00BF74
:10B200002DE9F04F2DED0A8BABB01CAF26AC4AF206
:10B21000B045C0F6030595E80F0084E80F00A7606D
:10B2200048F64163C0F60203E36020462AA9F8F716
:10B230003BF922AE95E80F0086E80F00B76048F6AC
:10B240005D60C0F60200F06030462146F8F72CF948
:10B250004FF000041B9442F20C00C2F201002146A0
:10B26000FAF782FF42F27C01C2F201010C72FFF791
:10B270007DFE09F091FE4FF00200FFF7E3FD42F280
:10B28000C012C2F2010215680DBB0DF069FCF0B9E5
:10B29000F6F704FA10F0C20F19D14FF00300FEF7D1
:10B2A000F9FB4FF47A754FF032063046FBF752FB4C
:10B2B000F6F7F2FA05F1FF343046FBF74BFBF6F7F1
:10B2C000EBFA651EF1D14FF00000FEF7E3FB42F20E
:10B2D0008C03C2F201034FF000041C604FF0010028
:10B2E000187040F2A066C1F2000606F51565284602
:10B2F000214642F654220BF075FE41F60870C2F268
:10B30000010021464FF480720BF06CFE06F51160CF
:10B3100021464FF040020BF065FE42F2BC00C2F243
:10B32000010021464FF0FC020BF05CFE21954FF02E
:10B330000A01C6F8741920462946FDF71DFD42F2A0
:10B340004402C2F20102146042F25803C2F2010345
:10B350001C6042F2C015C2F201054FF030042C60AF
:10B3600040F20004C0F6010494F82F0000F101003F
:10B3700094F82E1000EB0122101942F2B813C2F219
:10B3800001031860FBF760FF0B902B68E15CFF295D
:10B3900030D142F27C00C2F201004FF00101017293
:10B3A0000360219A106A18B100F1010052F82030B0
:10B3B00042F27C01C2F201014B604FF0FF024A727F
:10B3C00042F25400C2F201004FF00003036042F267
:10B3D0006801C2F20101087840F2A062C1F20002E5
:10B3E0004FF4117303FB0021D1F81C02FBF71CF989
:10B3F00004F00EBE05F0B4FA4FF000070A97BA4603
:10B400003C46DFEDC38A9FEDC39ADFEDC3AA9FEDF3
:10B41000C38ADFEDC39A9FEDC3AA01E04FF0000499
:10B420002CB94FF00000FEF7F7FB4FF0640404F175
:10B43000FF3442F28C06C2F20106357805F0F702BD
:10B440006FF30412327042F2C010C2F201000368BE
:10B45000099342F2C016C2F2010640F20007C0F69C
:10B46000010742F28C08C2F201084AF2D459C0F630
:10B47000030931687D5C01F10101316098F8002019
:10B4800012F0010F0ED10AF1010A40F2FF3082459D
:10B4900008D942F27C03C2F201034FF0360119725F
:10B4A00004F06EBD0DF1700C28464946FEF720F9F8
:10B4B0004AF6B873C0F6030353F825204BF2007B1D
:10B4C000C0F6030B42F0010108473268B85C0C90EB
:10B4D00002F1010232600F2804F24A850DF1700C6E
:10B4E0005946FEF705F94AF62863C0F603030C999E
:10B4F00053F82120E6E73268B85C0C9002F10102B3
:10B500003260102802D9054604F033BD0DF1700CED
:10B510000C984AF6D411C0F60301FEF7E9F84BF295
:10B52000C453C0F603030C9953F82120CAE73268CC
:10B53000B85C0C9002F1010232600F2802D9054676
:10B5400004F017BD0DF1700C0C984AF6D821C0F626
:10B550000301FEF7CDF84AF66863C0F603030C99C1
:10B5600053F82120AEE73268B85C0C9002F101027A
:10B5700032602F2802D9054604F0FBBC0DF1700C97
:10B580000C984AF61831C0F60301FEF7B1F84AF6F6
:10B590001823C0F603030C9953F8212092E7326870
:10B5A000B85C0C9002F1010232603B2802D90546DA
:10B5B00004F0DFBC0DF1700C0C984AF6D831C0F6DF
:10B5C0000301FEF795F84BF2D443C0F603030C9940
:10B5D00053F8212076E73268B85C0C9002F1010242
:10B5E00032603F2802D9054604F0C3BC0DF1700C4F
:10B5F0000C984AF62851C0F60301FEF779F84AF292
:10B60000C043C0F603030C9953F821205AE732686F
:10B61000B85C0C9002F101023260432802D9054661
:10B6200004F0A7BC0DF1700C0C984AF6A861C0F6A6
:10B630000301FEF75DF84BF2C433C0F603030C9927
:10B6400053F821203EE7219F97F846600DF1700CDA
:10B65000FDF7F4FA219D301895F8503003F0010100
:10B6600042181C9285F84720FF2A94BF002201222D
:10B6700085F85020D4E6219F97F846600DF1700CB4
:10B68000FDF7DCFA35181C95219880F84750FF2DFE
:10B6900094BF0025012580F85050C1E60DF1700CD3
:10B6A000FDF7CCFA30B1219991F84720131C18BF4F
:10B6B000012301E04FF00003219F87F84730AFE6F8
:10B6C0000DF1700CFDF7BAFA219E96F8475028400C
:10B6D00086F84700A4E61D98A0F1FB001C9013E13A
:10B6E0001D9BA3F1FB031C939BE11D99A1F1FB01A1
:10B6F0001C91CCE11D9AA2F1FB021C9268E21D9EF6
:10B70000A6F1FB061C964FF002001B9000E200BF62
:10B7100000000034FFFF7F4BFFFF7FCB00000000E5
:10B72000FEFFFFCAFEFFFF4A1D9BA3F1FB031C9314
:10B730001E991B911DE21D9AA2F1FB021C9217E1BA
:10B740001D9EA6F1FB061C9699E21D98A0F1FB0038
:10B750001C90D5E21D9FA7F1FB071C971E9B1B9316
:10B7600012E31D99A1F1FB011C911E9A1B924FF04F
:10B7700000068DF86A60C0E31D98A0F1FB001C90E4
:10B780001E9B1B934FF001018DF86A10B5E31D9AC3
:10B79000A2F1FB021C9200F04DBC1D9DA5F1FB0522
:10B7A0001C9500F0A2BC9DF874004FF00101FEF75B
:10B7B000A7FD8DF86B0000283FF432AE42F27C0406
:10B7C000C2F20104207204F0DBBB1D9E1C964FF0F8
:10B7D00001038DF86A301E46219890F847100B42FD
:10B7E00005D09DF870003146FEF78AFD68B99DF8D6
:10B7F0006A304FEA43008DF86A001C9A02F1010298
:10B800001C9210F0FE03E7D10CE09DF86A60012E57
:10B8100008D19DF86B4042F27C01C2F201010C722A
:10B8200004F0AEBB0DF1700CFDF708FAF8E59DF8D9
:10B83000740005F087F8F3E50DF1700CFDF7FEF9E3
:10B840001C9042F2C016C2F2010630681C9900EB4F
:10B8500041023260FDF708FA1C9001F0DDBC1D9832
:10B86000FA2808D942F27C06C2F201064FF013040E
:10B87000347204F085BB41F60872C2F20102135C17
:10B880001C93DEE7219991F852001C90D9E7219A88
:10B8900092F850301C93D4E74FF0000AC0E50DF148
:10B8A000700CFDF7CBF91C90219F97F847101B9166
:10B8B000FDF77AFA87F84700B2E5219D95F8470031
:10B8C00095F84610FDF770FA85F85000A8E50DF1DF
:10B8D000700CFDF7DBF91E9B41F60876C2F20106FB
:10B8E000F05C1D9920EA0102F25499E542F2BC0095
:10B8F000C2F201004FF000014FF0FB020BF072FBAF
:10B900008EE54FF000031C930DF1A80C1CF8386D68
:10B91000FDF794F90146304607F07AFE8DF86B008A
:10B9200000283FF47DAD42F27C04C2F20104207293
:10B9300004F026BB06F0FEF972E506F003FA8DF876
:10B940006B0000283FF46CAD42F27C01C2F20101B1
:10B95000087204F015BB42F2B817C2F201073D6845
:10B960001D98281806F0DAF95AE54FF000021C92EB
:10B970001C9B40F2A066C1F200064FF4117101FB5E
:10B98000036090F82022032A3FD140F2A067C1F261
:10B99000000701FB03F303F58876B919FB1803F1DF
:10B9A00004034FF00000D1F80021FE2A94BF551C7B
:10B9B0000025D1F80471BD4214BF0025012565F3AF
:10B9C0000000BA4214BF0022012262F34100D3F802
:10B9D0000051FE2D94BF013500250DF1A80C4CF847
:10B9E000385DD3F80461B54214BF0025012565F325
:10B9F0008200D3F80811D1F1010338BF002363F3AB
:10BA0000C300C0B2FDF702F90AE542F27C04C2F2BB
:10BA100001044FF04803237204F0B2BA4FF0000063
:10BA20001C901C9E40F2A062C1F200024FF4117102
:10BA300001FB062393F8200203281CD140F2A067E3
:10BA4000C1F2000701FB0675D5F81022D5F81412D3
:10BA5000531AB3F5807F88BF03F580731C931C983D
:10BA6000FF2884BFFF201C900DF1A80C1CF8380D96
:10BA7000FDF7CCF8D4E442F27C04C2F201044FF0AA
:10BA80004806267204F07CBA4FF000061C961C9BF8
:10BA900040F2A062C1F200024FF4117101FB0320D9
:10BAA00090F82062032E24D140F2A067C1F2000773
:10BAB00001FB037505F58876D6F80021D6F8041148
:10BAC000501AB0F5807F88BF00F580701C900DF192
:10BAD000700CFDF7B3F88DF86A001C9B984238BFD4
:10BAE0001C90D6F804711C9DEA19D1B2C6F8041155
:10BAF00096E442F27C04C2F201044FF04803237240
:10BB000004F03EBA4FF000061C964FF002001B9066
:10BB10001C9B40F2A062C1F200024FF4117101FBC4
:10BB2000032696F82002032815D140F2A067C1F23F
:10BB3000000701FB03750DF1700C1B9848F6BD5111
:10BB4000C0F6020148F6D152C0F6020205F588732C
:10BB5000FDF7AEF864E442F27C04C2F201044FF057
:10BB60004803237204F00CBA4FF000021C921D9996
:10BB70001B911C9E40F2A060C1F200004FF41173B3
:10BB800003FB060292F82012032915D140F2A067A8
:10BB9000C1F2000703FB06750DF1700C1B9848F607
:10BBA000BD51C0F6020148F6D152C0F6020205F5B9
:10BBB0008873FEF7C5F833E442F27C04C2F2010454
:10BBC0004FF04806267204F0DBB94FF000001C90DD
:10BBD0001C9B40F2A062C1F200024FF4117101FB04
:10BBE000032696F8200203283DD140F2A067C1F257
:10BBF000000701FB037505F588750DF1700CFDF765
:10BC00001DF88DF86A00D5F804211C924FF0000150
:10BC10001B91D5F800711346974207D0AE5C86425F
:10BC200019D04FF001024FF0000E0CE04FF0FF0072
:10BC30001B9010E002F10106E95C814202D11C93E5
:10BC40001B9208E03246FF2B14BF013373469F421C
:10BC5000F0D11C93EAE70DF1700C9DF86C00FCF735
:10BC6000D5FFFFF7DDBB42F27C04C2F201044FF0C6
:10BC70004803237204F084B94FF000031C931C9E08
:10BC800040F2A062C1F200024FF4117101FB0620E4
:10BC900090F82032032B27D140F2A065C1F20005B5
:10BCA00001FB065707F58875D7F81462D7F81022FC
:10BCB000964212D00DF1700CFCF7C0FF8319DFB271
:10BCC0001C970DF1700CE85DFCF7A0FF4FF000052C
:10BCD000219E86F85050FFF7A3BB4FF00101219839
:10BCE00080F85010FFF79CBB42F27C04C2F20104C2
:10BCF0004FF04806267204F043B94FF000021C9240
:10BD00001C9840F2A063C1F200034FF4117101FBD3
:10BD1000003696F82022032A28D140F2A067C1F20B
:10BD2000000701FB007505F58876D6F80431D6F8D2
:10BD300000118B4213D00DF1700CF05CFCF766FF24
:10BD4000D6F80471FF2F14BF01370027C6F804711D
:10BD50004FF00005219E86F85050FFF761BB4FF071
:10BD60000102219880F85020FFF75ABB42F27C0470
:10BD7000C2F201044FF04800207204F001B94FF004
:10BD800000031C931D991B9142F2B812C2F20102EA
:10BD9000D2F800801B9F08EB070640F20000C0F6B7
:10BDA0000200864208D942F27C06C2F201064FF038
:10BDB0001F02327204F0E4B81C9B032B08D942F234
:10BDC0007C00C2F201004FF03703037204F0D8B8D0
:10BDD000F1780D2908D942F27C04C2F201044FF037
:10BDE0003701217204F0CCB840F2A065C1F2000521
:10BDF0004FF4117202FB035090F820323BB118F857
:10BE0000071021B10FE04846FDF706FF05E04CF2B0
:10BE10004F354FF09609DDF82CB0FBF715FACBEB58
:10BE20000002AA42EFD918F80770032F3FF6F8AACC
:10BE3000DFE807F002080F169DF87000FFF702F820
:10BE4000FFF7EEBA9DF87000314607F003FCFFF7EC
:10BE5000E7BA9DF87000314605F0C8FEFFF7E0BA7A
:10BE60009DF87050B77828464FF00301FEF7BEFFEB
:10BE70004FF4117000FB05F340F2A061C1F2000124
:10BE8000C85800283FF4CCAA4AF2C053C0F60303B6
:10BE900007EB470703EB0708F6784AF6C842C0F6F7
:10BEA000030252F82610DA5D98F8013098F8027013
:10BEB00000974FF00006019649F28D17C0F6020771
:10BEC000029749F2CD17C0F60207039749F2FD1712
:10BED000C0F60207049749F21D47C0F6020705970E
:10BEE000069646682846B047FFF79ABA4FF0000119
:10BEF0001C911D981B908DF86A101C9840F2A0634D
:10BF0000C1F200034FF4117101FB003696F82022B4
:10BF1000032A79D140F2A065C1F2000501FB005768
:10BF200007F5887942F2B813C2F201031968219E1D
:10BF3000B26B01EB020B8B5CFF2B5CD0D8464FF051
:10BF400001054FF0000B0994CDF830A0AA4698F8EF
:10BF5000014004EB032742F2B813C2F201031E684A
:10BF6000F219D9F804111C919DF86A0018B1F75D17
:10BF700002F1010200E05F4602F1FF349DF86A50D1
:10BF80002DB177B9099C5046DDF830A005E0637803
:10BF90003BB9099C5046DDF830A01C99C9F8041142
:10BFA0002BE01C99D9F800618E4218D014F8016F6B
:10BFB00019F801501B9A3AB930460AF081FBC6B213
:10BFC00028460AF07DFBC5B2AE4208D11C98FF2876
:10BFD00014BF013058461C9007F1FF37CEE70AF135
:10BFE000010A18F8023FFF2BB1D1099CDDF830A0FF
:10BFF0004FF0000001E04FF000000DF1700CC0B2F6
:10C00000FCF704FEFFF70CBA42F27C04C2F2010412
:10C010004FF04800207203F0B3BF4FF000031C93B1
:10C020001E9E1B964FF001028DF86A2065E74FF0C7
:10C0300000021C921C9E40F2A060C1F200004FF46E
:10C04000117303FB060191F82022032A31D140F23B
:10C05000A065C1F2000503FB065707F588750DF1D1
:10C06000700CFCF7EBFD8DF86A004FF000031C9399
:10C07000D5F80471D5F800118F4212D0EA5D8242E2
:10C080000FD14FF00006FF2F14BF01373746B942DA
:10C0900002D1C5F8047104E0EB5D8342F3D0C5F82A
:10C0A00004710DF1700C4FF00000FCF7AFFDFFF7CD
:10C0B000B7B942F27C04C2F201044FF0480626727E
:10C0C00003F05EBFFBF7C0F80B9D401B0DF1700C39
:10C0D0004CF24F37B8428CBF00200120FCF796FD90
:10C0E000FFF79EB94FF000001C901C9E40F2A0622A
:10C0F000C1F200024FF4117101FB062393F82052A4
:10C10000032D7FF48DA940F2A067C1F2000701FB67
:10C11000067000F10406D0F80811D6F8002102F1EB
:10C120000102914238BF01F580718B1AFF2B34BF99
:10C130001D46FF250DF1700CE8B2FCF767FDFFF717
:10C140006FB91D9F41F60870C2F20100C65D06F18D
:10C15000FF31C155FFF764B91D9BFA2B08D942F294
:10C160007C04C2F201044FF01300207203F008BFF8
:10C1700041F60870C2F20100C25C02F1FF36F1B272
:10C18000C15400293FF44CA91E9B1C9301F044B8F4
:10C190001D9EFA2E08D942F27C04C2F201044FF02F
:10C1A0001306267203F0ECBE41F60871C2F20101DB
:10C1B0008A5D02F1FF33D8B28855002842F03584F9
:10C1C000FFF72EB91D9BFA2B08D942F27C04C2F26C
:10C1D00001044FF01303237203F0D2BE41F608713D
:10C1E000C2F20101CA5C02F1FF30C6B2CE54002E89
:10C1F00002F01B84FFF714B9219D95F8517007F1E7
:10C20000FF3185F85110FFF70BB9219890F84720BE
:10C2100002F1FF3680F84760FFF702B9219BD86C26
:10C220000AF060F9219DE864FFF7FAB8219F97EDC5
:10C23000137AD7ED127A37EE270A87ED130A219980
:10C24000C86C0AF0C3F830B14FF00205219981F8AB
:10C250005050FFF7E5B8219BD86C0AF0C7F830B111
:10C260004FF00102219880F85020FFF7D9B84FF025
:10C270000006219F87F85060FFF7D2B89DF8740040
:10C28000219901F14C01FEF7B9F88DF86B000028F7
:10C290003FF4C6A842F27C04C2F20104207203F00B
:10C2A0006FBE9DF874002199C96CFEF7DBF88DF81C
:10C2B0006B0000283FF4B4A842F27C02C2F20102F3
:10C2C000107203F05DBE2198C06C0AF08FF820B99F
:10C2D000219EB06C0AF08AF830B14FF00300219E25
:10C2E00086F85000FFF79CB8219BD3ED13BA93ED6D
:10C2F00012BA7BEECB0A10EE900A0AF0F3F80CEEBD
:10C30000100A1BEE900A1BEE101A0AF085F801467F
:10C310004FF07E500AF080F801EE100A61EE281A04
:10C32000B4EEE1CAF1EE10FA06D84FF00001219AFE
:10C3300082F85010FFF774B8219D95ED132AD5EDC2
:10C34000122AB4EEE22AF1EE10FA05DD4FF00107F1
:10C3500085F85070FFF764B8B4EEE22AF1EE10FAF7
:10C360004CBF0222032285F85020FFF759B8219BC9
:10C3700093ED133AF7EE003A33EE634A83ED134A36
:10C380002198C06C0AF032F830B14FF003072199C0
:10C3900081F85070FFF744B8219A92ED13BA7BEE02
:10C3A00049BA1BEE900A0AF09DF80BEE900A1BEEBC
:10C3B000100A19EE101A0AF02FF801464FF07E50BD
:10C3C0000AF02AF800EE100A60EE280AF4EEE0BA4D
:10C3D000F1EE10FA1ED9219E96ED13BA3BEE091A22
:10C3E00011EE100A0AF07EF80BEE900A1BEE100A0E
:10C3F0001AEE901A0AF010F801464FF07E500AF03B
:10C400000BF801EE900A21EEA82AF4EEC2BAF1EE82
:10C4100010FA06D84FF00406219B83F85060FEF70F
:10C42000FFBF219BDF6C38460AF05CF80BEE100A68
:10C43000384618EE101A09F0EFFF01464FF07E5013
:10C4400009F0EAFF02EE900A22EEA83AB4EEC3BA6F
:10C45000F1EE10FA06D84FF00000219A82F8500051
:10C46000FEF7DEBF2199D1ED133AF4EEC83AF1EEB2
:10C4700010FA05DD4FF0010581F85050FEF7D0BFEE
:10C48000F4EEC83AF1EE10FA4CBF0222032281F812
:10C490005020FEF7C5BF219DD5ED124A95ED135AE8
:10C4A000C4EE855AC5ED135AC9E62199C86C09F046
:10C4B00089FF002840F0AE86FEF7B2BF219AD66C05
:10C4C00030460AF00FF80BEE100A304618EE101A3C
:10C4D00009F0A2FF01464FF07E5009F09DFF06EEE5
:10C4E000100A66EE286AB4EEE6BAF1EE10FA00F32E
:10C4F0009186FEF795BF2198C06C09F063FF002874
:10C5000000F08886FEF78CBF219B93ED137AD3ED64
:10C51000127AB4EEE77AF1EE10FA80F27B86FEF73B
:10C520007FBF219991ED130AD1ED120AB4EEE00A12
:10C53000F1EE10FA00F36E86FEF772BF219A92EDCB
:10C54000131AD2ED121AB4EEE11AF1EE10FA40F21B
:10C550006186FEF765BF219E96ED132AD6ED122A5D
:10C56000B4EEE22AF1EE10FA00F15486FEF758BF5D
:10C570002198C66C304609F0B5FF0BEE100A304624
:10C5800018EE101A09F048FF01464FF07E5009F0EE
:10C5900043FF03EE100A63EE283AB4EEE3BAF1EE7D
:10C5A00010FA40F23786FEF73BBF219FF86CFCF78C
:10C5B0007DF9F8640DF1700C4FF00000FCF712FCEF
:10C5C000FEF72EBF1D9BF62B08D942F27C04C2F267
:10C5D00001044FF01203237203F0D2BC219DE86CDA
:10C5E00009F0F0FE38B9219AD2ED134AB6EE005A9E
:10C5F00034EE85BA06E0219991ED13BAB6EE004A01
:10C600003BEE44BA1BEE100A09F0DCFE88B9B4EE2A
:10C61000CABAF1EE10FA04DC1BEE100A09F0D6FEDD
:10C6200038B14FF00100219E86F850006FF00040B5
:10C630002CE01BEE100A09F0C5FE88B1B4EEE9BA91
:10C64000F1EE10FA04D41BEE100A09F0BFFE38B167
:10C650004FF00101219A82F850104FF0004015E090
:10C660001BEE100A09F0C2FE38B14FF00205219B03
:10C6700083F850504FF0000008E0BDEECBBA1BEE3F
:10C68000100A4FF00006219F87F850604FEA0067BC
:10C6900047EA106500F47F4345EA032100F47F0276
:10C6A00041EA122042F2BC06C2F201061D9FF0517F
:10C6B000FEF7B6BE1D99F62908D942F27C04C2F2F3
:10C6C00001044FF01203237203F05ABC42F2BC057E
:10C6D000C2F201056A584FEA026040EA126602F4AB
:10C6E0007F4746EA072302F47F0143EA112505EE5E
:10C6F000905AB8EEE56A219880ED136AB4EECA6AE2
:10C70000F1EE10FA04DCB4EEE96AF1EE10FA05D5A8
:10C710004FF0010680F85060FEF782BE4FF0000235
:10C7200080F85020FEF77CBE0DF1700C4FF0010038
:10C73000FCF758FB219FF86CFCF7E2F82199C864DC
:10C74000FEF76EBE219DD5ED136AB7EE007A76EE48
:10C75000877AC5ED137A13E6219DE86C09F046FE51
:10C7600050B1219F4FF0000187F847104FF00405AA
:10C7700087F85050FEF754BE219890ED134AB4EE5E
:10C78000C84AF1EE10FA23DB9FEDD66AB4EEC64A32
:10C79000F1EE10FA0FD5FCEEC46A16EE902A0DF1F8
:10C7A000700CD0B2FCF732FA4FF00006219B83F8F0
:10C7B0005060FEF735BE0DF1700C4FF0FF00FCF736
:10C7C00025FA4FF00205219880F85050FEF728BE58
:10C7D000B4EEC84AF1EE10FA7EF522AEDFEDC24AA1
:10C7E000B4EEE44AF1EE10FA11DDB1EE445AFCEE7B
:10C7F000C55A15EE903A0DF1700CD8B2FCF706FA56
:10C800004FF00107219981F85070FEF709BE0DF134
:10C81000700C4FF0FF00FCF7F9F94FF00302219E76
:10C8200086F85020FEF7FCBD1D98F92808D942F281
:10C830007C04C2F201044FF01300207203F0A0BB8D
:10C84000219A92ED137AFDEEC77A17EE906A33B211
:10C850001C939FB2C6F3072141EA072541F60872EF
:10C86000C2F201021552FEF7DBBD1D9EF92E08D95A
:10C8700042F27C04C2F201044FF01306267203F068
:10C880007FBB219B93ED130AFCEEC00A10EE907A59
:10C89000BDB21C954FEA152141EA052241F6087008
:10C8A000C2F201008253FEF7BBBD1D9F219B9F6416
:10C8B000FEF7B6BD1D9D2199CD64FEF7B1BD0DF10A
:10C8C000700CFCF7BBF901EE100AF8EE411A219A40
:10C8D000C2ED131AFEF7A4BD1D98F92808D942F23B
:10C8E0007C04C2F201044FF01300207203F048BB35
:10C8F00041F60876C2F20106375A4FEA172343EA97
:10C900000725A9B202EE101AF8EE422A219AC2EDCA
:10C91000132A9FED763AF4EEC32AF1EE10FAFEF6F2
:10C920007FADDFED733A32EEE34A82ED134AFEF754
:10C9300077BD1D9EF92E08D942F27C04C2F2010493
:10C940004FF01306267203F01BBB41F60877C2F2C4
:10C950000107BB5B4FEA132545EA03218AB204EEC7
:10C96000902AB8EE645A219880ED135AFEF758BD0C
:10C970001D98072808D942F27C03C2F201034FF048
:10C980000801197203F0FCBAFCF7ACFD05EE900A41
:10C99000B8EE656A219F87ED136AFEF741BD219DC0
:10C9A000D5ED136A95ED127A66EE877AC5ED137AA6
:10C9B00045E4219A92ED130AF1EE400AC2ED130A02
:10C9C000FEF72EBD4FF000004FF001010A46FDF7C3
:10C9D000D9FC219890ED131AF1EE041A21EE212AC8
:10C9E0004FF000060096019642F2C810C2F2010014
:10C9F000FCEEC22A12EE901A4FF0FF024AF2E9331F
:10CA0000C0F60203FAF7EAFBFEF70ABD1D9BF72BFF
:10CA100008D942F27C04C2F201044FF013022272E0
:10CA200003F0AEBA41F60877C2F20107F858FBF7F7
:10CA300067FF21998864FEF7F3BC1D98F72808D991
:10CA400042F27C03C2F201034FF01301197203F0AA
:10CA500097BA41F60875C2F201052858FBF750FF56
:10CA6000219EF064FEF7DCBC1D9A072A08D942F229
:10CA70007C04C2F201044FF00806267203F080BA6B
:10CA8000219F97ED133AB4EEC83AF1EE10FA0DDBA0
:10CA9000B4EEC93AF1EE10FA08D8FCEEC33ACDED87
:10CAA0001C3A4FF0000587F8505028E0B4EEC93A20
:10CAB000F1EE10FA07DD6FF07F421C924FF001009B
:10CAC00087F850001BE04FF000001C9013EE100A96
:10CAD00009F078FC70B14FF00201219B83F85010EF
:10CAE0000DE000BF00008043000080C3000000474D
:10CAF000800080474FF00305219E86F850501D9816
:10CB00001C99FCF7C1FCFEF78BBC219FF86C09F067
:10CB10006DFC00287EF484AC219991ED134AB4EEAB
:10CB2000C84AF1EE10FA04DD4FF07E52CA64FEF7F7
:10CB300077BCB4EEC84AF1EE10FA7EF571AC4FF056
:10CB40000003CBF68073CB64FEF76ABC2198856A3C
:10CB5000CDB1FAF779FB219FB96AC1F10403181826
:10CB60004CF6CD42CCF6CC42A2FB00154FEA95061E
:10CB7000796AB6FBF1F304EE903AB8EE645A87EDA9
:10CB8000135AFEF74DBC4FF6FF76C7F67F76C664A4
:10CB9000FEF746BC1D9EF72E08D942F27C04C2F275
:10CBA00001044FF01300207203F0EAB9219FF86CE2
:10CBB000FBF77CFE41F60872C2F201029051FEF7CB
:10CBC0002FBC219DD5ED125A95ED136A75EEC66AFC
:10CBD000C5ED136AFFF733BB219BDE6C1C969F6C7F
:10CBE000DF649E64FEF71CBC219AD06C09F0FEFB4A
:10CBF00030B14FF00306219981F85060FEF710BC68
:10CC00002198C06C09F0E2FB30B14FF00400219D87
:10CC100085F85000FEF704BC219DEE6C304609F00B
:10CC200061FC0BEE100A304618EE101A09F0F4FB06
:10CC300001464FF07E5009F0EFFB07EE100A67EE59
:10CC4000287AB4EEE7BAF1EE10FA06D84FF00007F2
:10CC5000219A82F85070FEF7E3BB219991ED130AF7
:10CC6000B4EEC80AF1EE10FA05DD4FF0010381F8C9
:10CC70005030FEF7D5BBB4EEC80AF1EE10FA4CBF47
:10CC80000222032281F85020FEF7CABB219BD3ED7C
:10CC900013BA93ED12BA3BEECBCA1CEE100A09F0A0
:10CCA00021FC0CEE100A1BEE900A1BEE101A09F084
:10CCB000B3FB01464FF07E5009F0AEFB00EE900A48
:10CCC00020EEA81AB4EEC1CAF1EE10FA0DF1700C04
:10CCD0008CBF00200120FBF799FFFEF7A1BB219F2D
:10CCE000FD6C284609F0FEFB0BEE100A284618EEF4
:10CCF000101A09F091FB01464FF07E5009F08CFBB1
:10CD000001EE900A21EEA82AB4EEC2BAF1EE10FAB2
:10CD10000DF1700C8CBF00200120FBF777FFFEF7B0
:10CD20007FBB219AD2ED132A92ED123AF4EEC32A78
:10CD3000F1EE10FA0DF1700CB4BF00200120FBF7EA
:10CD400065FFFEF76DBB2198D0ED133AF5EEC03AC2
:10CD5000F1EE10FA0DF1700CB4BF00200120FBF7CA
:10CD600055FFFEF75DBB219E96ED134AD6ED124AA4
:10CD7000B4EEE44AF1EE10FA0DF1700CD4BF0020CD
:10CD80000120FBF743FFFEF74BBB219991ED135AAE
:10CD9000D1ED125AB4EEE55AF1EE10FA0DF1700C25
:10CDA0008CBF00200120FBF731FFFEF739BB219B30
:10CDB00093ED136AD3ED126AB4EEE66AF1EE10FA5F
:10CDC0000DF1700C54BF00200120FBF71FFFFEF790
:10CDD00027BB219F97ED137AB5EEC07AF1EE10FADA
:10CDE0000DF1700C54BF00200120FBF70FFFFEF780
:10CDF00017BB219DD5ED13BA95ED12BA7BEECB7A18
:10CE000017EE900A09F06EFB0CEE100A1BEE900A6A
:10CE10001BEE101A09F000FB01464FF07E5009F09E
:10CE2000FBFA00EE100A60EE280AB4EEE0CAF1EE5A
:10CE300010FA0DF1700CD4BF00200120FBF7E6FEC4
:10CE4000FEF7EEBA219AD66C304609F04BFB0BEE9A
:10CE5000100A304618EE101A09F0DEFA01464FF0BB
:10CE60007E5009F0D9FA01EE100A61EE281AB4EEEC
:10CE7000E1BAF1EE10FA0DF1700CD4BF00200120E0
:10CE8000FBF7C4FEFEF7CCBA1D98F82808D942F289
:10CE90007C04C2F201044FF01303237203F070B854
:10CEA000FAF7D2F9219B00F104004CF6CD41CCF603
:10CEB000CC41A1FB00174FEA97055A6AB5FBF2F780
:10CEC0001D9D41F60870C2F2010041194E78425D85
:10CED0004FEA024545EA0620897840EA01061B969A
:10CEE000BF1B27F07F421C9202EE102AF8EE422A66
:10CEF000C3ED132AFEF794BA219DE86CA864FEF7EF
:10CF00008FBA219991F85160002E40F08381FEF78D
:10CF100087BA219A92F85130002B00F07B81FEF7FE
:10CF20007FBA1D98FA2808D942F27C04C2F20104A3
:10CF30004FF01303237203F023B841F60871C2F2D5
:10CF400001010E5C002E7EF46BAA1E9A1C9263E116
:10CF50001D98FA2808D942F27C04C2F201044FF06D
:10CF60001303237203F00CB841F60871C2F20101F9
:10CF70000E5C002E3EF454AA1E9A1C924CE142F222
:10CF80007C00C2F201004FF00101017202F0F8BF13
:10CF90001D9EF92E08D942F27C04C2F201044FF022
:10CFA0001206267202F0ECBF42F2BC02C2F201028B
:10CFB000905D1E9B18427EF433AA1F991C912BE1B1
:10CFC0001D98F92808D942F27C04C2F201044FF0FE
:10CFD0001200207202F0D4BF42F2BC02C2F201027F
:10CFE000115C1E9B19423EF41BAA1F9E1C9613E166
:10CFF0001D99FA2908D942F27C04C2F201044FF0CB
:10D000001300207202F0BCBF41F60872C2F20102A6
:10D01000535C002B7EF404AA1E9E1C962DE11D99E4
:10D02000FA2908D942F27C04C2F201044FF013003D
:10D03000207202F0A5BF41F60872C2F20102535CF1
:10D04000002B3EF4EDA91E9E1C9616E11D99FA29AF
:10D0500008D942F27C04C2F201044FF0130121729C
:10D0600002F08EBF41F60872C2F20102565C1E9BAE
:10D070009E427EF6D5A91F981C90CDE01D9EFA2EEB
:10D0800008D942F27C04C2F201044FF01306267262
:10D0900002F076BF41F60872C2F20102905D1E9B5B
:10D0A0009842FEF4BDA91F991C91B5E01D98FA287D
:10D0B00008D942F27C04C2F201044FF0130020723E
:10D0C00002F05EBF41F60872C2F20102115C1E9BC3
:10D0D00099427EF4A5A91F9E1C969DE01D99FA29F0
:10D0E00008D942F27C04C2F201044FF0130121720C
:10D0F00002F046BF41F60872C2F20102565C1E9B66
:10D100009E423EF48DA91F981C9085E01D9EFA2E2C
:10D1100008D942F27C04C2F201044FF013062672D1
:10D1200002F02EBF41F60872C2F20102905D1E9B12
:10D1300098423EF675A91F991C916DE01D98FA283A
:10D1400008D942F27C04C2F201044FF013002072AD
:10D1500002F016BF41F60872C2F20102115C1E9B7A
:10D160009942BEF45DA91F9E1C9655E0219A92F843
:10D1700047101D9B99427EF453A91E9E1C967CE08D
:10D18000219890F847201D998A423EF449A91E9B98
:10D190001C9372E0219E96F847001D9A90427EF6FD
:10D1A0003FA91E991C9168E0219B93F847601D9848
:10D1B0008642FEF435A91E9A1C925EE0219991F8F0
:10D1C00047601D9B9E42BEF42BA91E981C9054E004
:10D1D000219A92F847101D9EB1423EF621A91E9B4E
:10D1E0001C934AE09DF874000DF16B01FCF7EAFF17
:10D1F0008DF86A009DF86B1031B142F27C04C2F2E6
:10D200000104217202F0BCBE00283EF409A91E9858
:10D210001C9001E01D9A1C921C9A40F20000C0F67E
:10D22000010090F82E1090F82F3043EA0126964224
:10D2300008D242F27C04C2F201044FF009022272C9
:10D2400002F09EBE42F2C017C2F201073A60FEF73A
:10D25000E7B80DF1700CFBF7F1FC1C900028D9D059
:10D26000FEF7DEB80DF1700CFBF7E8FC1C9000280F
:10D27000D0D1FEF7D5B81D9E1C96219E336A052B92
:10D2800008D942F27C04C2F201044FF00A0323726F
:10D2900002F076BE03F1020242F2C010C2F20100B7
:10D2A000016846F8221003F10103219E3362B3E7BF
:10D2B0000DF1700CFBF7C2FC1C900028DBD0FEF7D0
:10D2C000AFB80DF1700CFBF7B9FC1C900028D2D15F
:10D2D000FEF7A6B80DF1700CFBF7B0FC1C901D9B7F
:10D2E00098427EF49DA81E991C9195E70DF1700C53
:10D2F000FBF7A4FC1C901D9A90423EF491A81E9846
:10D300001C9089E70DF1700CFBF798FC1C901D9E9A
:10D31000B0427EF685A81E9B1C937DE70DF1700C34
:10D32000FBF78CFC1C901D998842FEF479A81E9A8C
:10D330001C9271E70DF1700CFBF780FC1C901D9E98
:10D34000B042BEF46DA81E981C9065E70DF1700CFC
:10D35000FBF774FC1C901D9B98423EF661A81E9939
:10D360001C9159E79DF874000DF16B01FCF7FAFE72
:10D370008DF86A009DF86B6036B142F27C04C2F20F
:10D380000104267202F0FCBD00283EF449A81E9A52
:10D390001C9241E79DF874000DF16B01FCF7E2FE71
:10D3A0008DF86A009DF86B3033B142F27C01C2F215
:10D3B00001010B7202F0E4BD00287EF431A81E9832
:10D3C0001C9029E70DF1700CFBF760FC41F6087624
:10D3D000C2F201061E9AB05C1D9B18423EF420A8C2
:10D3E0001F991C9118E70DF1700CFBF74FFC41F6EB
:10D3F0000876C2F201061E9AB05C1D9B18427EF4AC
:10D400000FA81F991C9107E70DF1700CFBF73EFC6C
:10D4100041F60876C2F201061E9AB05C1D9B1842C6
:10D420007DF4FEAF1F991C9127E70DF1700CFBF7FF
:10D430002DFC41F60876C2F201061E9AB05C1D9BD7
:10D4400018423DF4EDAF1F991C9116E798F8005073
:10D4500045F0080288F80020FEF70BB80DF1700CBB
:10D46000FBF7ECFB8DF86A00219991F851601D9B48
:10D47000F1181C911E9AC2F1FB06B14208D942F282
:10D480007C04C2F201044FF01303237202F078BD52
:10D490004FF000071B971E99D9B11C9D41F60873E8
:10D4A000C2F201035A5D824234D001F1FF3241F6EB
:10D4B0000876C2F20106731941F60877C2F2010735
:10D4C000C7F10101C5EB010E12F0010F1AD002F0F5
:10D4D000C2BD4FF0FF001B901CE013F8019F02F14A
:10D4E000FF36484504D11C95CDF86CC01E9211E062
:10D4F0003246CD180EEB030C13F8017FB84242F010
:10D50000B785F0E7CD180EEB030C002AE5D11C958A
:10D510001E92DEE70DF1700C9DF86C00FBF776FBB8
:10D52000FDF77EBF0DF1700CFBF788FB42F2340B68
:10D53000C2F2010B8BF800004FF001011C91CDF8F5
:10D5400034B095E0219E96F851201D9813181C9335
:10D55000F92B08D942F27C04C2F201044FF0130106
:10D56000217202F00DBD1E981B900DF1700C26ADBE
:10D5700045F0010122AF47F001024FF00003FBF735
:10D5800097FBFDF74DBF219E96F851201D9813186B
:10D590001C93FA2B08D942F27C04C2F201044FF02A
:10D5A0001301217202F0ECBC1F9D1E98A84228BFF7
:10D5B00028461B900DF1700C26AF47F0010122AEFA
:10D5C00046F001024FF00003FCF7BAFBFDF728BF5D
:10D5D0000DF1700CFBF732FB034642F2340BC2F242
:10D5E000010B58464FF010014BF2B462C0F6030233
:10D5F00009F0C2F81C90CDF834B039E01E9A1C92A4
:10D600001F981B904FF000030D9331E04FF0FF3651
:10D610001C960D962CE02199C86C9DF878109DF809
:10D620007C2042F23406C2F2010600964FF010034D
:10D6300001934FF00103FDF737FA4FF0FF321C92D0
:10D640000D9615E02198C06C9DF878109DF87C200F
:10D6500042F23406C2F2010600964FF01003019325
:10D660004FF00003FDF720FA4FF0FF311C910D96AB
:10D670001D9800F10506F2B20C92A0F1FB010329FE
:10D6800023D840F2A060C1F200004FF411760C9A4A
:10D6900006FB020191F82032032B08D042F27C00F5
:10D6A000C2F201004FF04806067202F069BC40F277
:10D6B000A060C1F200004FF411770C9E07FB060733
:10D6C00007F104074FF0000605E0219F97F851305D
:10D6D0001E184FF00007DDF870B0BBF1FF3F0CD112
:10D6E0004FF0FF0B4FF00009C84641F60872C2F236
:10D6F00001020E920F950D9D05E0BBF1000FF1D1D7
:10D700004FF0000961E01D99A1F1FB01032910D838
:10D71000D7F80061FF2E14BF01364646D7F8043112
:10D720009E4206D14046FCF777FAD7F804018642BC
:10D73000F8D0B5F1FF3F15D1219850F8343F1A6861
:10D74000D2F800C0494610AA4FF00103E0478DF817
:10D750006B0080B10F9D42F27C04C2F20104207282
:10D7600002F00EBC25B115F809108DF8401002E04A
:10D770001B9A8DF840201C98B0F1FF3F02D19DF814
:10D78000401011B31D9BA3F1FB03032B07D8D7F85F
:10D7900000119DF840307B54C7F8006111E0FA2E6B
:10D7A00009D90F9D42F27C04C2F201044FF0130626
:10D7B000267202F0E5BB9DF840200E98825506F1D6
:10D7C000010609F10109D9459DD31D9FA7F1FB076A
:10D7D000032F04D80C98FBF7C1FCFDF721BE219D57
:10D7E00095F8512009EB020E85F851E0FDF718BEBF
:10D7F0001D9AA2F1FB0003285AD802F10502D7B204
:10D8000040F2A060C1F200004FF4117101FB070269
:10D8100092F82032032B08D042F27C04C2F20104B9
:10D820004FF04803237202F0ABBB40F2A066C1F296
:10D8300000064FF4117505FB076505F104051E98F8
:10D8400000F1FF311E9170B34FF0000842F2C01991
:10D85000C2F2010940F200029346C0F6010BD5F86E
:10D860000061FF2E14BF01364646D5F804319E42B2
:10D8700006D14046FCF7D0F9D5F804018642F8D02D
:10D88000D9F80030D5F800211BF80310A95403F192
:10D890000103C9F80030C5F800611E9E06F1FF3093
:10D8A0001E90002EDBD13846FBF758FCFDF7B8BDC3
:10D8B0001E9B1C93219991F8510082181B92C3F171
:10D8C000FB06B24208D942F27C04C2F201044FF0D6
:10D8D0001306267202F054BBC51881F851501C9AE9
:10D8E00002F1FF351C95002A3DF49AAD42F2C017B3
:10D8F000C2F201073E681B9F41F60873C2F20103A2
:10D90000D91940F20000C0F6010030184FF00003B2
:10D9100005F0010E10F803C001F803C003F1010384
:10D92000934242F089830DE010F8038001F80380F0
:10D9300003F1010310F803E001F803E003F1010330
:10D940009342F1D1E819A91901F1010142F2C01283
:10D95000C2F2010211604FF0FF331C9300F101008D
:10D960001B90FDF75DBD4FF000028DF86A20219EEF
:10D9700096F851001D9BC1181C911E9A1B92C2F172
:10D98000FB00814208D942F27C04C2F201044FF04C
:10D990001303237202F0F4BA41F60877C2F20107CA
:10D9A00007EB01099DF87CB042F2B815C2F20105FF
:10D9B0002A68B66B9119975DFF2F52D088464FF0B9
:10D9C000010009900C9498F8014004EB072742F2FB
:10D9D000B815C2F201052A68D6194FF000011C9152
:10D9E0009DF86A30002B02F0FD82D75D06F101063A
:10D9F00002F0FABA9DF86A5015B15FB90C9C02E0CA
:10DA000062783AB90C9C219E96F85120851886F8C8
:10DA1000515029E014F8015F19F800B046B92846C2
:10DA200008F04EFEC5B2584608F04AFE5FFA80FB89
:10DA30005D4508D11C9800F101001C9007F1FF37EB
:10DA40001B998142D6D2B346099B03F10103099386
:10DA500018F8027FFF2FB6D10C9C4FF00000099000
:10DA600002E04FF0000309930DF1700C0999C8B260
:10DA7000FBF7CCF8FDF7D4BC4FF001018DF86A102C
:10DA800075E70DF1700CFBF7D9F8034642F2340B41
:10DA9000C2F2010B58464FF010014BF2BC62C0F6C7
:10DAA000030208F069FE1C90CDF834B0E0E50DF1FA
:10DAB000700CFBF7C3F8034642F2340BC2F2010BC1
:10DAC00058464FF010014BF2C462C0F6030208F052
:10DAD00053FE1C90CDF834B0CAE50DF1700CFBF785
:10DAE000ADF8034642F2340BC2F2010B58464FF038
:10DAF00010014BF2C862C0F6030208F03DFE1C9014
:10DB0000CDF834B0B4E50DF1700CFBF797F803468F
:10DB100042F2340BC2F2010B58464FF010014BF2A7
:10DB2000D062C0F6030208F027FE1C90CDF834B096
:10DB30009EE5219991F8513003F1010381F85130AC
:10DB4000FDF76EBC1D9F41F60875C2F20105EA5D46
:10DB500002F10102EA55FDF763BC219890F8476095
:10DB600006F1010680F84760FDF75ABC9DF8740085
:10DB70000DF16B01FCF7F6FA0DF1700CFBF746F8AE
:10DB80009DF86B1000293DF44BAC42F27C04C2F2CC
:10DB90000104217202F0F4B99DF874000DF16B01DB
:10DBA000FCF748FB0DF1700CFBF730F89DF86B307B
:10DBB000002B3DF435AC42F27C02C2F2010213723A
:10DBC00002F0DEB91D981C904FF000061B964FF036
:10DBD00001018DF86A109DF870000DF16B01FCF7E2
:10DBE000C1FA9DF86B309BB920B19DF86A201B9853
:10DBF00010431B909DF86A604FEA46018DF86A1049
:10DC00001C9B03F101031C9311F0FE0FE3D10AE00A
:10DC10009DF86A20012A06D142F27C04C2F2010476
:10DC2000237202F0ADB90DF1700C9DF86C00FAF79B
:10DC3000EDFFFDF7F5BB1D981C904FF000061B96FD
:10DC40004FF001018DF86A109DF870000DF16B0125
:10DC5000FCF7F0FA9DF86B309BB920B19DF86A2073
:10DC60001B9810431B909DF86A604FEA46018DF89F
:10DC70006A101C9B03F101031C9311F0FE0FE3D10A
:10DC80000AE09DF86A20012A06D142F27C04C2F221
:10DC90000104237202F074B90DF1700C9DF86C0050
:10DCA000FAF7B4FFFDF7BCBB9DF874000DF16B01F2
:10DCB000FCF788FA8DF86A009DF86B6036B142F285
:10DCC0007C00C2F20100067202F05AB90DF1700C2C
:10DCD000FAF79CFFFDF7A4BB1D991C914FF00003C0
:10DCE0001B934FF001008DF86A00219A92F847606B
:10DCF00030420ED09DF870000DF16B01FCF762FA16
:10DD00009DF86B1099B920B19DF86A001B9B0343E5
:10DD10001B939DF86A204FEA42068DF86A601C99B1
:10DD200001F101011C9116F0FE00DED10AE09DF820
:10DD30006A30012B06D142F27C04C2F20104217246
:10DD400002F01EB91B9F219D85F84770FDF768BB47
:10DD50009DF874000DF16B01FCF79CFA0DF1700C4D
:10DD6000FAF754FF9DF86B60002E3DF459AB42F278
:10DD70007C02C2F20102167202F002B91D991C91D6
:10DD8000C8B20DF16B01FCF785FA1B909DF86B0092
:10DD900030B142F27C04C2F20104207202F0F0B809
:10DDA0004FF001038DF86A301C9FFA181C92D0B214
:10DDB0000DF16B01FCF76EFA9DF86A5000FA05F060
:10DDC0001B9E06431B9605F101058DF86A501C9AAF
:10DDD00002F101021C92E9B20729E8D90DF1700C99
:10DDE0009DF86C00FAF712FFFDF71ABB0DF1700CED
:10DDF000219890F85100FAF709FFFDF711BBFDF7E4
:10DE00000FBB42F26903C2F201034FF001071F701A
:10DE1000FDF706BB42F26905C2F201054FF00006AC
:10DE20002E70FDF7FDBA21984FF000014FF054021B
:10DE300009F0D8F84FF00002219242F24401C2F2F8
:10DE400001010C6804F1FF30086002F005B842F2ED
:10DE50004402C2F2010211687F2908D942F27C040F
:10DE6000C2F201044FF03000207202F089B84FF086
:10DE700001071C9740F2A065C1F20005D5F8A8097A
:10DE8000002842F0BC8005E0D6F8AC1000294ED145
:10DE90001C9301E04FF001031D9840F2A066C1F20F
:10DEA00000064FF0540505FB03F3F218C2F85009C1
:10DEB000C2F854091E9982F8A2194FF00A07C2F855
:10DEC000747906F51567F81800F13400219901F10D
:10DED00034014FF0100209F061F81C9B05FB037040
:10DEE00000F14400219901F144014FF0040209F0CE
:10DEF00055F81C9805FB007000F14800219901F1CC
:10DF000048014FF0080209F049F8219A92F851109F
:10DF10001C9F05FB076686F8A11942F24405C2F270
:10DF200001052B6803F101032B60FDF779BA03F1BA
:10DF300001073B4606F15406D6F8AC50002D42F0DE
:10DF40007280A5E71C93FDF76BBA219B93F8526092
:10DF50001E967CE70DF1700CFAF770FE1E9076E7C6
:10DF60001D9A219981F85120FDF75ABA0DF1700CD4
:10DF70009DF87400FAF74AFEFDF752BA219EB36A83
:10DF8000002B3DF44DAAF9F75FF921998A6A801AAE
:10DF90004E6A1D9B06FB03F303EB83018842BDF42D
:10DFA0003FAA1E9A1C92FFF737B9F9F74DF9219F46
:10DFB000B862FDF735BA42F2BC00C2F2010090F837
:10DFC000FB201E9E9319FB2B08D942F27C00C2F263
:10DFD00001004FF01206067201F0D2BF1D9BC2F184
:10DFE000FB018B4208DD42F27C04C2F201044FF0D7
:10DFF0001302227201F0C4BF42F2BC05C2F2010555
:10E00000A81941F60877C2F20107F91808F0C6FF0F
:10E01000FDF706BA98F8003043F0100188F80010B8
:10E02000FDF727BA219D95F84770002F0CBFFF22FE
:10E03000002285F84720FDF7F3B9219890F8476052
:10E040006FEA060380F84730FDF7EAB90DF1700C6E
:10E05000FAF71CFE1E9D41F60877C2F201077A5DB1
:10E060001D9951407955FDF7DBB92198866B1D9BB1
:10E070009A191C92A1E12199C86B8E6B83191C938C
:10E080009BE121990A6C42B942F27C04C2F201047C
:10E090004FF02000207201F073BF02F1FF350D64D4
:10E0A000FDF7BEB9219E336C03F101033364002BED
:10E0B0007DF4B6A942F27C01C2F201014FF02002C8
:10E0C0000A7201F05DBF2198466B3368596841B907
:10E0D00042F27C00C2F201004FF01E03037201F015
:10E0E0004FBF0DF1700CFAF7A9FD1C90219850F864
:10E0F000342F166876681D991CAA4FF00103B047AB
:10E100008DF86B0000283DF48BA942F27C04C2F22A
:10E110000104207201F034BF0DF1700CFAF78EFD8E
:10E120001C9038E10DF1700CFAF788FD219FF8631F
:10E13000FDF776B90DF1700CFAF780FD219D28648A
:10E14000FDF76EB9219850F8341F0A6816681D99BA
:10E150001CAA4FF00103B0478DF86B0030B142F2BA
:10E160007C04C2F20104207201F00ABF0DF1A80C78
:10E170001CF8380DFAF74AFDFDF752B92198436BA8
:10E180000DF1700C187AFAF741FDFDF749B90DF160
:10E19000700C219F97F83C00FAF738FDFDF740B965
:10E1A00021990A6CFF2A08D942F27C06C2F20106C4
:10E1B0004FF02004347201F0E3BE0DF1700CD0B2C8
:10E1C000FAF724FDFDF72CB9219850F8345F2B683D
:10E1D0009F68B84703EE100AF8EE433A2198C0ED65
:10E1E000133AFDF71DB9219991ED0E4AF8EE444A14
:10E1F000C1ED134AFDF714B9219A92ED105AF8EEC9
:10E20000455AC2ED135AFDF70BB9219E96ED136ADC
:10E21000FCEEC66ACDED1C6ACFE0219BD3ED137AEC
:10E220009FEDC17AF4EEC77AF1EE10FA08DB42F204
:10E230007C04C2F201044FF02000207201F0A0BE65
:10E24000BCEEE70A83ED100AFDF7EAB8219850F812
:10E25000341F0A6816681D991CAA4FF00403B047C2
:10E260008DF86B0030B142F27C03C2F201031872E8
:10E2700001F086BE1C98FAF743FB219DA864FDF7C8
:10E28000CFB8219850F8341F0A6816681D991CAA47
:10E290004FF00403B0478DF86B0030B142F27C04BC
:10E2A000C2F20104207201F06BBE1C98FAF728FB41
:10E2B000219FF864FDF7B4B82198436B19684A6848
:10E2C00042B942F27C00C2F201004FF01E0101721D
:10E2D00001F056BEC06CFAF7E9FA1C90219850F88C
:10E2E000346F33685E681D991CAA4FF00403B04771
:10E2F0008DF86B0000283DF493A842F27C04C2F232
:10E300000104207201F03CBE1D9A2198C36BC3F139
:10E31000FB06B24208D942F27C04C2F201044FF07B
:10E320001300207201F02CBE50F8347F39680E685B
:10E330004FF0000141F60877C2F20107BA18B04762
:10E340008DF86B0000283DF46BA842F27C03C2F20A
:10E350000103187201F014BE219850F8342F11688F
:10E360000E681D991BAA4FF00403B0478DF86B008F
:10E3700030B142F27C04C2F20104207201F000BE0E
:10E380001B9B98B2C3F3072242EA00218EB21C966F
:10E3900013E01D9B1C931C982199FAF7EDFC8DF856
:10E3A0006B0000283DF43CA842F27C02C2F201025C
:10E3B000107201F0E5BD1D981C901C9EB6F5803FC3
:10E3C00008D342F27C04C2F201044FF01F0323720F
:10E3D00001F0D6BD219DAE63FDF722B81D9D219FA2
:10E3E000FD63FDF71DB81D99219E3164FDF718B836
:10E3F000219B9A6B1D98111A1C91DEE71E9A219B96
:10E40000D96B8818FB2808D942F27C03C2F20103B9
:10E410004FF012021A7201F0B3BD42F2BC07C2F211
:10E42000010787F8FB10184650F8346F31680E6802
:10E430001D99BA18DB6BB0478DF86B0000283CF4CF
:10E44000EFAF42F27C04C2F20104207201F098BDE9
:10E450002198416B0E68766846B942F27C06C2F29A
:10E4600001064FF01E02327201F08ABD1D9AC36B85
:10E47000C3F1FB018A4208D942F27C00C2F20100DA
:10E480004FF01303037201F07BBD00F134004FF035
:10E49000000141F60877C2F20107BA18B0478DF8BB
:10E4A0006B0000283CF4BCAF42F27C04C2F20104D1
:10E4B000207201F065BDF7F72FFA00287CF4B0AFA9
:10E4C0001D991C91FEF7A8BEF7F726FA00283CF428
:10E4D000A7AF1D981C90FEF79FBE1D9B072B08D968
:10E4E00042F27C04C2F201044FF00506267201F0EC
:10E4F00047BDD8B24FF00001F7F7CCF900EE900A13
:10E50000B8EE601A219F87ED131AFCF789BF1D9A98
:10E51000072A0BD942F27C01C2F201014FF005003B
:10E52000087201F02DBD00BF00008047D0B24FF04F
:10E530000101F7F7AFF901EE900AB8EE612A219DCB
:10E5400085ED132AFCF76CBF1D9B072B08D942F2FF
:10E550007C04C2F201044FF00506267201F010BDE2
:10E56000D8B24FF00001F7F705F9FCF759BF1D9A33
:10E57000072A08D942F27C01C2F201014FF00500DE
:10E58000087201F0FDBCD0B24FF00101F7F7F2F8CC
:10E59000FCF746BF1D9B072B08D942F27C04C2F250
:10E5A00001044FF00506267201F0EABCD8B24FF024
:10E5B0000001F7F72FF9FCF733BF1D9A072A08D996
:10E5C00042F27C01C2F201014FF00500087201F035
:10E5D000D7BCD0B24FF00101F7F71CF9FCF720BF10
:10E5E0009DF87400F2F774FF00287CF419AF42F232
:10E5F0007C03C2F201034FF028041C7201F0C0BC7E
:10E600009DF87400219901F14C01F2F781FF002877
:10E610007CF406AF42F27C06C2F201064FF02802FB
:10E62000327201F0ADBC2199D1ED132A9DF874002E
:10E63000BCEEE23A13EE101AF2F79CFF00287CF4CD
:10E64000EFAE42F27C00C2F201004FF028030372E9
:10E6500001F096BCFCF7E4BE0DF1700CFAF7EEFA8F
:10E6600030B9219F97F847502E1C18BF012601E0B2
:10E670004FF00106219A82F84760FCF7D1BE9DF861
:10E6800074600DF1700CFAF7D9FA014630464FF07C
:10E690000102FBF777FE8DF86B0000283CF4C0AE5A
:10E6A00042F27C04C2F20104207201F069BC0DF157
:10E6B000700CFAF7C3FA01468DF86A009DF87400F1
:10E6C000FBF71EFE8DF86B0000283CF4A9AE42F269
:10E6D0007C01C2F20101087201F052BC1D981C902D
:10E6E0004FF001038DF86A301E46219A92F84710C8
:10E6F0000B420AD092F846109DF87000194032463D
:10E70000FBF740FE8DF86B0068B99DF86A304FEA60
:10E7100043008DF86A001C9A02F101021C9210F06D
:10E72000FE03E2D10AE09DF86A60012E06D142F2B2
:10E730007C04C2F20104207201F022BC4FF00007F9
:10E740008DF86B700DF1700CFAF778FA0DF1700C12
:10E75000FAF774FAFCF764BE9DF874004FF00101FB
:10E760000A46FBF70FFE8DF86B0000283CF458AE0C
:10E7700042F27C01C2F20101087201F001BC9DF875
:10E7800074004FF000014FF00102FBF7FBFD8DF824
:10E790006B0000283CF444AE42F27C02C2F201025B
:10E7A000107201F0EDBB0DF1700CFAF747FA219DE4
:10E7B00095F84730184385F84700FCF731BE1D989F
:10E7C0000DF1A80C4CF8380DFAF7E6FE00287CF4A1
:10E7D00027AE42F2C010C2F20100099E066001F0AD
:10E7E00052BB10A8FAF76AFD014640B19DF840708F
:10E7F000022F04D0D1484FF00D0208F0CFFB0DF1ED
:10E80000700C9DF84000FAF701FAFCF709BEFBF71F
:10E8100017FAFCF705BE0DF1700CFAF70FFAFCF7CA
:10E82000FFBD1D9EFA2E08D942F27C04C2F20104FB
:10E830004FF01202227201F0A3BB0DF1700CFAF737
:10E84000FDF942F2BC01C2F201018855FCF7E8BDB6
:10E850000DF1700CFAF7F2F942F2BC05C2F20105B3
:10E8600085F8FB00FCF7DCBD0DF1700C219B93F8E3
:10E870004700FAF7CBF9FCF7D3BD1D98FA2808D961
:10E8800042F27C06C2F201064FF01201317201F031
:10E8900077BB0DF1700C42F2BC07C2F20107385C85
:10E8A000FAF7B4F9FCF7BCBD0DF1700C42F2BC02F2
:10E8B000C2F2010292F8FB00FAF7A8F9FCF7B0BD2A
:10E8C0001D9EF62E08D942F27C04C2F201044FF0DC
:10E8D0001200207201F054BB219DA86CF9F7E6FFED
:10E8E00042F2BC03C2F201039851FCF799BD1D9995
:10E8F000FA2908D942F27C06C2F201064FF013024F
:10E90000327201F03DBB0DF1700C41F60877C2F296
:10E910000107785CFAF77AF9FCF782BD0DF1700C0B
:10E92000FAF7B4F941F60875C2F201051E9BE85CDE
:10E930001D9908420DF1700C0CBF0020FF20FAF762
:10E9400065F9FCF76DBD1D9EF92E08D942F27C00D9
:10E95000C2F201004FF01301017201F011BB41F648
:10E960000872C2F20102905D9319597841EA0026BB
:10E970001C96002E3CF454ADFEF74EBC1D9BFA2BAA
:10E9800008D942F27C04C2F201044FF01300207255
:10E9900001F0F6BA41F60876C2F20106F25C002AEE
:10E9A00043D1FCF73DBD1D99FA2908D942F27C04F8
:10E9B000C2F201044FF01302227201F0E1BA41F6F3
:10E9C0000873C2F201035E5C7EB3FCF729BD0DF152
:10E9D000700CFAF733F91C9038BBFCF721BD0DF130
:10E9E000700CFAF753F941F60870C2F201001E9953
:10E9F000465C1D9B1E4218D0FCF712BD0DF1700C39
:10EA0000FAF744F941F60872C2F201021E98115C4D
:10EA10001D9E314209D1FCF703BD0DF1700CFAF7D0
:10EA20000DF91C9000287CF4FBAC219B1A6A42B9BA
:10EA300042F27C04C2F201044FF00300207201F0A4
:10EA40009FBA02F1FF351D6202F1010253F82270F4
:10EA500042F2C011C2F201010F60FCF7E1BC219D3E
:10EA600095F847704FEAD71343EA470285F84720E5
:10EA7000FCF7D6BC219890F847604FEA560141EA6E
:10EA8000C61580F84750FCF7CBBCFAF7E9FCFCF759
:10EA9000C7BC41F60077C2F20107FB784FF00100D6
:10EAA00000FA03F03A7922EA00023A71FCF7B8BCA6
:10EAB00042F27C04C2F201044FF00106267201F01A
:10EAC0005FBA41F60071C2F20101CD7845B941F655
:10EAD0000070C2F201004FF00602C270FCF7A0BC49
:10EAE00005F1FF3741F60073C2F20103DF70FCF756
:10EAF00097BC41F60076C2F20106317801F1FF358C
:10EB0000EFB237703379FF2B0BD1632F7CF688ACD3
:10EB100041F60076C2F201064FF063013170FCF756
:10EB20007FBC172F7CF67CAC41F60070C2F201006E
:10EB30004FF017020270FCF773BC00BF0E1F0120DC
:10EB400041F60075C2F201056F7807F1FF33D8B2C4
:10EB500068702A79FF2A0BD100287CF461AC41F659
:10EB60000075C2F201054FF00C076F70FCF758BC3E
:10EB70003B287CF655AC41F60076C2F201064FF018
:10EB80003B017170FCF74CBC42F27C04C2F2010400
:10EB90004FF00103237201F0F3B942F27C00C2F29C
:10EBA00001004FF00102027201F0EAB942F27C0664
:10EBB000C2F201064FF00101317201F0E1B942F2F7
:10EBC0007C04C2F201044FF00103237201F0D8B9B2
:10EBD00041F60075C2F20105EF78052F08D941F61C
:10EBE0000076C2F201064FF00002F270FCF718BC8A
:10EBF00007F1010741F60070C2F20100C770FCF78F
:10EC00000FBC41F60071C2F201010B7803F1010360
:10EC1000DDB20D700F79FF2F0BD1632D7CF600ACA8
:10EC200041F60071C2F201014FF000020A70FCF7D8
:10EC3000F7BB172D7CF6F4AB41F60070C2F2010071
:10EC40004FF000060670FCF7EBBB41F60075C2F210
:10EC500001056B7803F10103DFB26F702879FF289B
:10EC60000BD10C2F7CF6DCAB41F60075C2F201052E
:10EC70004FF001026A70FCF7D3BB3B2F7CF6D0ABA0
:10EC800041F60076C2F201064FF000017170FCF708
:10EC9000C7BB42F27C04C2F201044FF001032372AD
:10ECA00001F06EB941F60077C2F20107F8784FF033
:10ECB000010606FA00F6397986EA01053D71FCF78E
:10ECC000AFBB0DF1700CF9F7B9FF41F60072C2F25B
:10ECD00001021071FCF7A4BB0DF1700CF9F7AEFF47
:10ECE000062841F60073C2F2010392BFD8700027D4
:10ECF000DF70FCF795BB0DF1700CF9F79FFF41F643
:10ED00000076C2F201063070FCF78ABB0DF1700C80
:10ED1000F9F794FF41F60071C2F201014870FCF767
:10ED20007FBB0DF1700CF9F789FF41F60075C2F257
:10ED30000105A870FCF774BB0DF1700C41F6007072
:10ED4000C2F201000079F9F761FFFCF769BB0DF130
:10ED5000700C41F60072C2F20102D078F9F756FF4A
:10ED6000FCF75EBB0DF1700C41F60073C2F20103BB
:10ED70001878F9F74BFFFCF753BB0DF1700C41F617
:10ED80000077C2F201077878F9F740FFFCF748BB3B
:10ED90000DF1700C41F60076C2F20106B078F9F779
:10EDA00035FFFCF73DBB42F27C04C2F201044FF098
:10EDB0000101217201F0E4B81D9A0F2A08D942F22C
:10EDC0007C04C2F201044FF02700207201F0D8B891
:10EDD000C24D05EB820041F60073C2F2010315F843
:10EDE00022701F7046785E704FF000019970D970E4
:10EDF00082781A71FCF714BB42F27C03C2F2010361
:10EE00004FF001061E7201F0BBB841F60075C2F268
:10EE10000105EF784FF0010101FA07F12A7941EA83
:10EE200002002871FCF7FCBA42F27C04C2F2010431
:10EE30004FF00103237201F0A3B842F27C06C2F244
:10EE400001064FF00101317201F09AB84FF0000550
:10EE5000139512951195199541F60077C2F20107A5
:10EE60003A7802F164021692787800F1FF33159334
:10EE7000BE78149611A807F0B7FE179919B101F1E1
:10EE8000FF37FDB201E04FF0060541F60072C2F215
:10EE90000102D570FCF7C4BA1D9E0F2E08D942F2AC
:10EEA0007C04C2F201044FF02706267201F068B814
:10EEB0008A4800EB860141F60073C2F201031D7817
:10EEC00000F826505F784F701A798A70FCF7A8BA5C
:10EED00042F27C00C2F201004FF00101017201F028
:10EEE0004FB80DF1700C219B93F85000F9F78EFE8E
:10EEF000FCF796BA42F28C02C2F20102147814F0C6
:10EF0000010F08D142F27C04C2F201044FF030023A
:10EF1000227201F035B842F24406C2F201063068AE
:10EF200040B942F27C01C2F201014FF031030B7291
:10EF300001F026B842F28C01C2F201010B7803F015
:10EF4000FE0242F004040C7042F25806C2F20106BE
:10EF50004FF00000306000F07FBF42F28C06C2F23A
:10EF60000106307810F0010F08D142F27C06C2F29F
:10EF700001064FF03000307201F002B842F2440155
:10EF8000C2F201010B6843B942F27C04C2F20104EF
:10EF90004FF03402227200F0F3BF42F28C04C2F24E
:10EFA0000104227802F0FE0646F00200207042F2D0
:10EFB0005801C2F201014FF000030B6000F04CBF9A
:10EFC000219D95F846700DF1700CF9F737FE2199E7
:10EFD0003B1A91F8502002F00106981B1C9081F812
:10EFE0004700FF2894BF0020012081F85000FCF763
:10EFF00017BA1D9BFA2B08D942F27C04C2F2010415
:10F000004FF01301217200F0BBBF41F60875C2F248
:10F0100001051E9FEF54FCF703BA4FF000021C924B
:10F020001AE04FF001061C9616E04FF002001C900B
:10F0300012E04FF003031C930EE04FF004051C9503
:10F040000AE04FF005071C9706E04FF006011C91FF
:10F0500002E04FF007021C921D991B911C98FAF7D1
:10F0600013FAFCF7DDB90DF1700CF9F70FFE1E9ED7
:10F0700041F60873C2F20103985D1D9D05439D553D
:10F08000FCF7CEB91D9EF92E08D942F27C04C2F2DB
:10F0900001044FF01202227200F072BF42F2BC076C
:10F0A000C2F201071E99B955FCF7BAB942F2BC0089
:10F0B000C2F201001D9B80F8FB30FCF7B1B942F2AF
:10F0C0007826C2F20106316851B942F27C00C2F2E0
:10F0D00001004FF00106067200F052BF443A0010E2
:10F0E0004E681D981E994FF001020DF16A03B0475A
:10F0F0008DF86B009DF86A20D2F1010138BF002124
:10F10000219B83F8501000283CF48AA942F27C0429
:10F11000C2F20104207200F033BF42F27822C2F240
:10F120000102116841B942F27C00C2F201004FF0C5
:10F130000106067200F024BF0B681D981E999847BF
:10F140008DF86B0000283CF46BA942F27C04C2F2FB
:10F150000104207200F014BF42F27822C2F20102D0
:10F16000116841B942F27C00C2F201004FF0010681
:10F17000067200F005BF4E681D981E994FF0000200
:10F180000DF16A03B0478DF86B009DF86A30D3F13A
:10F19000010238BF0022219981F8502000283CF458
:10F1A0003FA942F27C04C2F20104207200F0E8BEE2
:10F1B0000A981E99F9F762FF0A9040B942F27C065C
:10F1C000C2F201064FF01702327200F0D9BE0A9B5C
:10F1D0001A68966A46B942F27C00C2F201004FF00A
:10F1E0001503037200F0CCBE0A9988689DF874106C
:10F1F00042F2BC02C2F20102B0478DF86B00002857
:10F200003CF40EA942F27C04C2F20104207200F028
:10F21000B7BE0A981E99F9F731FF0A9040B942F239
:10F220007C00C2F201004FF01703037200F0A8BE89
:10F230000A990868436943B942F27C01C2F20101AC
:10F240004FF015020A7200F09BBE0A9EB0689DF84E
:10F25000741042F2BC02C2F2010298478DF86B00B2
:10F2600000283CF4DDA842F27C04C2F201042072C2
:10F2700000F086BE0A981E99F9F700FF0A9040B97F
:10F2800042F27C06C2F201064FF01701317200F023
:10F2900077BE0A9F3E68B76947B942F27C00C2F266
:10F2A00001004FF01503037200F06ABE42F2BC0683
:10F2B000C2F201060A9988689DF8741032460DF171
:10F2C0006A03B8478DF86B009DF86A2032700028F9
:10F2D0003CF4A6A842F27C04C2F20104207200F0C1
:10F2E0004FBE0A981E99F9F7C9FE0A901D9E7F2EFF
:10F2F00009D1051C18BF012542F2BC07C2F2010763
:10F300003D70FCF78DB80A9A42B942F27C00C2F215
:10F3100001004FF01703037200F032BE0A98036831
:10F320005B6843B942F27C06C2F201064FF0150257
:10F33000327200F025BE0A998868F1B242F2BC022E
:10F34000C2F2010298478DF86B0000283CF468A8CF
:10F3500042F27C04C2F20104207200F011BE0A984D
:10F360001E99F9F78BFE0A9040B942F27C06C2F270
:10F3700001064FF01702327200F002BE0A990E68C1
:10F38000B76847B942F27C00C2F201004FF01501A4
:10F39000017200F0F5BD42F2BC06C2F201060A9A03
:10F3A00090689DF8741032780DF16A03B8478DF8B3
:10F3B0006B009DF86A30337000283CF431A842F2AB
:10F3C0007C04C2F20104207200F0DABD0A981E9992
:10F3D000F9F754FE0A9040B942F27C06C2F20106E7
:10F3E0004FF01700307200F0CBBD0A9F3B68DF681A
:10F3F00047B942F27C03C2F201034FF015021A72C0
:10F4000000F0BEBD42F2BC06C2F201060A98806856
:10F410009DF8741032460DF16A03B8478DF86B0001
:10F420009DF86A10317000283BF4FAAF42F27C0478
:10F43000C2F20104207200F0A3BD0A981E99F9F7E8
:10F440001DFE0A9040B942F27C03C2F201034FF064
:10F4500017061E7200F094BD0A9F39680F6947B9FC
:10F4600042F27C00C2F201004FF01501017200F07F
:10F4700087BD0A9BD3F808809DF8749042F2BC06C1
:10F48000C2F201063068F9F73BFA024640464946A7
:10F490000DF16A03B8478DF86B009DF86A20327051
:10F4A00000283BF4BDAF42F27C04C2F2010420729A
:10F4B00000F066BD0A984FF00001F9F7DFFD0A90F1
:10F4C00040B942F27C00C2F201004FF01703037210
:10F4D00000F056BD0A9A1068C36A43B942F27C062E
:10F4E000C2F201064FF01502327200F049BD0A99CE
:10F4F00088689DF8741098478DF86B0000283BF4DD
:10F500008FAF42F27C04C2F20104207200F038BDD9
:10F510000A981E99F9F7B2FD0A9040B942F27C06AA
:10F52000C2F201064FF01703337200F029BD0A99A9
:10F530000E68F36943B942F27C00C2F201004FF059
:10F540001501017200F01CBD0A9A90689DF87410B4
:10F5500042F2BC02C2F2010298478DF86B0000280B
:10F560003BF45EAF42F27C04C2F20104207200F070
:10F5700007BD0A981E99F9F781FD0A9040B942F239
:10F580007C00C2F201004FF01706067200F0F8BCD2
:10F590000A9A1068066A46B942F27C03C2F2010375
:10F5A0004FF015021A7200F0EBBC0A9988689DF8BA
:10F5B000741042F2BC02C2F20102B0478DF86B0037
:10F5C00000283BF42DAF42F27C04C2F20104207209
:10F5D00000F0D6BC0A981E99F9F750FD0A9040B980
:10F5E00042F27C01C2F201014FF017020A7200F0F0
:10F5F000C7BC0A990B685E6A46B942F27C03C2F244
:10F6000001034FF015061E7200F0BABC0A9A90680A
:10F610009DF8741010AAB0478DF86B001098F9F798
:10F6200045F942F2BC01C2F2010108609DF86B008D
:10F6300000283BF4F5AE42F27C04C2F201042072D1
:10F6400000F09EBC0A984FF00001F9F717FD0A90F0
:10F6500040B942F27C03C2F201034FF017061E725A
:10F6600000F08EBC0A9803681E6B46B942F27C001B
:10F67000C2F201004FF01502027200F081BC0A993B
:10F6800088689DF8741042F2BC02C2F20102B047D1
:10F690008DF86B0000283BF4C3AE42F27C04C2F24A
:10F6A0000104207200F06CBC1D99072908D942F2B0
:10F6B0007C04C2F201044FF00801217200F060BC2A
:10F6C00040F2A065C1F2000505EBC107D7F81009AB
:10F6D00000287BF4A5AEF7F7B7FD002808BF01208E
:10F6E00040F2A062C1F200021D9B02EBC306C6F805
:10F6F0001009FBF795BE1D98072808D942F27C0433
:10F70000C2F201044FF00801217200F039BC40F24E
:10F71000A065C1F2000505EBC007D7F81029002A43
:10F720003BF47EAEF7F790FD1D9B40F2A066C1F260
:10F73000000606EBC305D5F81019401A1C90D5F841
:10F740001479B8428CBF0027C0EB07071B9740F223
:10F75000A062C1F2000202EBC3031B9EC3F814694E
:10F760004FF00005C3F81059FBF75ABE1D9EFA2E44
:10F7700007D942F27C00C2F201004FF0130202727C
:10F78000FEE30DF1700CF9F759FA41F60877C2F271
:10F790000107B855FBF744BE0DF1700CF9F776FA86
:10F7A0000DF1700CF9F74AFA1C9050B11E9B41F60E
:10F7B0000872C2F20102D05C1D9D0543D554FBF7CF
:10F7C0002FBE1E9B41F60875C2F20105EE5C1D9925
:10F7D00026EA0107EF54FBF723BE1D9E1E9A9119DE
:10F7E000CBB242F2BC00C2F2010080F8FB30FA2B2F
:10F7F00007D942F27C04C2F201044FF012012172D7
:10F80000BEE342F2C017C2F201073D6842F2BC01FA
:10F81000C2F20101881940F20006C0F60106A919DA
:10F8200007F0BCFB3A681E9BD0183860FBF7F8BDA8
:10F830001D9EF82E07D942F27C04C2F201044FF05B
:10F84000130323729CE3F7F7FFFC00F104004CF66E
:10F85000CD47CCF6CC47A7FB00154FEA9500219A7F
:10F86000536AB0FBF3F61C961D9F41F60871C2F275
:10F8700001014FEA1645CD55C8194FEA16224270CC
:10F880008670FBF7CDBD1D9EF82E07D942F27C0491
:10F89000C2F201044FF01302227271E3F7F7D4FCB5
:10F8A00000F104004CF6CD47CCF6CC47A7FB002175
:10F8B0004FEA91052198426AB5FBF2F61D9B41F68D
:10F8C0000877C2F20107F8184178FD5C4FEA05425B
:10F8D00042EA0127837847EA03001B90361A26F094
:10F8E0007F411C910DF1700C1E9881422CBF0020AD
:10F8F0000120F9F78BF9FBF793BD219D95F8467030
:10F900000DF1700CF9F79AF9381A1C90219B83F8C5
:10F910004700FF2894BF0020012083F85000FBF728
:10F920007FBD1D9EF92E07D942F27C06C2F2010668
:10F930004FF01303337223E342F2C011C2F201010C
:10F940000A6841F60873C2F201034FEA1220985583
:10F950009E197270FFF769B8219D95F847201C9297
:10F9600095F8467085F8477085F84620FBF758BD36
:10F970001D98072807D942F27C01C2F201014FF01D
:10F9800008040C72FCE2F9F7ADFD0DF1A80C4CF87F
:10F99000380D003018BF0120F9F738F9FBF740BDEA
:10F9A000219E96F8470096F846300DF1700C98426B
:10F9B00014BF00200120F9F729F9FBF731BD219D83
:10F9C00095F8470095F846200DF1700C801A18BF85
:10F9D0000120F9F71BF9FBF723BD219F97F847009A
:10F9E00097F846100DF1700C88422CBF00200120C2
:10F9F000F9F70CF9FBF714BD219E96F8470096F82D
:10FA000046300DF1700C984294BF00200120F9F7A8
:10FA1000FDF8FBF705BD219D95F8470095F84620B8
:10FA20000DF1700C90428CBF00200120F9F7EEF828
:10FA3000FBF7F6BC219F97F8470097F846100DF1A9
:10FA4000700C884234BF00200120F9F7DFF8FBF783
:10FA5000E7BC1D98F62807D942F27C04C2F20104E3
:10FA60004FF0120222728BE242F2BC06C2F2010691
:10FA70003058F8F745FF219BD864FBF7D1BC1D999E
:10FA8000F62907D942F27C00C2F201004FF01206BB
:10FA9000067275E242F2BC05C2F201056858F8F739
:10FAA0002FFF219FB864FBF7BBBC42F2BC03C2F23C
:10FAB000010393F8FB201D9E9119FB2907D942F2FF
:10FAC0007C06C2F201064FF01201317258E21E9B11
:10FAD000C2F1FB00834207DD42F27C04C2F2010462
:10FAE0004FF0130222724BE241F60875C2F2010593
:10FAF000E81842F2BC07C2F20107B91907F04EFA42
:10FB0000FBF78EBC2198436B1A6856683EB942F2E7
:10FB10007C06C2F201064FF01E02327230E21E9ADB
:10FB200042F2BC01C2F2010191F8FB309918FB29A5
:10FB300007D942F27C00C2F201004FF012030372B7
:10FB40001EE200F134001D9942F2BC07C2F2010727
:10FB5000BA18B0478DF86B0000283BF461AC42F254
:10FB60007C04C2F2010420720AE242F27C01C2F279
:10FB700001014FF001040C7202E20DF1700CF9F773
:10FB800085F841F60875C2F201051E9FE85D1D9BD0
:10FB900018423BF445AC42F2C016C2F20106099A83
:10FBA000326070E10DF1700CF9F770F841F60871F0
:10FBB000C2F201011E9D4F5D1D9807427BF430ACDF
:10FBC00042F2C014C2F20104099B23605BE19DF87C
:10FBD00074000DF16B01FAF7C5FA8DF86A009DF813
:10FBE0006B602EB142F27C00C2F201000672C7E1E6
:10FBF00000283BF415AC42F2C012C2F2010209998E
:10FC0000116040E19DF874000DF16B01FAF7AAFA5A
:10FC1000D0F1010338BF00238DF86A309DF86B00E6
:10FC200028B142F27C02C2F201021072A8E1219DC9
:10FC3000EF6A17B98DF86A7002E09DF86A2062B920
:10FC40000DF1700C1E98F9F7A7FC30B942F2C01400
:10FC5000C2F201040999216015E10DF1700C9DF8C3
:10FC60006A00F8F7D3FF4FF00006219BDE62FBF736
:10FC7000D7BB9DF874000DF16B01FAF773FA8DF89C
:10FC80006A009DF86B602EB142F27C04C2F201045E
:10FC9000267275E100287BF4C3AB42F2C015C2F2B4
:10FCA0000105099F2F60EEE09DF874000DF16B01D6
:10FCB000FAF788FA8DF86A009DF86B1029B142F2C4
:10FCC0007C03C2F2010319725AE100287BF4A8AB4D
:10FCD00042F2C010C2F20100099A0260D3E09DF81E
:10FCE00074000DF16B01FAF76DFA061C18BF0126BE
:10FCF0008DF86A6092E79DF874000DF16B01FAF7D8
:10FD000031FA011C18BF01218DF86A1086E71D9E8B
:10FD1000F62E07D942F27C03C2F201034FF012041F
:10FD20001C722DE12198C06CF8F7C0FD42F2BC05B1
:10FD3000C2F20105A851FBF773BB0DF1700CF8F787
:10FD40007DFF219F97F84710D1F1010238BF0022B3
:10FD5000002814BF164682F0010687F84760FBF7BB
:10FD60005FBB0DF1700CF8F769FF219D95F84730E6
:10FD7000584085F84700FBF753BB0DF1700CF8F7BE
:10FD80005DFF219F87F85100FBF74ABB05F088FD16
:10FD90000DF1A80C4CF8380DFF2828BFFF20C0B289
:10FDA000F8F734FFFBF73CBB05F070FD0DF1A80C34
:10FDB0004CF8380DFF2828BFFF20C0B2F8F726FF07
:10FDC000FBF72EBB05F076FD0DF1A80C4CF8380DB5
:10FDD000FF2828BFFF20C0B2F8F718FFFBF720BBB1
:10FDE00005F04AFD0DF1700C00280CBFFF2000202B
:10FDF000F8F70CFFFBF714BB42F2B810C2F2010097
:10FE000001681D9A881805F099F88DF86B00002894
:10FE10003BF406AB42F27C04C2F201042072AFE074
:10FE20001D9805F049F8FBF7FBBA0DF1700CF8F7D7
:10FE300005FF05F03BF8FBF7F3BA42F2B816C2F241
:10FE4000010635681D9BE81805F052F8FBF7E8BA83
:10FE500005F036F8FBF7E4BA42F24400C2F20100C2
:10FE6000016881B942F28C02C2F20102147804F0F6
:10FE70000206F3B23BB142F27C04C2F201044FF03D
:10FE8000350323727CE042F28C07C2F201073D7811
:10FE900015F0010F7BF4C2AA219828B142F2C011DB
:10FEA000C2F201010A68426042F25804C2F201043F
:10FEB00026687F2E00F29F8006F101061B961C9695
:10FEC00016B94FF001071B976B4E4FF0540542F2E5
:10FED0008C04C2F2010442F24407C2F201071C9BE7
:10FEE00005FB036021909BB9217801F00402D1B297
:10FEF00009B93A6842B9217841F001026FF38202F0
:10FF00002270426842B115E04FF001001C90E6E714
:10FF100042687AB9802B02D003F1010301E04FF06F
:10FF200000031C931B988342D9D14FF00000F9F7CE
:10FF300073FED4E742F25806C2F20106336042F281
:10FF4000C015C2F201052A604FF0000A5446FBF7C3
:10FF500067BA219F396A41F000423A63FBF760BA01
:10FF60004FF00006219D2E63FBF75ABAFBF758BAF3
:10FF70000C9D42F27C00C2F201004FF001040472B9
:10FF800042F27C02C2F20102099E16602198046AC4
:10FF900024B104F1010450F82430099342F27C01A9
:10FFA000C2F20101099A4A604D72F1F775FCF1F74E
:10FFB00073FC219D2E6A7EB14FF000001C90219CA5
:10FFC000236A4BB1F1F768FC1C9901F101011C9106
:10FFD000219A156A8D42F5D84FF00000F9F71CFE02
:10FFE000FBF745B94FF0000706F1FF344FF0000072
:10FFF0005E46FDF7FFBC4FF000031C9361E74FF036
:020000040803EF
:1000000002031C931C4ED6F8AC2032B9FDF740BF5A
:100010002BB0BDEC0A8BBDE8F08F03F1010306F1B4
:100020005406FDF731BF07F1010306F15406812B99
:100030007DF42AAFFDF786BFBEF1000F3DF474AC2E
:1000400010F8039001F8039003F1010393427DF44B
:100050006BACFDF777BCCD180EEB030C13F8017FEA
:1000600002F1FF36B8423DF43EAA3246FDF74ABAE5
:1000700006F1FF32FDF746BAF00F00100000000055
:100080002DE9F04F2DED028B8FB04FF0000842F2BA
:100090005407C2F2010742F24C03C2F20103039378
:1000A00042F2680BC2F2010B40F2A066C1F20006F8
:1000B0009FEDB98B39684FF0FF3041B9F1F7ECFB98
:1000C000386800280CBFFA204FF0FF30FFE7F6F742
:1000D00041FC28B1B8F1320F09D808F1010806E057
:1000E000B8F1330F0CBF4FF034084FF000083A68F6
:1000F000D2B9F1F7D1FBB8F1320F0ED1039C2068D1
:10010000F6F7D4FC4FF00005039B1D60F5F7AAFE3F
:100110004FF00200F9F7BEFC06E0B8F1340F03D14E
:100120004FF00100F9F7B6FC9BF800104FF4117086
:1001300000FB0162D2F81842002CBBD04FF41175BD
:1001400005FB01F303F5887406EB0409315DE02932
:100150000CD199F801000E2808D14FF6FF704946DE
:10016000D9F80021F8F73CFB10B36BE2325D02F0E6
:100170001F0509EB05035A78294605F0010019F817
:100180000550521B01F1FF33002940F078820BE04B
:1001900019F80300151A03F1FF3119F80120AA1A02
:1001A00001F1FF330029F3D112F0FF0F40F04A8232
:1001B000335D4FEA5310072800F23C82DFE810F06D
:1001C00008003A023A023500A6003A028A002601E7
:1001D000335D09F1010513F01F0000F0338209F1CE
:1001E000020905F1020500F1FF3255FA82F402948A
:1001F0004FF000054FF0010A15E019F8011CE8B2B4
:1002000021405246FAF7BEF8002840F01B8205F163
:1002100001054FEA4404FF2CEFD909F101090299C5
:10022000894500F00F825446E7E799F801403868A5
:1002300070B1F6F73BFC4FF000003860F5F712FEA6
:10024000FAF794FE4FF00100F9F724FCF1F724FBD4
:1002500003990B686BB94BF2D460C0F603004FF002
:1002600007014AF29972C0F60202F6F735FB039DC8
:10027000286005A84FF00001F9F73AFE7CB9F6F7BF
:10028000E3FFC1B201F1FF33DDB2FD2D42F2900078
:10029000C2F2010092BF01700122027009E042F235
:1002A0009000C2F20100027802FB04F404EB142473
:1002B000047042F29004C2F2010421780EAB03F8FC
:1002C000241D4FF003004FF000014FF01802F9F722
:1002D00005FCEFE60DF11300F8F7F0FF01469DF87D
:1002E00013508DF81450012D06D828B10DF11500CA
:1002F0004FF00D0206F052FE4FF006004FF00001E5
:100300004FF00E0205ABF9F7E9FBD3E69BF80010BE
:100310004FF4117303FB01F499F80100032872D81C
:10032000DFE800F002263E504FF00100FAF7CEFE63
:100330004FF000050EAB03F8255D4FF00400294691
:100340004FF00102F9F7CAFB4FF0C800F8F730FA96
:1003500032599BF800004FF0010400940195D2F847
:100360000CC04FF416512A464FF00803E04766E1EF
:100370004FF0000142F27C03C2F2010319724FF008
:1003800001040EAB03F8254D4FF004002246F9F7A7
:10039000A5FB54E1AFF300800000000000E06F40D7
:1003A000F9F74EFC0EAB4FF0020103F8251D4FF09C
:1003B00004004FF000014FF00102F9F78FFB4FF0FE
:1003C00001043CE10EAB4FF0120203F8252D4FF073
:1003D00004004FF000014FF00102F9F77FFB4FF0EE
:1003E000C800F8F7E5F935599BF800004FF0010413
:1003F00000944FF000020192ED684FF416414FF067
:100400000803A8471BE14FF0000418E199F80150D8
:10041000A5F102050C2D00F21081DFE815F00D00AA
:1004200067007E000E010E010E010E010E010E018D
:100430000E010E010E019D00315DC1F30403DAB21D
:10044000012A00F0FF8009F1050509F1080403EB1A
:10045000C30003EB400101EBC10303F15403DAB223
:1004600002EB42002418C5EB040CACF1030E0EF0B5
:10047000010A99F8029015F8010C05F035FB53ECD0
:10048000182B05F043FE05F009FC01464846F9F734
:10049000E9FF05F10305A54240F0D780D2E015F849
:1004A000039C15F8010C05F01FFB53EC182B05F00D
:1004B0002DFE05F0F3FB01464846F9F7D3FF05F1A1
:1004C000030515F803AC15F8010C05F00DFB53EC12
:1004D000182B05F01BFE05F0E1FB01465046F9F72D
:1004E000C1FF05F10305A542D9D1ABE099F802306F
:1004F000305DC0F30405A5F10305EAB209F103017B
:100500009C18FF2CC4BF5A42D2B241F60870C2F206
:100510000100C01806F042FD94E099F8023099F805
:1005200003500EAC04F8243D0DF1150041F608719E
:10053000C2F20101C918202D34BF2A46202206F03C
:100540002DFD05F101024FF007004FF00301D2B27B
:100550002346F9F7C3FAADE599F80240C4B999F812
:100560000310A9B904F018FD039A1068F6F79EFA73
:100570004FF0000303980360F5F774FC4BF2E4605E
:10058000C0F6030008F0FCFAF9F73AFC002848D05E
:1005900099F8025099F803404BF2F460C0F603005A
:1005A00044EA052108F0ECFA99F803A0494611F84D
:1005B000022F40F20003C0F6010303EB022541F6CF
:1005C0000874C2F2010404EB0A0001F102014FF0C9
:1005D000800206F0E3FC4FF68071CFF6FF71CAEBA4
:1005E0000100C2B2A018A9184FF0800206F0D6FC94
:1005F000204629464FF48072F2F766F9A0B92046EA
:1006000029464FF4807206F073F880B94FF001006C
:100610004FF000010A460B46F9F760FA4FF001046B
:100620000DE04FF000040AE04FF0000407E04FF047
:10063000000404E04FF0000401E04FF00004002C3F
:100640007FF438ADF8F71CFE34E5BAF1000F3FF443
:1006500026AF15F803AC15F8010C05F045FA53EC7C
:10066000182B05F053FD05F019FB01465046F9F72C
:10067000F9FE05F10305A5427FF411AFE2E700287A
:100680003FF486AD19F80310521A03F1FF33B3F1AA
:10069000FF3F7FF47DAD87E542F28803C2F201039C
:1006A0001B684B634BB19A68824209D0DB684B638D
:1006B0001BB19A688242F9D102E04FF01E007047E8
:1006C0004FF00000704700BF42F2ED13C2F2010389
:1006D0001A78027042F2EC10C2F2010003780B703B
:1006E000704700BF42F2ED13C2F201031B78834250
:1006F00025D842F2EC12C2F2010212789A18904206
:1007000020DAC01A4FEA50034FF0010202FA03F355
:1007100010F0010F09D042F2F810C2F20100026895
:1007200013400B704FF00100704742F2F010C2F21C
:100730000100026813400B704FF0010070474FF04A
:10074000000070474FF00000704700BF10B542F244
:10075000ED13C2F201031B7883427AD842F2EC1205
:10076000C2F2010212789A18904275DAC31A03F0A5
:10077000FE0442F2FC10C2F201000278A418E4B2B6
:100780004FEA53024FF0010000FA02F213F0010F9A
:1007900012D041B142F2F810C2F20100016842EAFF
:1007A000010303601AE042F2F810C2F2010003688C
:1007B00023EA0203036011E041B142F2F010C2F2F9
:1007C0000100036842EA0301016007E042F2F0130E
:1007D000C2F20103196821EA0201196042F2F01025
:1007E000C2F2010001680A4224D042F2F813C2F2B8
:1007F0000103186802420ED020464FF00001F0F7C6
:10080000C9FC04F10102D0B24FF00101F0F7C2FCC3
:100810004FF0010010BD20464FF00101F0F7BAFC87
:1008200004F10101C8B24FF00001F0F7B3FC4FF042
:10083000010010BD20464FF00001F0F7ABFC04F1C1
:100840000102D0B24FF00001F0F7A4FC4FF001001C
:1008500010BD4FF0000010BD4FF0000010BD00BFF4
:1008600008B542F2FC13C2F20103187042F2F4130D
:10087000C2F20103197042F2ED13C2F201031A70C1
:10088000091A01F10101C8B242F2EC12C2F20102EE
:100890001070412801D9EFF791FE40F2E410C2F246
:1008A00000004FF00101F9F7CDFB08BD2DE9F84339
:1008B00042F2FD13C2F2010318784FEA400111F031
:1008C000FF0405D042F2FD12C2F20102147006E0EC
:1008D00042F2FD15C2F201054FF001062E7042F200
:1008E0002027C2F20107387842F2FD13C2F2010359
:1008F000197808420CBF4FF000094FF001094FF082
:1009000000052C464FF0010742F20026C2F2010614
:10091000A84604F01F0207FA02F0AB59184204D0AF
:10092000204649464246F9F72DFD04F10104E4B2A0
:1009300014F01F0FEDD105F10405202DE9D1BDE81C
:10094000F88300BF42F22023C2F20103187042F282
:10095000FD10C2F201004FF001020270704700BFAB
:1009600000B583B042F20020C2F201004FF0000156
:100970004FF00802EFF732FE4FF0000300934FF004
:100980000100019042F22420C2F201004FF47A717A
:100990004FF0060240F6AD03C0F60303F6F71EFC67
:1009A00003B000BD08B542F22420C2F20100F6F700
:1009B0006FFB4FF0CC00FFF7C5FF08BD89B14FEAD0
:1009C000501242F20023C2F2010300F01F004FF068
:1009D000010101FA00F053F82210084343F8220005
:1009E00011E04FEA501242F20023C2F2010300F07C
:1009F0001F004FF0010101FA00F053F8221021EA24
:100A0000000143F822104FF00000704708B54FF482
:100A100040404BF25471C0F6030142F24822C2F248
:100A20000102F9F7CDFA08BD10B584B0144649BBF0
:100A30000DF10D0300930DF10E0001904FF0000039
:100A400001460DF10A020DF10B03F5F7B7F84FF06F
:100A500000018DF80C109DF80B201AB14FF0010326
:100A60008DF80C309DF80A0028B19DF80C1041F06B
:100A700002028DF80C204FF000008DF80F00039B50
:100A8000236001E04FF0140004B010BD70B51446AF
:100A90008AB199B94FF0000001460246F5F706F910
:100AA00006462578F5F7E6F985420AD2735D23708C
:100AB0004FF0000070BD4FF0160070BD4FF01400F5
:100AC00070BD4FF0160070BDF8B515461F464FF0CB
:100AD00000033B70A9B992F8FB0060B14FF000042D
:100AE0002646285D3146F4F7DBFF04F1010495F852
:100AF000FB20A242F5D84FF0010139704FF0000001
:100B0000F8BD4FF01400F8BD10B586B04FF00104E9
:100B10001C70F1B942F25423C2F20103197842F277
:100B20005520C2F20100037802AC00944FF010008F
:100B3000019010461A464FF00103F9F7B5FF4BF24A
:100B40005070C0F60300214608F01AF84FF000007C
:100B500004E04FF000021A704FF0140006B010BD10
:100B60002DE9F04115461C464FF00103237004297E
:100B70007CD8DFE801F0030B7B1B640068782978E0
:100B8000F5F784F84FF00000BDE8F081287842F2D4
:100B90005421C2F2010108706A7842F25523C2F270
:100BA00001031A704FF00000BDE8F0812C786D78D9
:100BB00005F1040546F26761C6F2666181FB052313
:100BC0004FEA630202EB820010F0FF0555D04FF0B0
:100BD0000007A5F1050808F00108042C94BF26467B
:100BE000052630463946F4F75BFFA41BE4B2A5F1B5
:100BF000050515F0FF0544D11DE0042C94BF2646E1
:100C0000052630463946F4F74BFFA31BA5F1050531
:100C100005F0FF0503F0FF04042C94BF26460526CB
:100C200030463946F4F73CFFA21BD4B2A5F10505C6
:100C300015F0FF05E1D14FF00000BDE8F0812E78FE
:100C4000F5F718F9864206D34FF0000020704FF0F8
:100C50001600BDE8F081304605F101014FF00102B8
:100C6000F5F740F84FF00000BDE8F0814FF00000CC
:100C700020704FF01400BDE8F0814FF00000BDE897
:100C8000F0814FFA88F6002EB7D0042C94BF264688
:100C9000052630463946F4F703FFA11BCCB2A5F177
:100CA000050515F0FF05A8D1C5E700BF10B51C4626
:100CB0004FF001032370052941D8DFE801F0030E4E
:100CC00018222C361046F4F7A9FF00283DD14FF02A
:100CD000000020704FF0160010BD4BF2D060C0F63F
:100CE0000300114607F04CFF4FF0000010BD4BF21F
:100CF000C860C0F60300114607F042FF4FF0000045
:100D000010BD4BF2C460C0F60300114607F038FF77
:100D10004FF0000010BD4BF2BC60C0F6030011465E
:100D200007F02EFF4FF0000010BD4BF2B460C0F68C
:100D30000300114607F024FF4FF0000010BD4FF0F4
:100D4000000121704FF0140010BD4FF0000010BDE5
:100D500008B5012805D0022814BF0022012211463F
:100D600003E04FF000024FF001014FF00100F5F7F2
:100D70005FF808BD08B54FF00103137001F1FF31B2
:100D8000032921D8DFE801F0020B12194BF20860A9
:100D9000C0F6030007F0F4FE4FF0000008BD4FF06E
:100DA0000000FFF7D5FF4FF0000008BD4FF0010035
:100DB000FFF7CEFF4FF0000008BD4FF00200FFF735
:100DC000C7FF4FF0000008BD4FF0000010704FF05B
:100DD000140008BD08B5F5F745F84FF001004FF0D5
:100DE00000010A46F5F724F8F5F748F84FF00C0033
:100DF0004FF00001F4F754FEF5F734F808BD00BFDA
:100E0000037B13B9437B13B90EE0994208D301F178
:100E1000FF318A18437B9A428CBF0020012001E0F9
:100E20004FF00000C0B270474FF00100704700BFA4
:100E300010B540F2EC13C2F20003187800F1FF3154
:100E4000CAB2FD2A31D940F6F071C1F200014C6BF3
:100E5000A4684FF00200FFF71FFC38B940F2EC1312
:100E6000C2F200034FF00200187017E04FF00300C9
:100E700040F6F071C1F20001FFF70EFC38B940F204
:100E8000EC11C2F200014FF003020A7006E040F2DA
:100E9000EC13C2F200034FF000001870204640F639
:100EA000F071C1F20001FFF7F7FB40F2EC11C2F262
:100EB0000001087810BD00BF70B4447A24B14FF02F
:100EC000320606FB04F610E0C5784AF6C844C0F6C0
:100ED000030454F82550B5F5964F9DBF49F264665A
:100EE000B6FBF5F606EB86060826847A24B14FF0A9
:100EF000320505FB04F501E041F28835C07A18B1EE
:100F0000FF2808BF012001E04FF0010001B10E6091
:100F100002B1156003B1186070BC704740F2A06365
:100F2000C1F200034FF4117202FB00304FF00001D8
:100F3000C0F810124FF6FF73C0F82C32C0F8181228
:100F4000704700BFF8B505460E4640F2A064C1F2F6
:100F500000044FF4117303FB0044D4F8240200EBA7
:100F60005007F6F771F9D4F82812421A974202D9BD
:100F7000B81AF5F7EFFC23689A6928464FF001018B
:100F8000904740F2A060C1F200004FF4117101FBE4
:100F900005014FF6FF7001F104013246F7F720FC1E
:100FA000A31918714FEA10225A7106F10206C4F80B
:100FB00004614FF00000C4F8080121680B6A28465C
:100FC0009847F5F7FFFA2846FFF7A8FFF8BD00BFDE
:100FD00030B583B040F2A064C1F200044FF4117543
:100FE00005FB0040D0F83002B1F57A7F1BD3A1F5A4
:100FF0007A7163B1837B13B9C37B13B907E099425C
:1010000023D38A1802F1FF32C07B824220D8C8B2B3
:101010000DF10701F9F73EF99DF80710D1F1010034
:1010200038BF002019E04FEAD10402F107024FEA6D
:10103000D20523B121462A46FFF7E2FE58B128190E
:10104000FA288CBF0020012007E04FF0000004E0E8
:101050004FF0000001E04FF0000003B030BD00BFD2
:1010600008B5B0F57A7F21D279B14FEAD00341F6C5
:101070000872C2F2010200F007004FF0010101FA0C
:1010800000F0D15C0843D05408BD4FEAD00341F6CC
:101090000872C2F2010200F007004FF0010101FAEC
:1010A00000F0D15C21EA0000D05408BD00F1180026
:1010B000C0B24FF00102F9F765F908BD10B540F272
:1010C000A064C1F200044FF4117303FB0044D4F890
:1010D0001C02F5F7EBFC4FF00000C4F81C0210BD39
:1010E00038B54FF4117101FB00F140F2A062C1F27A
:1010F00000028C18D4F80831D4F80451AB420BD05C
:101100008958E3188A6A1979904728B1D4F80801F8
:1011100000F10100C4F8080138BD00BF08B540F275
:10112000A063C1F200034FF4117202FB0031D1F849
:10113000082101F10401D1F800319A420BD140F2AB
:10114000A061C1F200014FF4117202FB0010D0F84F
:101150001C02F5F769FA08BD70B582B005468DF836
:10116000071040F2A064C1F200044FF4117303FBB6
:101170000044D4F81802002850D11AB12846FFF7CD
:10118000CDFE4BE0F6F760F8D4F82812431AC4F805
:101190002802D4F81002D4F82422934204D800F193
:1011A0000103B3F5807F04D12846FFF7B7FE4FF067
:1011B0000103D4F81012621802A911F8010D82F887
:1011C0001001C4F81032B4F82C024FF00102F7F706
:1011D00007FBC4F82C0208BB04F5887694F820328B
:1011E000012B03D1304602F0A5FA38B994F8201249
:1011F000022913D1304600F0C1FD78B14FF0010251
:10120000C4F8182240F2A060C1F200004FF411733C
:1012100003FB0505D5F81C02F5F706FA02B070BD10
:10122000836B42F25C22C2F201021360016C42F253
:101230005823C2F201031960C16B40F2F012C2F2EE
:10124000000211604FF0000383630364C3637047BF
:1012500042F25C23C2F201031968816342F2582210
:10126000C2F201021368036440F2F011C2F20001FD
:101270000A68C263704700BF2DE9F04180461746F7
:101280001E4640F6F074C1F20004656BAD68084676
:101290002146FFF701FA002840D1606B0468002C5A
:1012A00031D0616800292ED040F6F074C1F20004FC
:1012B0002046FFF7B5FF204650F8342F13685C68CE
:1012C00041463A463346A04770B140F6F074C1F249
:1012D00000042046FFF7BCFF28462146FFF7DCF953
:1012E0004FF00000BDE8F08140F6F074C1F2000458
:1012F0002046FFF7ADFF28462146FFF7CDF94FF016
:101300000100BDE8F081284640F6F071C1F200010D
:10131000FFF7C2F94FF00000BDE8F0814FF0000088
:10132000BDE8F0812DE9F8430446894690461F4602
:10133000FFF77EFD0146D0B140F6F075C1F2000521
:101340004FF00006AE632E64EE632068C9EB000226
:101350009DF8203002FB03F042463B46FFF78CFF2E
:1013600021689DF824208B182360BDE8F8834FF096
:101370000000BDE8F88300BFF0B585B00D461E46FD
:10138000ADF80E2040F2A062C1F200024FF41171DC
:1013900001FB0020D0F83002037BFF2B03D1427BFE
:1013A000FF2A00F0D0802C68B4F57A7F28D2F92C7F
:1013B00018D821464FF00202FFF722FD002800F066
:1013C000C580002E40F0C58041F60873C2F20103CB
:1013D000BDF80E20E252296801F1020129604FF0A8
:1013E0000100C7E04FF0010000904FF002030193AD
:1013F00028464FF000010DF10E02FFF793FFB9E010
:10140000A4F57A77B7F57A7F2AD240F2E1418C428F
:101410001AD839464FF00102FFF7F2FC002800F01D
:101420009B80002E40F09B80BDF80E004FEA1022FA
:1014300041F60873C2F20103DA55296801F101018E
:1014400029604FF0010095E04FF0010300930193F4
:1014500028464FF47A710DF10E02FFF763FF89E021
:10146000A4F6B831B1F57A7F2ED240F634439C42CF
:101470001CD804F10044A4F6B8344FEA44014FF0FC
:101480000202FFF7BDFC00286CD0002E6DD141F6A2
:101490000871C2F20101BDF80E2021F814202B685A
:1014A00003F101032B604FF0010063E04FF00203F2
:1014B00000934FF001000190284640F6B8310DF13D
:1014C0000E02FFF72FFF55E0A4F5BB50A0F110006E
:1014D000B0F57A7F0FD24EF69002C7F6FF72A118D0
:1014E0004FEA41004FF001010DF10E024FF00203EF
:1014F000FFF7C2FE3EE0A4F5DA53A3F11803B3F5FB
:101500007A7F0ED24EF2A840C7F6FF7023184FEA3A
:1015100043004FF002010DF10E020B46FFF7ACFE47
:1015200028E0A4F5FA52B2F57A7F21D24FEA4401BD
